:020000040800F2
:10200000C09E002095AB010875AC010835A60108FB
:1020100079AC01087DAC010881AC0108000000002A
:1020200000000000000000000000000085AC010876
:1020300089AC0108000000008DAC0108EBA6010886
:1020400091AC010895AC010899AC01089DAC010860
:10205000A1AC0108A5AC0108A9AC010857A601086C
:10206000BFA60108ADAC01085BA60108D9A601080E
:10207000B1AC0108B5AC0108E3A60108E7A6010868
:10208000B9AC0108BDAC0108C1AC0108C5AC010880
:10209000C9AC0108CDAC0108D1AC010877A6010894
:1020A000D5AC0108D9AC0108DDAC0108E1AC0108F0
:1020B000E5AC0108E9AC010839A60108EDAC01085E
:1020C000F1AC0108D1B40008D9B40008F5AC01089E
:1020D000F9AC0108D5A60108FDAC010801AD010865
:1020E000B1A6010805AD010809AD01080DAD010853
:1020F00051A6010811AD010815AD010819AD01087F
:102100001DAD010821AD010841A6010825AD01085A
:10211000DFA6010829AD01082DAD010849A6010877
:1021200031AD010835AD0108F3A60108EFA601089D
:1021300000F5E0700268914203D343681A4491426B
:1021400002D380680028F5D170471849086880B923
:102150004FF4805048604FF480324FF0FF30C86039
:1021600008610420124B8A604861C3F8BC01114821
:1021700008600120704701F1080313F0070F0EBF3C
:102180000023C3F1080303F007031944D21A816145
:10219000C26042F001034B60091D4FF0280C41F86A
:1021A00002C0024A1369C361704700000C7E002020
:1021B000A87300206859883C2DE9F04705460E4673
:1021C00091467068C10706EB09083AD4346810F0EC
:1021D000030F00F042826042296906448E42A14406
:1021E000C0F037826869864200F0BC80E4081F2C8A
:1021F00055D8D6F80CA0B768564508BF01F00AFEBE
:10220000BE4208BF01F006FE7068C008C000B0EB17
:10221000C40F18BF01F0FEFD05F1280000EBC4005B
:10222000874205D029698F4236D3FA68B24233D14A
:10223000BA4523D12868012101FA04F420EA0404F4
:102240002C6029698845C0F00482D8F80440A007B2
:1022500000F16081AA69904540F09780E8684844A1
:10226000E860AE6140F0010070606869864240F04D
:10227000F48100216961A960BDE8F087824506D03C
:102280002869824508D3DAF80810B14204D1C7F8AA
:102290000CA0CAF80870D4E701F0BCFDD1E7F468DF
:1022A000B769B4420BD0B068884222D3C168B1424A
:1022B00004BFA268B2421CD1C460A0601BE006F15A
:1022C0001402146834B906F1100214689CB101E0DC
:1022D0001A46146804F114031868002802BF04F1B8
:1022E000100318680028F3D18A4202D3002111603C
:1022F00001E001F08FFD002FA3D0F16905F5987082
:1023000000EB81000268964209D10460200011D1DF
:10231000F0696968012282409143696091E7286908
:10232000874205D33969B14214BF7C613C6101E049
:1023300001F070FD002C84D029698C42ACD3A761D8
:10234000306928B1884226BF2061846101F062FDB6
:10235000706900283FF475AF296988429CD3606199
:1023600084616EE798F8040000F0030003287FF40E
:1023700068AFC5F8089049F00101D8F8040040089A
:102380004000C8F8040071600AE0686980450BD11C
:10239000A9686E618944C5F8089049F00100706031
:1023A00046F80990BDE8F087E408E400A144E40899
:1023B0001F2C3AD8D8F80CA0D8F80870D04508BF20
:1023C00001F028FDB84508BF01F024FDD8F804004D
:1023D000C008C000B0EBC40F18BF01F01BFD05F131
:1023E000280000EBC400874207D029698F42C0F063
:1023F0008380FA68424540F07F80BA4507D128685B
:10240000012101FA04F420EA04042C6076E08245FC
:1024100006D0286982456FD3DAF8081041456BD1A0
:10242000C7F80CA0CAF8087068E0D8F80C40D8F8D3
:10243000187044450CD0D8F80800884222D3C168EF
:10244000414504BFA26842451CD1C460A0601BE0A6
:1024500008F11402146834B908F1100214689CB130
:1024600001E01A46146804F114031868002802BF3A
:1024700004F1100318680028F3D18A4202D3002126
:10248000116001E001F0C6FC002F37D0D8F81C1015
:1024900005F5987000EB8100026890450AD1046050
:1024A000200012D1D8F81C006968012282409143B3
:1024B000696023E02869874205D33969414514BF23
:1024C0007C613C6101E001F0A5FCBCB129698C4252
:1024D00012D3A761D8F8100028B1884226BF206126
:1024E000846101F097FCD8F8140038B1296988425A
:1024F00002D36061846101E001F08CFC49F00100CD
:10250000706046F8099069698E420CD1C5F8089050
:10251000BDE8F08764086400C8F8044049F0010091
:10252000706046F809904FEAD9071F2F23D805F1AC
:10253000280000EBC704A046B9F1100F38BF01F026
:1025400069FC286820FA07F1CA0705D4012101FABD
:1025500007F707432F6006E0A068296988422CBF6F
:10256000804601F057FCA660C8F80C60C6F80880E9
:10257000F460BDE8F0875FEA192008BF002123D08E
:10258000B0F5803F28BF1F211ED2A0F58072120C2B
:1025900002F008029040A0F58051090C01F00401FE
:1025A0008840A0F580431B0CC2F10E0203F0020329
:1025B000521AD21A984002EBD032D01D29FA00F1FB
:1025C00001F0010101EB420105F59872002302EBD5
:1025D0008100F161736133616A6822FA01F3DC07FB
:1025E00007D4012303FA01F1114369600660B06169
:1025F0001DE002681F291DBF4908C1F1190109FA30
:1026000001F1494600E002465068C008C000484554
:1026100011D002F11003C80F03EB800349001868C2
:102620000028F0D12869834213D31E60B261F6609E
:10263000B660BDE8F087296990688A4228BF884261
:1026400007D3C6609660B060F2600020B061BDE85C
:10265000F087BDE8F04701F0DDBBBDE8F087000082
:102660002DE9F84F84B00646AFF30080F52E1E4DDD
:1026700080F00F820B2E31BF10260B36F608F600C5
:102680002868F408E04010F0030F4AD0C04300F07F
:102690000100041905F1280000EBC408E700D8F890
:1026A00008607068C008C000B84218BF01F0B2FBF3
:1026B000D6F80890464508BF01F0ACFB4E4508BF70
:1026C00001F0A8FB7068C008C000B84218BF01F054
:1026D000A1FBC8450AD12868012101FA04F420EAC7
:1026E00004042C6010E000BFA87300202869814515
:1026F00008D3D9F80C10B14204D1C8F80890C9F831
:102700000C8001E001F086FB47F00300311D706092
:10271000301DCA5942F00102C25106F1080800F00A
:1027200010BFA968B14280F09F83002800F0A2800A
:102730004FF0010808FA04F1490000FA04F4484295
:1027400001430C4060420440641E200B00F0100066
:10275000C440610901F00801CC40A20802F0040263
:10276000D440630803F002030818DC401018C4F3D7
:10277000400718183818FC40241805F1280000EB11
:10278000C40AE700DAF80890D9F80400C008C000CD
:10279000B84218BF01F03EFBD9F808B0D14508BFD8
:1027A00001F038FBD94508BF01F034FBD9F804002B
:1027B000C008C000B84218BF01F02CFBDA4506D1B2
:1027C000286808FA04F420EA04042C600DE0296962
:1027D0008B4508D3DBF80C00484504D1CAF808B093
:1027E000CBF80CA001E001F015FBBF1B46F0030085
:1027F00009F10402C9F8040047F00101915109EB05
:1028000006020192D751AC684FEAD40ABAF11F0F01
:1028100088BF01F0FFFA34B3CDF800A005F128001D
:102820006E6900EBCA0AD346102C38BF01F0F2FAE9
:102830002968009821FA00F2D30704D408FA00F0BE
:102840000843286007E0DAF80800296988422CBFAD
:10285000834601F0DFFACAF80860CBF80C60C6F8CE
:1028600008B0C6F80CA0AF6009F1080801986861CB
:1028700000F067BE6868002800F0178341420840F6
:10288000401E010B01F01001C840420902F008028D
:10289000D040830803F00403D840440804F0020445
:1028A0005118E0405918C0F34007611805F59878B1
:1028B0007918F840401858F820104868C008C0003F
:1028C0008A46A0EB060B08E001464868C008C00035
:1028D000801B58453CBF83468A4608690028F3D1CF
:1028E00049690029F1D128698245C0F0CF80DAF822
:1028F0000410C90806EB0B09C900494518BF01F0CF
:1029000089FA0AEB06008245019080F0BF80DAF870
:102910000C40DAF8187054450DD0DAF8080029692F
:10292000884223D3C268524504BFA16851451DD1D6
:10293000C460A0601CE00AF114010C6834B90AF10B
:1029400010010C68A4B101E011460C6804F11402F6
:102950001068002802BF04F1100210680028F3D1AB
:102960002869814202D300220A6001E001F052FA94
:10297000002F34D0DAF81C0008EB800001688A458B
:1029800009D1046094B9DAF81C0069680122824018
:102990009143696023E02869874205D3396951452D
:1029A00014BF7C613C6101E001F034FABCB12969DB
:1029B0008C4212D3A761DAF8100028B1884226BFF2
:1029C0002061846101F026FADAF8140038B129692F
:1029D000884202D36061846101E001F01BFABBF11F
:1029E000100F0ED249F003000AF10401CAF80400E6
:1029F0000AF1040051F8092042F0010240F80920D0
:102A00003EE046F003010AF10402CAF804104BF05C
:102A100001009051019941F80BB0A8680090C408DA
:102A20001F2C88BF01F0F6F9009828B305F12800A3
:102A300000996F6900EBC408C146102938BF01F046
:102A4000E9F9286820FA04F1CA0705D4012101FA3E
:102A500004F404432C6007E0D8F808002969884290
:102A60002CBF814601F0D6F9C8F80870C9F80C707F
:102A7000C7F80890C7F80C80C5F808B001986861DD
:102A80001AF1080800F0F08100F05BBD01F0C2F916
:102A9000EAE116F1400F28BF4FF0FF3680F0E481E5
:102AA0000B36F6086B68F600002B00F0DD8100277E
:102AB000300AC6F1000908BF002423D0B0F5803FDA
:102AC00028BF1F241ED2A0F58071090C01F0080157
:102AD0008840A0F58052120C02F004029040A0F54C
:102AE0008044240CC1F10E0104F00204891A091B70
:102AF000A04001EBD031C81D26FA00F404F0010417
:102B000004EB410405F5987858F8240030B31F2CE5
:102B10000FBFB4464FEA540CCCF1190C06FA0CFC6A
:102B2000BE46494601E04FEA4C0C4268D208D2004A
:102B3000921B8A4202D2110007460CD04269103023
:102B40004FEADC7950F82900002A1CBF82429646E1
:102B50000028E8D170468946A8BBB7BB012101FA1D
:102B600004F4640060420443234000F07D81584235
:102B700003405B1E180B00F01000C340590901F020
:102B80000801CB409A0802F00402D3405C0804F02C
:102B900002040818E3401018C3F3400C20186044E6
:102BA00023FA0CF31B1858F823000CE00846416880
:102BB000C908C900891B49453CBF894607460169C8
:102BC0000029F3D140690028F1D1002F00F04C8199
:102BD000A868801B814580F0478129698F42FFF4F6
:102BE00055AF7868C008C00006EB0901884218BFDD
:102BF00001F010F907EB060B5F45BFF447AFFC6827
:102C0000D7F818A0BC420CD0B8682969884223D3F1
:102C1000C268BA4204BFA168B9421DD1C460A060B5
:102C20001CE007F114010C6834B907F110010C68BD
:102C3000A4B101E011460C6804F1140210680028E8
:102C400002BF04F1100210680028F3D12869814204
:102C500002D300220A6001E001F0DCF8BAF1000FB3
:102C600034D0F86908EB800001688F4208D1046015
:102C7000A4B9F8696968012282409143696025E03E
:102C80002869824508D3DAF81010B94214BFCAF88F
:102C90001440CAF8104001E001F0BCF8B4B1296951
:102CA0008C4211D3C4F818A0386928B1884226BFD5
:102CB0002061846101F0AEF8786938B129698842F1
:102CC00002D36061846101E001F0A4F8B9F1100F52
:102CD0000CD2B14449F00300391D7860381D51F819
:102CE000092042F0010240F80920B9E046F0030152
:102CF0003A1D796049F0010090514FEAD9004BF834
:102D000009901F2822D805F1280101EBC004296889
:102D100021FA00F2D307A04605D4012202FA00F0FE
:102D20000843286006E0A068296988422CBF8046D5
:102D300001F070F8C4F808B007F10800C8F80CB04A
:102D400040F8068007F10C018C5189E05FEA1920F8
:102D500008BF002123D0B0F5803F28BF1F211ED21D
:102D6000A0F58072120C02F008029040A0F580518C
:102D7000090C01F004018840A0F580431B0CC2F14E
:102D80000E0203F00203521AD21A984002EBD0321C
:102D9000D01D29FA00F101F0010101EB420107F118
:102DA0001403CBF81C1000229A5107F1100308EB12
:102DB00081009A516A6822FA01F3DC0711D40123D9
:102DC00003FA01F111436960C0F800B0CBF81800B4
:102DD00007F1080107F10C0040F806B041F806B011
:102DE0003EE002681F291DBF4908C1F1190109FA17
:102DF00001F1494600E002465068C008C00048455D
:102E000018D002F11003C80F03EB800349001868C3
:102E10000028F0D12869834220D3C3F800B007F11D
:102E20000C01CBF8182041F806B007F1080040F873
:102E300006B015E0296990688A4228BF88420DD300
:102E4000C0F80CB007F10801C2F808B0885107F1CA
:102E50000C0082510022CBF8182001E000F0DAFFCC
:102E600017F1080840F06D83A868B0421DD3811B9C
:102E70006A6910290AD390196861A96041F00103B9
:102E80004360415046F0030656600BE00021A96004
:102E90006961131D40F003015160111D1C5844F07D
:102EA00001040C5002F108084BE3E8688642C0F0C8
:102EB0003883DFF8B89BD9F8000008B9FFF745F967
:102EC000D9F8081088192F30491E20EA01018E42D6
:102ED00080F0358305F5D877B86838B13A68891835
:102EE0008A4280F02C838842C0F0298300F0B2FF30
:102EF00000281CBFD0F8008010F1010F00F01F83E4
:102F000039687A68414439608A4238BF7960AC696F
:102F100004BB296909B1884200D2286100213861C7
:102F2000C7F81480F9614FF0FF31D9F800206A62C8
:102F3000296205F128020021D260926002F10804A2
:102F400054611461891C10321F29F5D9A8F1280297
:102F500001461DE005F5E0710A46814600E09268F1
:102F6000D2B11068536803449945F8D1107B030728
:102F700012D413689C420FD3D2F804C063449C421D
:102F80000AD2C444C2F804C02146E86808EB000233
:102F90002846FFF7F0F8C1E22869814538BFC5F837
:102FA000109009EB080000E08968002900F0BD815D
:102FB0000A688242F8D1087B020700F1B6810868EE
:102FC000C1F800904A6842444A6009F1080111F0D2
:102FD000070F08BFCDF8049006D0C1F1080101F039
:102FE000070109EB0102019200F1080111F0070F3E
:102FF00004D0C1F1080101F007010844804601989E
:10300000A8EB00018419A1EB060B274646F0030646
:103010004660474528BF00F0FDFE98F80400C10750
:1030200058BF00F0F7FEBBF1100F38BF00F0F2FE02
:10303000A869804508D1E9688B44C5F80CB0AF6138
:103040004BF0010078606CE1686980450AD1A9689D
:103050008B44C5F808B06F614BF00100786047F809
:103060000BB05EE1D8F8040000F00301012940F044
:10307000B880C008C000C1081F29039040D8D8F804
:1030800008200092D8F80C600291B04508BF00F00B
:10309000C1FE0098804508BF00F0BCFED8F80400CF
:1030A0000299C008C000B0EBC10F18BF00F0B2FE1B
:1030B0000299009A05F1280000EBC100824208D075
:1030C00011462A699142C0F08780CA68424540F0A3
:1030D000838000998E4206D102982A68012383409A
:1030E0009A432A607AE0864205D029698E4273D3DA
:1030F000B068404570D10098C6600099B1606DE03D
:10310000D8F818000090D8F80C6046450DD0D8F8D3
:1031100008002969884223D3C268424504BFB168C8
:1031200041451DD1C660B0601CE008F114010E6875
:1031300036B908F110010E68A6B101E011460E681B
:1031400006F114021068002802BF06F11002106890
:103150000028F3D12869814202D300220A6001E0ED
:1031600000F058FE0098002838D0D8F81C0005F56B
:10317000987101EB80000168884509D106609EB90D
:10318000D8F81C006968012282409143696025E0FB
:1031900000982969884205D30169414514BF4661F9
:1031A000066101E000F036FEC6B129698E4213D3F4
:1031B0000098B061D8F8100028B1884226BF30616D
:1031C000866100F027FED8F8140038B129698842DA
:1031D00002D37061866101E000F01CFE039988440F
:1031E0008B44D8F8041049084900C8F804104BF083
:1031F000010078604FEADB0647F80BB01F2E22D89B
:1032000005F1280000EBC604A146BBF1100F38BF42
:1032100000F000FE286820FA06F1CA0705D4012153
:1032200001FA06F606432E6006E0A0682969884286
:103230002CBF814600F0EEFDA760C9F80C70C7F8FE
:103240000890FC606DE05FEA1B2008BF002123D0DE
:10325000B0F5803F28BF1F211ED2A0F58072120C4E
:1032600002F008029040A0F58051090C01F0040121
:103270008840A0F580431B0CC2F10E0203F002034C
:10328000521AD21A984002EBD032D01D2BFA00F11C
:1032900001F0010101EB4201F961002305F598728B
:1032A0007B6102EB81003B616A6822FA01F3DE0771
:1032B00007D4012303FA01F1114369600760B86183
:1032C0001DE002681F291DBF4908C1F119010BFA51
:1032D00001F1594600E002465068C008C000584558
:1032E00010D002F11003C80F03EB800349001868E7
:1032F0000028F0D12869834211D31F60BA61FF60B2
:10330000BC600EE0296990688A4228BF884206D3D3
:10331000C7609460B860FA600020B86101E000F016
:1033200079FD019800F108080BE121462846FEF7D7
:10333000FFFE0168406808440090A0F1270111F0E9
:10334000070000980EBF0021C1F1080101F007013C
:103350000844A0F12F0B04F110018B4538BFA346A0
:103360000BF11802002102920191A8F128024946AE
:103370002846FEF700FF0BF1080010F0070F18BFFA
:1033800000F048FD1B20CBF8040005F5E07292E840
:1033900009500BF1080181E8095000210BF10800E8
:1033A000F961B861009A02980199C7F81090C7F8BE
:1033B0001480072300E0001D491C00F10807974214
:1033C0004360F8D30129D8BF00F024FDA34500F0E5
:1033D000A580ABEB040B201D221D50F80B104908F3
:1033E000490042F80B104BF0010060604FEADB0926
:1033F00044F80BB0B9F11F0F22D805F1280000EBFB
:10340000C907B846BBF1100F38BF00F003FD2868AC
:1034100020FA09F1CA0705D4012101FA09F108438C
:10342000286006E0B868296988422CBF804600F011
:10343000F1FCBC60C8F80C40C4F80880E7606DE09F
:103440005FEA1B2008BF002123D0B0F5803F28BFD2
:103450001F211ED2A0F58072120C02F008029040CB
:10346000A0F58051090C01F004018840A0F58043CB
:103470001B0CC2F10E0203F00203521AD21A98403A
:1034800002EBD032D01D2BFA00F101F0010101EB6B
:10349000420105F59872002302EB8100E16163614E
:1034A00023616A6822FA01F3DF0707D4012303FAD4
:1034B00001F1114369600460A0611DE002681F29E9
:1034C0001DBF4908C1F119010BFA01F1594600E08D
:1034D00002465068C008C000584510D002F11003E1
:1034E000C80F03EB8003490018680028F0D1286951
:1034F000834211D31C60A261E460A4600EE02969DC
:1035000090688A4228BF884206D3C4609460A06055
:10351000E2600020A06101E000F07CFCE8688642E7
:103520000DD2801BA969E8608A19AA6140F00100E8
:10353000506046F003064E6001F1080801E04FF0CC
:103540000008AFF30080404605B0BDE8F08F0028CA
:1035500000D170472DE9F047A0F10805AFF30080D6
:10356000DFF8A46831698D42C0F07A82686800F0A3
:103570000302012A00F07482C2084FEAC209C2079E
:1035800005EB090839D42C6810F0030F00F06A82AB
:10359000604205448D42A144C0F062827069854258
:1035A00000F0DA80E408202C72D2D5F80CA0AF68C5
:1035B000554508BF00F02EFCBD4208BF00F02AFCB4
:1035C0006868C008C000B0EBC40F18BF00F022FC50
:1035D00006F1280000EBC400874205D031698F4214
:1035E00053D3FA68AA4250D1BA4540D1306801217C
:1035F00001FA04F420EA04043460454580F0308286
:10360000D8F80440E00740F12B82A10700F17C814B
:10361000B069804540F0B380F168B5618944C6F86F
:103620000C9049F00100686071698D4202D1002060
:103630007061B060F169494580F01482DFF82C2494
:10364000106808B9FEF781FDB169002900F00A820F
:10365000F068292824BF3046FEF76AFDF069F1685A
:10366000884280F0FF814FF0FF30F061FAE182453F
:1036700006D03069824508D3DAF80810A94204D18F
:10368000C7F80CA0CAF80870B7E700F0C3FBB4E7AE
:10369000EC68AF69AC420BD0A868884222D3C168FD
:1036A000A94204BFA268AA421CD1C460A0601BE06A
:1036B00005F11402146834B905F1100214689CB1C4
:1036C00001E01A46146804F114031868002802BFC8
:1036D00004F1100318680028F3D18A4202D30021B4
:1036E000116001E000F096FB002F86D0E96906F535
:1036F000987000EB81000268954209D104602000B7
:1037000011D1E8697168012282409143716074E7C8
:103710003069874205D33969A94214BF7C613C6195
:1037200001E000F077FB002C3FF467AF31698C4279
:10373000ABD3A761286928B1884226BF2061846184
:1037400000F068FB686900283FF457AF3169884290
:103750009BD36061846150E798F8040000F0030097
:1037600003287FF44AAFC6F8089049F00101D8F861
:10377000040040084000C8F8040069600AE070696D
:1037800080450AD1B16875618944C6F8089049F04E
:103790000100686045F8099064E1E408E400A14490
:1037A000E408202C3AD2D8F80CA0D8F80870D045FC
:1037B00008BF00F02FFBB84508BF00F02BFBD8F87E
:1037C0000400C008C000B0EBC40F18BF00F022FB1B
:1037D00006F1280000EBC400874207D031698F4210
:1037E000C0F08580FA68424540F08180BA4507D133
:1037F0003068012101FA04F420EA0404346078E01E
:10380000824506D03069824571D3DAF80810414507
:103810006DD1C7F80CA0CAF808706AE0D8F80C405F
:10382000D8F8187044450DD0D8F80800316988429E
:1038300023D3C268424504BFA16841451DD1C4607D
:10384000A0601CE008F114010C6834B908F1100103
:103850000C68A4B101E011460C6804F11402106870
:10386000002802BF04F1100210680028F3D130696B
:10387000814202D300220A6001E000F0CBFA002F5F
:1038800037D0D8F81C1006F5987000EB810002685C
:1038900090450AD10460200012D1D8F81C0071684C
:1038A000012282409143716023E03069874205D351
:1038B0003969414514BF7C613C6101E000F0AAFA1E
:1038C000BCB131698C4212D3A761D8F8100028B17D
:1038D000884226BF2061846100F09CFAD8F8140069
:1038E00038B13169884202D36061846101E000F03F
:1038F00091FA49F00100686045F8099071698D42BC
:103900000BD1C6F80890ADE064086400C8F8044024
:1039100049F00100686045F809904FEAD907202F67
:1039200022D206F1280000EBC704A046B9F1100F1F
:1039300038BF00F06FFA306820FA07F1CA0705D4E3
:10394000012101FA07F70743376006E0A0683169F3
:1039500088422CBF804600F05DFAA560C8F80C5084
:10396000C5F80880EC607DE05FEA192008BF0021FF
:1039700023D0B0F5803F28BF1F211ED2A0F5807252
:10398000120C02F008029040A0F58051090C01F0E1
:1039900004018840A0F580431B0CC2F10E0203F025
:1039A0000203521AD21A984002EBD032D01D29FAE3
:1039B00000F101F0010101EB420106F598720023CC
:1039C00002EB8100E9616B612B61726822FA01F3FD
:1039D000DC0707D4012303FA01F11143716005608C
:1039E000A8611DE002681F291DBF4908C1F1190126
:1039F00009FA01F1494600E002465068C008C000DB
:103A0000484510D002F11003C80F03EB80034900B2
:103A100018680028F0D13069834211D31D60AA6173
:103A2000ED60AD600EE0316990688A4228BF88423F
:103A300006D3C5609560A860EA600020A86101E037
:103A400000F0E8F9306A401E30620BD1D6F8C801A8
:103A500000E080680028FCD14FF0FF30306201E0C8
:103A600000F0D8F9AFF30080BDE8F0870C7E0020AD
:103A70002DE9F84F0F4606467B6831690024D808C7
:103A8000C0008F428146C0F07A8103F00305012D0A
:103A900000F0758107EB090A574580F07081DAF86C
:103AA00004B05FEACB7540F16A8113F0030F15464D
:103AB0000FD1E908202924BF2A1D9042C0F061815E
:103AC000DFF848138A685200451BAA42C0F05981AA
:103AD00053E1A9451CD3A9EB0504102CC0F04D817E
:103AE00003F001032B4343F0020379197B6044F098
:103AF0000302486840F0010048604A600819224605
:103B0000436843F0010343603046FEF755FB34E160
:103B1000B269924516D1F0684844854280F03181FF
:103B200003F00103441B2B4343F0020378197B602D
:103B300044F00102416841F0010141604260B0611E
:103B4000F4601AE1706982452FD1B0688144A945BB
:103B5000C0F01781A9EB0501102903F0010314D36C
:103B600078191D4345F002057D604218436843F013
:103B70000103436041F001044460415053685B0815
:103B80005B005360B1607061F7E049EA030343F002
:103B90000203381D7B603A1D50F8091041F0010105
:103BA00042F80910B4607461E7E05FEA8B7000F1DD
:103BB000E8804FEADB00C2009144A945C0F0E180F3
:103BC0004FEAD20BA9EB0500BBF1200F00903BD2CE
:103BD000DAF80C40DAF80880A24508BF00F01AF9BC
:103BE000C24508BF00F016F9DAF80400C008C000AA
:103BF000B0EBCB0F18BF00F00DF906EBCB0000F1D6
:103C00002801884508D032699045C0F08980D8F8ED
:103C10000C10514540F08480444506D130680122A3
:103C200002FA0BF1884330607CE000F128018C42FD
:103C300005D03069844273D3A168514570D1C8F86A
:103C40000C40C4F808806DE0DAF80C40DAF818800F
:103C500054450CD0DAF80800884222D3C168514597
:103C600004BFA26852451CD1C460A0601BE00AF1E9
:103C70001402146834B90AF1100214689CB101E00E
:103C80001A46146804F114031868002802BF04F1EE
:103C9000100318680028F3D18A4202D30021116072
:103CA00001E000F0B7F8B8F1000F3BD0DAF81C00E3
:103CB00006EB800101F59870026892450AD1046014
:103CC000200015D1DAF81C0071680122824091436E
:103CD000716027E03069804508D3D8F8101051454D
:103CE00014BFC8F81440C8F8104001E000F092F882
:103CF000C4B131698C4213D3C4F81880DAF81000CB
:103D000028B1884226BF2061846100F083F8DAF888
:103D1000140038B13169884202D36061846101E0E6
:103D200000F078F800981028387900F001000DD2E2
:103D300049EA000040F0020078603A1D381D50F852
:103D4000091041F0010142F8091016E0284340F043
:103D5000020078607919486840F0010048600098D6
:103D600040F00300486000980844426842F00102B5
:103D700042603046009AFEF71FFA3C4601E000F030
:103D800049F82046BDE8F28F70B505460E4600247E
:103D900025B93046FEF764FC044632E016F1400FC8
:103DA0002FD20B2E31BF102406F10B04E408E400DF
:103DB000AFF3008001232246A5F10801DFF850008F
:103DC000FFF756FE0446AFF300800CB1083418E04C
:103DD0003046FEF745FC040013D055F8042C12F0D1
:103DE000030F0CBF08200420D208D200121AB242DE
:103DF00088BF32462946204600F042F82846FFF7A1
:103E0000A6FB204670BD0000A87300200C7E002099
:103E1000A8730020012000F093B830B4002513E00F
:103E200050F8042BD30744BFA9F101039A18091FC6
:103E3000042942F8045BFAD213468C0744BF15806C
:103E40009B1CC90748BF1D7050F8041B0029E7D10F
:103E500030BC70470749086808B100207047064821
:103E6000C008C00008600549C908C900091A0160F6
:103E7000704700BFB07E0020C79E0020C0BE00205B
:103E800062B38B0708D0521E11F8013B00F8013BCA
:103E900000F024808B07F6D1830740F0208000BF1C
:103EA000103A07D330B4B1E83810103AA0E838100F
:103EB000F9D230BC530724BFB1E80810A0E80810BD
:103EC00044BF51F8043B40F8043BD20724BF31F80B
:103ED000022B20F8022B44BF0B7803707047121F8F
:103EE00017D35B0009D151F8043B20F8023B1B0CAF
:103EF000121F20F8023BF6D20BE051F8043B00F809
:103F0000013B1B0A20F8023B1B0C121F00F8013B6F
:103F1000F3D238BF121D521E24BF11F8013B00F826
:103F2000013BF8D870478268521C8260426832B107
:103F30000268531C036011704168491E416070475C
:103F400080B5AFF30080024A11001820ABBEFBE73A
:103F50002600020010B501F020F9DFF87C4B617BF0
:103F6000084301D100F0D2BDA07850B904F170002F
:103F700001F0FEFA207920B901F06AFC08B900F0DE
:103F8000F8BDBDE8104072E3DFF84C0B017881B05A
:103F90000846009101B0704780B5DFF83C1B002057
:103FA000087302F098F918E138B504460D46DFF8B9
:103FB000281BDFF8CC0B05224A70543182689047E9
:103FC00029462046BDE8344001F0D0B910B5DFF8ED
:103FD000084B01212173002001F068FA04F1E80088
:103FE000BDE81040DFF8F42ADFF8981B01F089BA29
:103FF000DFF8940B01F02FB9DFF8DC1A8862704704
:10400000DFF8D41AC8627047DFF8CC1A086370472B
:10401000DFF8C41A48637047DFF8BC1A886370473A
:10402000DFF8B41AC8637047DFF8AC1A0864704749
:10403000DFF8A41A48647047DFF89C1A8864704758
:1040400070B5044602F012FA002818BF002C04D004
:10405000DFF8841A0120087113E070BD70B5DFF835
:10406000785A05210446002068626970EC6402F009
:10407000FDF9002818BF002C02D00120287100E0B3
:1040800070BD0025264605E016F8011BE8B201F0D8
:10409000A4F96D1C204602F0D9FD8542F4D3BDE899
:1040A0007040002001F0C7B910B5DFF82C4A00209D
:1040B000207102F0DBF9E0B1E06C10B1FFF7C0FF56
:1040C00003E001F0E2F90020E06403F035F810B1FC
:1040D00000F040F809E000F06DFEDFF8B02ADFF8EC
:1040E0003C1C04F1700001F00CFABDE8104003F034
:1040F00061B910BD70B50C461546DFF8DC690021CA
:10410000052271627270FFF79BFF0DB10020F06411
:10411000224606F1D000BDE87040DFF8401C01F0F7
:10412000F0B910B5044602F0A1F918B9200010D07A
:10413000A04710BDDFF8A009417803291EBF02295E
:1041400005214170002242622046BDE8104001F086
:104150009CB910BD80B5DFF880090021C1640171F0
:1041600004F0A1FA10B104F0AAFA01E04FF4FA70D9
:10417000DFF8001BA1F88400DFF8A40B0268012A15
:10418000ACBFDFF8A00BDFF8580C24E010B50446F4
:1041900002F0D2FF10B1BDE81040DBE72046BDE8D9
:1041A00010405BE780B502F0C7FF08B100F0FEBD2C
:1041B000DFF824090021C164017104F074FA10B120
:1041C00004F07DFA01E04FF4FA70DFF8A81AA1F8C4
:1041D0008400DFF8AC0B00F00EFEBDE802400020CA
:1041E00000F02FBE10B500F0DCFFDFF8EC482079BE
:1041F000B8B96078042807D1002000F022FE03201F
:1042000000216070616210BD01F022FB48B904F129
:104210007000BDE81040DFF8C428DFF8001B01F093
:1042200070B910BDF1B5DFF8B048216C82B000293B
:104230001FBF9DF808200F2A02A8884701F099FAAD
:1042400000281EBF9DF808000F2801F09EFA01F01B
:10425000DAFA38B19DF80800226A2070002104F1D2
:104260001000904701F0FFFA00281CBF9DF80800DD
:104270000F2806D00121A17004F1700001F078F937
:10428000EBE1207900289DF8080019D00A2800F0F9
:10429000DD800B2817D00C2800F097810D2800F046
:1042A000C5804CF250320FF6390104F1580001F08C
:1042B00028F9DFF8B82BDFF8B81B04F17000D2E161
:1042C0000B2840F0B18004F08BFD60B105F0BFFC1D
:1042D000002839D1606A42F21071884234D280B22B
:1042E00004F081FD30E001F09DFA28B1606A01F030
:1042F00063FA00283FD170E001F089FA18B1606AD2
:1043000004F040FA6CE16078032808D101F0A0FACB
:1043100028B1606A01F0B5FA0020606260E1606A6D
:10432000E0B903F06AFEA0B103F067FE4FF6FF713B
:1043300088421CBF606B00280BD003F067FE00288A
:1043400040F04E81616B88470020052160626170FA
:1043500046E10020FFF7E5FE01200DE0617801292C
:104360000CD1DFF8B81BDFF8B82B0918914258D3ED
:10437000E16A01B188470520607031E103290FD15E
:10438000A16C002900F02C81C0B2884728B1002020
:10439000E064FFF789FE05206070002161621FE183
:1043A00002290AD1A26A002A00F01A8142F2107191
:1043B000884280F01581216D29E003F05FFE80B115
:1043C000606A42F2107188420BD203F063FED8B1EA
:1043D000022060700020616A21656062FFF7A1FE23
:1043E000FEE0606ADFF8501BDFF8502B091891429D
:1043F00002D2E16A8847F3E042F21072904208D29A
:10440000A06A002800F0EC80606AA26A0021904750
:10441000E6E0DFF8081BDFF8083B0918994280F056
:10442000DF8000F081FCDBE00D280DD1A06B0028BF
:1044300000F0D6806F2005F0A7F9002800F0D080AA
:10444000A16B00208847C3E00A2823D10021E16442
:1044500002F06CFE10B1FFF7A5FE11E060780328B2
:1044600003D00020FFF720FE0AE002F065FE10B145
:10447000FFF770FE04E000F09DFC002000F0E1FC7E
:10448000002060620521E06B6170002800F0A880C8
:104490008047A5E0064601F0E9FF002800F095807E
:1044A0000A2E80F2928001F064F9012508B101F032
:1044B0006CF901F0CDF998B304F1700001F058F8EF
:1044C0002021002000F089FF0021002000F0A5FF3E
:1044D0002021012000F081FF0021012000F09DFF3C
:1044E0002021022000F079FF0021022000F095FF3A
:1044F0002021032000F071FF0021032000F08DFF38
:104500002021042000F069FF0021042000F085FF35
:104510002021052000F061FF0021052000F07DFF33
:10452000616ADFF8480981424FD2009105E00098A6
:104530000A22B0FBF2F200926D1C00980028F6D11E
:10454000607801EB810206EB42010128616216D11D
:104550006F1E3036F1B2F8B200F03FFF012D04DDDE
:10456000A81E2A21C0B200F038FFE77004F18800CD
:10457000DFF818260FF2E97100F0C3FF22E00026F1
:10458000002D1FDD304605F06FFC02460B46002073
:10459000DFF8101B05F07AFC06F022F8616AB1FB27
:1045A000F0F10A20B1FBF0F000EB8002A1EB420138
:1045B0003031C6F10500C9B2C0B200F00EFF761C62
:1045C000AE42DFDB002000F036FF01F041F938B9E0
:1045D000DFF89828DFF8981804F1700000F091FFD8
:1045E0000120A070002000F0B6FEE071002000F075
:1045F000B6FE2072E8B1A07A002804BF606A0028E5
:1046000017D103F0FAFCA0B103F0F7FC4FF6FF71ED
:1046100088421CBF606B00280BD003F0F7FC40B150
:104620009C2005F0B1F8C0B10120A07204F584719E
:104630000FE0E07988B1A079002804BF606A002803
:104640000BD1652005F0A0F838B10120A07104F568
:104650008071DFF8540A05F0D7FF4CF250320FF2A8
:10466000814104F1580000F04CFF03B0F0BDFEB5ED
:10467000DFF86444607B002800F022820021DFF82C
:104680002C0A61730278216C8DF8002000291EBF6E
:104690000F2A6846884701F06CF800281EBF9DF875
:1046A00000000F2801F071F801F0ADF838B19DF865
:1046B0000000226A2070002104F11000904701F0F0
:1046C000D2F800281CBF9DF800000F2806D0012159
:1046D000A17004F1700000F04BFFEAE1207900289E
:1046E0009DF8000019D00A2800F0DD800B2817D0B3
:1046F0000C2800F096810D2800F0C5804CF2503255
:104700000FF2DD3104F1580000F0FBFEDFF85C270A
:10471000DFF85C1704F17000D1E10B2840F0B180A4
:1047200004F05EFB60B105F092FA002839D1606AAE
:1047300042F21071884234D280B204F054FB30E06F
:1047400001F070F828B1606A01F036F800283FD116
:1047500070E001F05CF818B1606A04F013F86BE1E6
:104760006078032808D101F073F828B1606A01F07D
:1047700088F8002060625FE1606AE0B903F03DFC08
:10478000A0B103F03AFC4FF6FF7188421CBF606B8A
:1047900000280BD003F03AFC002840F04D81616BFB
:1047A0008847002005216062617045E10020FFF725
:1047B000B8FC01200DE0617801290CD1DFF85C170D
:1047C000DFF85C270918914258D3E16A01B18847A4
:1047D0000520607030E103290FD1A16C002900F0A1
:1047E0002B81C0B2884728B10020E064FFF75CFC51
:1047F00005206070002161621EE102290AD1A26ACF
:10480000002A00F0198142F21071884280F0148170
:10481000216D29E003F032FC80B1606A42F2107130
:1048200088420BD203F036FCD8B102206070002021
:10483000616A21656062FFF774FCFDE0606ADFF881
:10484000F816DFF8F8260918914202D2E16A884783
:10485000F2E042F21072904208D2A06A002800F002
:10486000EB80606AA26A00219047E5E0DFF8AC16B1
:10487000DFF8AC360918994280F0DE8000F054FA77
:10488000DAE00D280DD1A06B002800F0D5806F2054
:1048900004F07AFF002800F0CF80A16B0020884749
:1048A000C2E00A2823D10021E16402F03FFC10B1EC
:1048B000FFF778FC11E06078032803D00020FFF7B1
:1048C000F3FB0AE002F038FC10B1FFF743FC04E010
:1048D00000F070FA002000F0B4FA002060620521B8
:1048E000E06B6170002800F0A7808047A4E00646D6
:1048F00001F0BCFD002800F094800A2E80F2918027
:1049000000F037FF012508B100F03FFF00F0A0FFE5
:1049100098B304F1700000F02BFE2021002000F07D
:104920005CFD0021002000F078FD2021012000F036
:1049300054FD0021012000F070FD2021022000F034
:104940004CFD0021022000F068FD2021032000F032
:1049500044FD0021032000F060FD2021042000F030
:104960003CFD0021042000F058FD2021052000F02E
:1049700034FD0021052000F050FD616ADFF8EC04F1
:1049800081424ED2019105E001980A22B0FBF2F279
:1049900001926D1C01980028F6D1607801EB81022C
:1049A00006EB42010128616215D16F1E3036F1B26B
:1049B000F8B200F012FD012D04DDA81E2A21C0B2BC
:1049C00000F00BFDE77004F18800704A0FF291319E
:1049D00000F097FD22E00026002D1FDD304605F097
:1049E00043FA02460B460020DFF8B81605F04EFAEF
:1049F00005F0F6FD616AB1FBF0F10A20B1FBF0F0C1
:104A000000EB8002A1EB42013031C6F10500C9B2D2
:104A1000C0B200F0E2FC761CAE42DFDB002000F00A
:104A20000AFD00F015FF38B9DFF84024DFF8401424
:104A300004F1700000F065FD0120A070002000F07E
:104A40008AFCE071002000F08AFC2072E8B1A07AB4
:104A5000002804BF606A002817D103F0CEFAA0B185
:104A600003F0CBFA4FF6FF7188421CBF606B002841
:104A70000BD003F0CBFA40B19C2004F085FEC0B10E
:104A80000120A07204F584710FE0E07988B1A0796B
:104A9000002804BF606A00280BD1652004F074FE72
:104AA00038B10120A07104F58071DFF8FC0505F034
:104AB000ABFD4CF250320FF2290104F15800D2E55F
:104AC00001F0D4FC30B1002000F05FFBDFF8E0051E
:104AD00000F0C1FB03B0F0BD741F0020C0C62D0064
:104AE00010B500F05AFBDFF8CC45617B08430DD0D0
:104AF000A07848B904F1700000F03AFD207918B9A7
:104B000000F0A6FE00B934E0FFF73BBA00F023FC4A
:104B1000E071002000F023FCE179207209B9A1794D
:104B200011B9E0B9A07AD0B1002000F08AF9E0799B
:104B300040B9A07930B100216171A17104F1A000E8
:104B400000F016FD207A40B9A07A30B100216172E0
:104B5000A17204F1B80000F00BFD0520607004F1B3
:104B60005800BDE810404CF25032DFF84C1500F010
:104B7000C8BCBDE81040DFF84405FFF7D2BA00001A
:104B800098060020993F0008553F000820A1070023
:104B900070B501F06BFC00286BD003F01DFA0446E1
:104BA00003F011FADFF80C5500B96C716879A04276
:104BB00056DA201A401EC0B200EB4001DFF8006553
:104BC00049000020715C00F008FC6879201A411E41
:104BD000C9B201EB410206EB42020120517800F01C
:104BE000FCFB6879201A411EC9B201EB410206EBB9
:104BF00042020220917800F0F0FB6879201A411EF1
:104C0000C9B201EB410206EB42020320D17800F069
:104C1000E4FB6879201A411EC9B201EB410206EBA0
:104C200042020420117900F0D8FB6879241A621E30
:104C3000D2B202EB4203711D5B000520C95C00F09B
:104C4000CCFB002000F0F7FBDFF87824DFF87814C5
:104C500005F1A00000F055FC6879401C687170BD3A
:104C6000052169700020296B687111B1BDE87040A1
:104C7000084770BD0879002070B501F0F7FB0028E7
:104C80004BD003F0CCF9DFF82C44617A814239DA59
:104C9000401AC0B238B10B2805D2401EC0B200EB9A
:104CA00040014D0000E00025DFF82064715D002028
:104CB00000F093FB70194178012000F08EFB701911
:104CC0008178022000F089FB7019C178032000F080
:104CD00084FB70190179042000F07FFB7019417981
:104CE000052000F07AFB002000F0A5FBDFF8D423BC
:104CF000DFF8DC1304F1B80000F003FC607A401C1C
:104D0000607270BD00206072A0720520616B6070DF
:104D100009B1002088470020606270BD434E000842
:104D20006C7800207078002010B5DFF88843616C43
:104D300091B1884780B10020E06400F064FD30B993
:104D400004206070BDE81040DFF8880353E0BDE840
:104D50001040002000F0DEBF10BD0000A940000898
:104D600080B501F083FB48B1DFF84803C0782A2101
:104D700000F033FBBDE80240FFF793B901BD00002E
:104D800044AB010880B5DFF82C03052100224170F7
:104D90004262C26401F06AFB38B102F0CDF900B1A1
:104DA00004E000F007F8FFF718BA01BDBDE80140C4
:104DB000FFF7D0B938B5C84D4FF4FA70A5F88400A4
:104DC00003F071FC38B103F05FFC044603F077FC9C
:104DD000A5F8840004B9ACA42046BDE832400AE03E
:104DE00038AC010880B502F0A7F900B1DEE7FFF7A3
:104DF000E1FFFFF7F2B970B5044601F027FF054661
:104E0000B54E8021304605F01DFC802D28BF802541
:104E1000C6F88050642DC4BF6421C6F880100020FD
:104E200003E014F8011B3154401CD6F8801088426E
:104E3000F7DBA049C87A08B10022CA7270BDA64843
:104E4000704710B59B4C207B78B901F00FFB60B127
:104E5000207950B90021A17002F0BCFA28B9BDE850
:104E600010400FF2DD00FFF75CB910BDA086010015
:104E7000E54100082DE9F0418E4D297B2879014359
:104E80004AD101F0F3FA002846D002F0A3FA002834
:104E900042D105F1700000F06BFB00200121E872A7
:104EA000A97001F0E3FA002836D095F80B808A4EFD
:104EB0000027D6F88000F9B24144821D91FBF2F43C
:104EC00002FB1414315D2E2907D1F9B211B9E97A28
:104ED000491CE972641C08F10108401EA042B4BFDD
:104EE0002021315DF8B200F078FA301940782E2890
:104EF00003D10121F8B200F090FA7F1CF8B2052826
:104F0000D7DDE87AD6F88010401C491DC2B2914224
:104F1000B8BF0020E87253E0BDE8F0816079FEFF81
:104F2000A0BB0D006C49B1F884206C494FF47A7035
:104F300042436B4800F0E5BAF0D8FFFF905F0100F4
:104F40002DE9F04101F092FA002837D0594C624D1A
:104F500094F80B800027D5F88000F9B24144821DF7
:104F600091FBF2F602FB1616A95D2E2907D1F9B2C4
:104F700011B9E17A491CE172761C08F10108401E62
:104F8000B042B4BF2021A95DF8B200F026FAA819FA
:104F900040782E2803D10121F8B200F03EFA7F1CA0
:104FA000F8B20528D7DDE07AD5F88010401C491DFD
:104FB000C2B29142B8BF0020E07201E0BDE8F081CA
:104FC000BDE8F041474800F036BA3A49C864704736
:104FD00080B501F04BFA38B1002000F056FABDE878
:104FE0000840414A3D49A4E701BD80B50020FFF7D4
:104FF00035F8BDE802400020FFF756B810B502F0C2
:1050000095F828B10020FFF729F8BDE81040F2E735
:1050100004F030FE98B9274C606205216170334876
:10502000FFF70EF80020E064264A314904F1D00071
:1050300000F067FABDE81040052005F00FBCBDE8A0
:105040001040002004F01BBE2A49802008607047F1
:1050500029492A4A8020086029492A4800F051BA83
:105060003EB5054610680C4605F006FDCDE9000189
:10507000254B264A2146284605F022FD284603B046
:10508000BDE83040B7E60000202E00001CB500222D
:105090008DF800200123074C044A6373117001222C
:1050A00069463EE000002440947E0020BD7E002042
:1050B00025420008741F0020E14A00086F460008DE
:1050C00098A9010840420F00914B0008D4A901089B
:1050D000794C000874AB010808790020434E0008A1
:1050E000E41F0020254F000820A10700F8AB0108AD
:1050F000A940000800E100E080E100E0D0121300C8
:1051000049500008F47D002020AB0108A4AB010841
:105110001CB504460621684600F078F90622694667
:10512000204605F001FD13BD80B501F09FF988B15F
:105130000221DFF8980306F050F858B900F08BF818
:10514000BDE80840DFF88823DFF88813DFF888031C
:1051500000F0D7B901BD10B501F088F978B1DFF8DA
:105160007C43DFF86C23DFF86C1304F11C0000F0C3
:10517000C8F9022006F0C7F830B10120607402209F
:10518000BDE8104006F0CCB810BD411E8941C943AE
:10519000DFF84803C90F41747047DFF84003407CD3
:1051A00070470621DFF8380305F04CBA38B5DFF850
:1051B0002C53062205F10801284606F012F90F24A7
:1051C00020B9A969002945D00F2040E006222946D0
:1051D00005F10800FEF764FE2878012809D00228AE
:1051E00009D0042809D0082809D0102808BF0D24A8
:1051F00006E0012404E0042402E0072400E00A247D
:10520000A878012809D0022809D0042809D0082844
:1052100009D0102808BF0C2406E0022404E005246D
:1052200002E0082400E000242879012807D00228A1
:1052300007D0042807D0082808BF0B2404E0032463
:1052400002E0062400E00924A96919B12046BDE85E
:105250003440084731BD7CB5A04B5C694CB19861C6
:105260000626A04D019500964022E021204606F03A
:105270009FFA73BDFEB5994D686900285AD005F0B4
:10528000CAFF05F11C0000F073F900206874A861E2
:105290000621284605F0D6F9062105F1080005F09B
:1052A000D1F906248F4E686948B100210622A96110
:1052B000009201962B464022E02106F079FA6869B7
:1052C00006F0BCF960B9686906F04BF9A3208DF8C7
:1052D0000000686920B101236A46E02106F0CAF99E
:1052E000641EE0D1794F06240221384605F075FF8F
:1052F00088B9686948B100210622A9610092019627
:105300002B464022E02106F053FA686906F096F930
:1053100090B1641EE8D1A3208DF80000686920B127
:1053200001236A46E02106F0A5F9022005F0F8FF06
:1053300005F05DFF03B0F0BD686906F012F9A32027
:105340008DF8000068690028EFD001236A46E0214B
:1053500006F090F9DFE76148807A000903E05F48D2
:10536000007BFFE7C00800F0010070471CB55B4CF4
:105370006061080018BF884700F00BF881208DF8A5
:105380000000606920B101236A46E02106F072F94D
:1053900013BD1CB521208DF80000504C6069C0B1D0
:1053A00001236A46E02106F065F9812260698DF8E3
:1053B000002070B101236A46E02106F05BF9A320CA
:1053C0008DF80000606920B101236A46E02106F0F3
:1053D00051F9002000F040F813BD38B50446062C02
:1053E0000D4612DA404901EB450333F8400C06F054
:1053F000EFFB3E490A1964001574641C0022E4B2F4
:105400000A7008552144000A487031BD0A46072930
:10541000A8BF06223649FEF733BD4000401C334A80
:10542000C0B210440029427814BF42F0400202F09A
:10543000BF024270704780B501462848406920B9D4
:10544000080008D0BDE80140084700910D23274A15
:10545000E02106F06DF901BD20490B7C984200D196
:10546000704780B50874087C1028A4BF0F220A7406
:10547000087C40F0E0008DF80000486920B101236D
:105480006A46E02106F0F6F801BD38B50446174D2E
:105490000D21284605F0D6F82022072105F110003D
:1054A00006F0A2FB2046BDE83240C4E710B5044632
:1054B0000E48002300F8013BFF220C2106F0B2FB4E
:1054C0002046BDE81040B6E700000000000C014097
:1054D00020A1070029510008BC080020A0080020D6
:1054E000A8080020AD5100080CA00108947D002000
:1054F000A47D002000230FF2A1027849012006F0CC
:10550000C5BBF8B504460800154630D0206988426E
:105510001CBF0023E3602161204600F029F80A2D1A
:1055200006D204F10C01BDE8F4406D4805F06CB8FA
:1055300072B6656000F095F801466A4AA16002F112
:105540000C0300E00346186840B1856846684D1BAF
:10555000AE42F7D36768751BAF42F3D220601C6080
:10556000D268A24204BF084600F088F862B6F1BDD6
:1055700072B60021416081605B4A00E00A46116812
:1055800029B18142FAD1016811600022026062B63D
:105590007047012006F006BC70B5524D504E0121F7
:1055A000A96000222A70012006F0F3FB69686A688E
:1055B000401A80B2801868606A68EC6815E020685C
:1055C000E86000216160A1602160304604F10C01B7
:1055D00005F01AF8EC68012006F0DBFB69686A68E0
:1055E000401A80B2801868606A6854B1A068616827
:1055F000101A8142E3D36368181A6060A2602468BD
:10560000F3E7012006F0C5FB69686A68401A80B2BA
:10561000801868606A68E86840B181684368511A18
:105620008B42CAD34468611A416082600023AB6038
:10563000A968A9B940B1416847F6FF73994203D8F8
:10564000416882688A1804E0287848B902F5FE4269
:10565000FF3292B20021012006F070FB0120287079
:1056600070BD80B5012006F094FB1E494A684B6866
:10567000801A80B2C0184860486802BD10B5194C45
:105680000246A06880B9E06878B1416847F6FF73C8
:1056900099420AD8416882688A1892B20021012092
:1056A00006F04CFB0121217010BD20780028FBD1B1
:1056B00002F5FE42FF32F0E70C4B59889888814290
:1056C00002D3012119707047187830B9491C5980EC
:1056D00003F10800014A064913E7704740420F00F2
:1056E000947E00208420002090200020DC7C00207C
:1056F000B956000810B50FF22500DFF80C49FEF787
:1057000097FC0FF27970FEF797FCDFF800098268CA
:1057100004F1C00190470020207410BD10B504466C
:1057200002F0F0FF844222D102F0E3FF50B90022E0
:10573000DFF8DC18DFF8DC08FEF7DCFC022005F0FF
:105740008DF814E0DFF8C0385979187E01430BD189
:105750000121197603F19000DFF8BC280FF24D010A
:10576000FFF7CFFE012010BD002000F0D3FA00208B
:1057700010BDDFF89418087E28B94879401E804192
:10578000C043C00F704701207047DFF87C38187E97
:10579000002804BF5879002807D0DFF87C280FF2D2
:1057A0000D0103F19000FFF7ACBE7047DFF86C18F5
:1057B000DFF86C0804F028BF80B5DFF84C28117CB6
:1057C00021B9906001201074002002BD012918D178
:1057D000D06000201074906810B1D16888420AD35C
:1057E0000022DFF84018DFF82C08FEF783FC0220C7
:1057F00005F034F805E002F16801DFF8240804F050
:1058000003FF012002BDDFF8000840797047DFF890
:10581000F817487920B10879052801D1012070478F
:1058200000207047DFF8E017487920B10879042894
:1058300001D10120704700207047DFF8CC1748796C
:1058400020B10879022801D101207047002070475B
:10585000DFF8B417487920B108790A2801D101206E
:10586000704700207047DFF8A017487938B10879F1
:10587000801E02D0801E012801D801207047002020
:10588000704770B5DFF880570446287E002804BFB3
:105890006879002807D0DFF88027DFF88C1705F13A
:1058A0009000FFF72EFEA87ED0B90CB1042C02D3D5
:1058B0000FF62C002AE0641EE6B2DFF8700706EB54
:1058C0004602182100EBC20006F0C6FA05F11400EA
:1058D000002181550122AA766C760FF6140015E09E
:1058E0000CB1072C02D30FF608000FE06A7E05F119
:1058F0001401885C80B901206877EC76012205F1FB
:1059000019019F2005F010F90FF2F470FFF773FAF8
:10591000BDE87040FFF7AEBAE0B2BDE8704055E0B8
:10592000010004D0032802DC401EC0B270470328E7
:10593000A8BF03207047DFF8D016087F00220300BD
:105940000A7709D0072807D24A7E0A44117D002928
:1059500008BF00F002B839E0704730B585B001A843
:10596000102106F079FADFF8A046657E207D6D1CD7
:1059700018B15DA101A806F072FA607D18B15BA1B3
:1059800001A806F06CFAA07D18B159A101A806F093
:1059900066FA9DF80400C43448B101A900912B4671
:1059A0000FF2A4625021204605F08AF806E02B464B
:1059B0000FF2AC625021204605F082F82046FFF736
:1059C0001AFAFFF757FA05B030BD000018B5DFF836
:1059D0003846627E022A85B002DCA118097D19B919
:1059E00006B0BDE81040B8E7401E052821D8DFE822
:1059F00000F003223B4B5B6BDFF8301602EB4203F7
:105A000001EBC30250780FF26862002814BF0FF256
:105A100068630FF26C63502104F58A7005F050F84A
:105A200004F58A70FFF7E7F906B0BDE81040FFF70C
:105A300021BA06B010BDDFF8F40502EB420100EB1D
:105A4000C100C27A0492817A0391427A0292017A69
:105A50000191C27900928379DFF8D425502104F5B1
:105A60008A7005F02DF8DBE7DFF8C00502EB420194
:105A700000EBC1004279029201790191C278009253
:105A800083780FF20462E9E7DFF8A00502EB420138
:105A900000EBC100C27B0292817B0191427B0092AC
:105AA000037B0FF2F852D9E7DFF8800502EB4201E1
:105AB00000EBC100C27C0292817C0191427C009289
:105AC000037C0FF2EC52C9E7DFF8600502EB4201FC
:105AD00000EBC100C27D0292817D0191427D009266
:105AE000037D0FF2E052B9E73120000032200000C0
:105AF000332000002DE9F84F040000F0EE80172954
:105B0000ADF80210C0F0E980DFF8FC54687950B1BC
:105B100028790A2807D1697F4A1E9241D243D20FC1
:105B20008DF8002002E000218DF800100027BDF85C
:105B300002000026182841D31822B0FBF2F292B2DC
:105B400002EB4203B0EBC30038D1BDF80280DFF8AE
:105B5000DCA422E04FF0030906E00100FAD0B9F11D
:105B6000040FF7DAA0F101095FFA89F9B9F1020F20
:105B700011DC09EB49034FEAC30B1822A1190AEB08
:105B80000B00FEF77DF90AF80B9005F114000123D4
:105B900000F809307F1C1836B6B206F118018845A6
:105BA00007D3A019F7D0A05D8146B9F1020FD4DC6C
:105BB000DFE7FFB2002FADF802805DD19DF8000055
:105BC00068B9687910B128790A2808D02078FFF7D9
:105BD000A7FE8046B8F1020F03DDBDE8F18F95F80E
:105BE0001980B8F1020F42DCBDF8021018290FD35A
:105BF000607802280CD2207808F10103DBB29842C9
:105C000004D05FEA080203D0404501D1012700E03B
:105C1000002707F11700814229D308EB4801C9008A
:105C2000DFF8080400F801804618E05D7070E119A3
:105C30004A1CB01C116801600622E119491DB01D03
:105C4000FEF71EF9E01900F10B0106F10C020868DD
:105C5000106006F11002E01900F10F0108681060F1
:105C600006F11402E01900F113010868106005F153
:105C70001401012001F808009DF8000080B1E97EC0
:105C800000206877E87601B306291ED86B7E05F1FF
:105C90001402D05C08B129770BE0FFF75EFE14E038
:105CA000287F00281FBF05F114016A7E885C002848
:105CB0000BD005F1A8042046FFF75AFCDFF8742347
:105CC000DFF874132046FFF71CFC00208DF800005D
:105CD000012269464E2004F027FFBDE8F18F80B510
:105CE00001208DF800000022C9490FF2EC30FEF7C8
:105CF00001FA02F031FB01226946912004F014FF01
:105D0000002000F007F801BD012002F029BB0020AF
:105D100002F026BB10B5BC4C00202076A080A0600D
:105D2000E0602074032104F1140004F08BFC48218E
:105D3000BE4804F087FC0020A0836083607604F1F5
:105D40009000FFF715FC04F17800FFF711FC04F157
:105D5000A800FFF70DFCBDE81040FFF713B880B5B1
:105D6000FEF712F900909DF800000A2807D1B34908
:105D7000AB4804F049FCBDE802400020CAE701BD81
:105D800080B501208DF8000002F008F900280CBF52
:105D900084A00FF2443000229D49FEF7ABF902F0D7
:105DA000FDF8401E8041C00F02F0EBFA15E080B50F
:105DB00001208DF8000002F0E5F800280CBF79A062
:105DC0000FF2143000229249FEF794F902F0DAF84B
:105DD000401E8041C00F02F0D8FA0122694691208E
:105DE00004F0A2FE0020FFF795FF01BD80B5012061
:105DF0008DF8000002F046F800280CBF69A00FF2F1
:105E0000D82000228249FEF775F902F03BF8401EC7
:105E10008041C00F02F08DFADFE780B501208DF8D8
:105E2000000002F000F800280CBF5EA00FF2A820CE
:105E300000227749FEF75EF901F0F5FF401E804130
:105E4000C00F02F09AFAC8E780B56F48002141768A
:105E5000417741830FF28820FEF7CDFFBDE8014076
:105E6000FFF708B880B568488168C068ADF80010D1
:105E7000ADF80200042269469220B1E770B5624D88
:105E80000446287E2C710126002804BF687900286A
:105E900005D0614A644905F19000FFF732FB601EAE
:105EA00009283ED8DFE800F00512181E242C2F32F6
:105EB000353805F128015A4804F0A6FB0122291DB6
:105EC0008E2004F031FE012C35D132E06E710020BD
:105ED000002600F069F8F1E70020A860E86005F10D
:105EE0006801E8E76E710020A860E8600026F0E72E
:105EF00000206E7100F058F8002605F13001DAE755
:105F000005F13801D7E705F14001D4E705F1480173
:105F1000D1E705F15001CEE76E7105F17001002661
:105F2000C9E700223A493B48FEF7E4F8022004F0B2
:105F300095FC002070BD304670BD1CB5324C207EF3
:105F4000002804BF6079002805D0334A364904F19F
:105F50009000FFF7D6FA01F0E3F828B12079022883
:105F600008BF04F1200118D001F0DAF820B9207937
:105F7000022818BF042807D02079052808BF04F19B
:105F800058010AD00A280CD1FDF7FEFF00909DF8B9
:105F900000000A2805D104F16001BDE81C40FFF7AC
:105FA00007BC13BDC2CACB002DE9F041164C607985
:105FB00028B320790B2822DA0A2818D0FEF73FFFF1
:105FC000804620791E4D642670432F18384600F015
:105FD0003DFE02463946404605F050FF38B101F01B
:105FE0009FF820B920794643A819FEF704FF04F171
:105FF0007800BDE8F0410B4A1249FFF782BABDE8CC
:10600000F0410020FEF7EEBE1C1D0020841F002082
:1060100000093D00F0AB0108809698007C1D00202F
:10602000947E002040420F00AD570008C07A002047
:1060300088AA01083057050037590008801E002043
:10604000CC950108A95F0008696625752D6E6574F9
:1060500020646174612E2041763A257300000000AF
:10606000696625752D6E6574206461746100000099
:106070006D6F64652D257300444843500000000097
:1060800053544154000000006970202D2025752EC6
:1060900025752E25752E2575000000006777202DAB
:1060A0002025752E25752E25752E257500000000DE
:1060B000646E7331202D2025752E25752E25752EA5
:1060C00025750000646E7332202D2025752E2575F0
:1060D0002E25752E25750000C2DBCACB00000000FE
:1060E000312D33206966202A65786974000000002C
:1060F000312D3620706172202A65786974000000A5
:106100005A6170726F732E2E2E00000072B6BFF3AC
:106110004F8FB949B9480A6802F4E06202430A6045
:10612000BFF34F8F00BFFDE7B549B64804F06CBA26
:10613000B549488888B1401E488080B268B972B6B7
:10614000BFF34F8FAC49AD480A6802F4E0620243E6
:106150000A60BFF34F8F00BFFDE74AF6AA21AB4AA2
:106160001160704710B5A84C0020207120700123E9
:106170006371042140F6FF7005F099FE05F092FE70
:106180004FF4967060800023A14AA249002005F0D8
:106190007DFD002005F0ECFD04F12800BDE8104075
:1061A0009D4A0FF22D01FFF7ACB99749782048803E
:1061B00070479A49012008707047984800787047E6
:1061C00080B5002005F0EEFDBDE80140FFF7E1B924
:1061D000F8B58D4C207830BB914D924E924F934B39
:1061E000934900973246284605F099FE05F08AFE4D
:1061F000012006F03EFC3146284606F017FD06F069
:1062000096FC06F09AFCFFF775FA002001F001FAFF
:106210000120207004F14000BDE8F840854A0FF2EB
:106220000901FFF76EB9F1BD7CB5834D764C834E05
:1062300006F025FC294607F00DF8009015D23078BD
:1062400038B96A461E21E01DFEF70AFF04203070AF
:1062500001E0411E317001206071217906292ED1A3
:1062600000F045F80020207122E0002131700098F4
:10627000734906F0EFFF04D2042269468C2004F033
:1062800053FC2079A0B9607948B1002161710020E8
:10629000FEF7A8FD00F0EAF808B90120A07101217D
:1062A000217104F15800674A0FF26D01FFF729F9D7
:1062B000607920B90098294606F0CCFF01D25D4AEA
:1062C00000E0614A614904F14000FFF71AF973BD2B
:1062D0004D484079704710B54B4CA07930B1002241
:1062E0004D495B48FDF706FF0021A17110BD80B547
:1062F0008021584807F01EF84021574807F01AF847
:1063000056484FF4005101600822026000F03EFF41
:106310003D490020087101BD38B53B4C2279521E21
:10632000042A4ED8DFE802F0030F1C20370080213A
:10633000484806F0FCFF4A4A4A4904F12800FFF7A2
:10634000E0F802203CE0444D40230322102128467F
:1063500006F092FF4021284606F0E9FF03202FE0D7
:1063600000F088F804202BE03B4D4FF4005303224B
:106370001021284606F080FF01F099FD20B1374931
:106380004FF40050086004E04FF40051284606F036
:10639000D1FF052014E0304D0823032210212846A8
:1063A00006F06AFF01F09AFD18B12C490820086038
:1063B00003E00821284606F0BDFF00F0E7FE0620B6
:1063C000207106F05CFB1C4906F044FF04D2FFF785
:1063D0008EFF0620207131BD207906280BD0207950
:1063E0002149032804F15800BDE838400CBF094A90
:1063F000144AFFF786B831BD0CED00E00400FA0541
:10640000D41C0020947E0020007A00200030004040
:1064100029610008A086010080841E00BB7E002048
:10642000A788000829AB0008AF8D0008178D000869
:10643000F18C0008C0C62D000000E040BA7E0020AC
:106440000000204140420F00C0E1E4002962000842
:1064500020AC01080008014000100140101001406C
:1064600080969800E5DA000819630008DFF80C0749
:106470000078704710B5DFF80447207848BBDFF894
:106480000027DFF80017201D05F0AEF8DFF8F8163A
:10649000201DFDF789FD201D05F0D0F804F04AFD10
:1064A000201D05F0CBF8FDF791FD201D05F0C6F885
:1064B000201D06F0DBFF201D05F0C0F8FEF7DAFE18
:1064C00001202070FDF794FD201DBDE8104005F06F
:1064D000B5B810BD38B54FF4C06007F013F840F2FE
:1064E000026007F00FF840F2036007F00BF840F28B
:1064F000046007F007F807F0C7F840F2056007F0FE
:1065000001F840F20E6006F0FDFF4FF4A06006F0C7
:10651000F9FF40F2137006F0F5FF40F2015006F06B
:10652000F1FF40F2096006F0EDFF40F20A6006F06C
:10653000E9FF40F20F6006F0E5FF40F21D7006F043
:10654000E1FF40F20B6006F0DDFF40F20D6006F067
:10655000D9FF002006F0F9FF002006F0F1FF01212D
:10656000DFF82806DFF82846DFF8285606F0EFFEA9
:1065700007F03EF9012303220021204606F07CFEAD
:10658000022303220021204606F076FE0423032284
:106590000021204606F070FE102303220021204631
:1065A00006F06AFE202303220021204606F064FE46
:1065B0004FF4007303221821284606F05DFE4FF4C5
:1065C000807303221021284606F056FE4023032242
:1065D0001021284606F050FE4021284606F0A7FE6E
:1065E000802303221021284606F046FE80212846FB
:1065F00006F09DFE4FF4805303221021204606F042
:106600003BFE4FF48051204606F094FE07F01CF943
:10661000FEF770FF00F041FA07F044F9FFF7A2FD22
:1066200000F003FA07F08AF900F0EDF800F090F9B5
:1066300007F0FAF900F0BEF8DFF85C0507F059FA48
:1066400000F07AF807F090FD00F039F802F014FD40
:1066500007F0F0FDDFF8440507F042FE0FF2845228
:10666000D2E9000107F0C8FE802303221021204652
:1066700006F002FEDFF828450423032210212046FD
:1066800006F0FAFD0421204606F054FE06F0CFF98C
:106690004FF4807303221021284606F0EDFD4FF4DD
:1066A0008071284606F046FE00F034FE022007F016
:1066B00017F900F01FFABDE8314008F014B818B51A
:1066C00087B040F20F7006F01DFF04230322102153
:1066D000DFF8D004DFF8B84406F0CEFD4FF40043F5
:1066E00003221021204606F0C7FD4FF4004120464A
:1066F00006F01DFEDFF8A8442823032218212046B7
:1067000006F0BAFD102303220421204606F0B4FD52
:10671000DFF89404DFF8904400210160102241600A
:1067200006924FF4007103914FF482704FF40061B0
:1067300000900291002231E018B587B040F20E704F
:1067400006F0E0FEDFF858444FF480530322102196
:10675000204606F091FD4FF42043032218212046E5
:1067600006F08AFD4FF4804303220421204606F000
:1067700083FD4FF48051204606F0D9FDDFF82C044C
:10678000DFF8284400210160002242604FF482704B
:106790004FF40071009003910692029201920492CC
:1067A00005926946204608F043FD204608F05AFD50
:1067B00008B010BD10B592B0DFF8F443684621462A
:1067C0002422FDF76DFB09A804F124012422FDF722
:1067D00067FB002008F092FD684608F05DFD09A8FF
:1067E00008F05AFD009800230222012108F007FE5C
:1067F000009808F077FD099808F074FD009808F0FB
:106800007FFD12B010BD70B5B2B0EA4C28A8214689
:106810002822FDF745FB28A808F06CFE08F0A3FE2F
:106820001EA804F128012822FDF73AFB07F0FCFA24
:10683000229007F0FBFA24901EA808F05BFE08F0F7
:10684000D9FE08F0BCFE08F0B6FE14A804F1500111
:106850002822FDF725FB06F00AF9189014A808F085
:1068600049FED54D0021284608F045FF02220021AF
:10687000284608F0C4FF0021284608F04DFFCF4904
:10688000CF4DD04E002008704FF40062CE482A60F1
:10689000016841F0020101603046042108F0BAFEAF
:1068A0000321304608F0B6FE0AA804F17801282238
:1068B000FDF7F6FA0CAA0421304608F0D2FE0222B7
:1068C0000421304608F09BFF08220421304608F0DE
:1068D00096FF0421304608F02FFF0321304608F0D0
:1068E0002BFFBA49002008704FF00062B8486A6078
:1068F000016841F400310160026842F40022026044
:10690000016841F4802101600221026842F4803272
:106910000260304608F07EFE684604F1A00128229D
:10692000FDF7BEFA06F000F90490684608F0E2FDB3
:1069300002220221304608F062FF0822022130467E
:1069400008F05DFF0221304608F0E6FE32B070BD6F
:106950002DE9F84FA5A191E87C0098B013A807AFE6
:1069600080E87C00A6A393E8070F87E8070F139B36
:10697000079313A808F052FF07A808F053FF0899DF
:10698000099A079889B209F00FF90A9A08990798A5
:1069900092B289B209F0EEF80798012108F0D0FF11
:1069A000079808F0C5FF0798012109F047F98949C0
:1069B000894B002008704FF480521A606F46079888
:1069C00008F037FF95A191E87C000EA880E87C00D4
:1069D00097A393E8070F87E8070F0E9B00930EA875
:1069E00008F01CFF684608F01DFF0199029A009804
:1069F00089B209F0D9F8039A0199009892B289B244
:106A000009F0B8F801990098002289B209F0DCF881
:106A10000098012108F094FF009808F084FF009886
:106A200008F007FF19B0BDE8F08F38B55C4C4FF4A3
:106A3000007303221021204606F01EFC4FF4007163
:106A4000204606F077FC4FF4807303221021204685
:106A500006F012FC4FF48071204606F06BFC4D4DA1
:106A6000012303221021284606F006FC01212046BE
:106A700006F060FC022303221021284606F0FCFBEE
:106A80000221204606F056FC284601B0BDE8304001
:106A900003230322102106F0EFBB70B53D4C1023F9
:106AA00003222821204606F0E7FB0421022006F0FD
:106AB0007CFC00220021102004F0F2FB474D404EE8
:106AC000002028704FF480613160202303222821A8
:106AD000204606F0D1FB0521022006F066FC0022CC
:106AE0000021202004F0DCFB002068734FF400013B
:106AF000316070BD10B5274C4FF48063032218211C
:106B0000204606F0B9FB4FF400630322042120461F
:106B100006F0B2FB4FF4805303221021204606F00A
:106B2000ABFB2F4C4FF41651204609F0A5F800217D
:106B3000204609F0CDF80021204609F0CEF80021CA
:106B4000204609F0D3F80421204609F0DFF8082197
:106B5000204609F0D6F88021204609F0E8F84021C7
:106B6000204609F0DFF84FF44171204609F0F6F8AD
:106B70002046BDE8104009F0BEB80000E47B0020CC
:106B8000A086010000580040E3B100080002300078
:106B900000080140001001402FAF0008A78800083E
:106BA000000C014000140140003C0040003800404F
:106BB0000CA90108A4A40108000002400BE400E0B5
:106BC00000E100E000040240040002403BE400E079
:106BD000040402402CE400E004E100E00AE400E0E8
:106BE000004C00400BED0008DBFF000800340140C2
:106BF0000000000000000000B80B000000000000D2
:106C00000000000003000000DC0500006000000040
:106C1000010000000000000000000000002C014006
:106C200001000000000000005E1A000000000000EB
:106C300000000000000000002F0D000060000000B8
:106C400001000000000000000000000000F101034E
:106C5000810704D010F8011B820781B1FAD10268C4
:106C6000A2F10131914311F0803104BF50F8042F9B
:106C7000F6E709BAB1FA81F100EBD100401CC01A65
:106C800070470000DFF8E4047047DFF8E004C079E3
:106C90007047DFF8D814C8717047DFF8D004C179A5
:106CA0000B2901D10120704700207047032818BF2D
:106CB000042808D0082818BF052804D006281CBFBF
:106CC00009280A2801D101207047002070470328B5
:106CD00018BF04280BD0082818BF052807D006289D
:106CE00018BF092803D00A2818BF0B2801D101209A
:106CF00070470020704780B50C281CBF0D28152850
:106D000008D009F041F809F0F6F9401E8041C0436F
:106D1000C00F02BD012002BD0A2818BF052803D0FC
:106D2000062818BF092801D10120704700207047AC
:106D3000132818BF14280FD0172818BF01280BD00C
:106D4000022818BF072807D0162818BF0C2803D020
:106D5000122818BF112801D1012070470020704768
:106D6000132818BF142804D017281CBF0C28162875
:106D700001D101207047002070470D2818BF152849
:106D800001D10120704703281CBF0428082809D01E
:106D9000052818BF062807D0092818BF0A2803D0DD
:106DA00000207047002000E0012080F001007047C3
:106DB000312801D1481E05E000207047DFF8AC0300
:106DC000017964298041C00F704738B508F0DCFFB5
:106DD000044609F088F90546204609F088F940EA9A
:106DE0004500C0B232BD132818BF142807D00D28A3
:106DF00018BF112803D0152818BF162801D101206B
:106E000070470020704713281CBF1628142801D192
:106E1000012070470020704710B5DFF850436279B9
:106E20002079214603F080FE0021E17210BD1CB5DF
:106E300008F0B2FF0146DFF834430222204604F096
:106E4000E0FA02206071E079032818BF04280ED010
:106E5000082818BF13280AD00D2818BF162806D0F6
:106E60000C280AD102200321A070617121E00320C7
:106E70006071FFF7AAFFA0701BE00A2819D100205B
:106E8000ADF8000001F006F920B108F088FF008895
:106E9000ADF8000002226946204604F0B2FA08F07C
:106EA0007BFF01460222A01C04F0ABFA6079801C33
:106EB000607162792079214603F036FE13BD00002F
:106EC00070B5AA4DAA4C2875411E102900F29C806D
:106ED000DFE801F0333333913E3E70739A09094A7B
:106EE0001E91337689000A2809D108F055FF014622
:106EF0000222284604F085FAFF20A87004E004224C
:106F00000021284604F091FA03222946662077E002
:106F1000E87B10B9032003F0A1FC08F03DFF0088D6
:106F2000BDE8704000F0CDBA02F01FFB687B00287E
:106F30006AD1BDE87040FEF761B8E87B20B9012254
:106F40008C498D48FDF7D6F8BDE8704002F00DBBC6
:106F50000921052808BF0A2129700122287929461C
:106F600003F0E2FD0C202875A87B40B9687B40B98E
:106F700008F012FF01460222682003F0D5FDA87B2D
:106F800048B901F0A4FA064601F04FFA314606F07E
:106F90009BFA06F081FA02202070E8790A2818BFCF
:106FA000052804D006281CBF09280D28BCD102F0F2
:106FB000C7F8BBE7002028701FE00B2028701CE0FA
:106FC0000020FDF771F80220207008F0E5FE014670
:106FD0000222682003F0A8FDE8790B28C2D10A201C
:106FE00007F096FABEE70221217008F0D5FE0146AF
:106FF00002227D20B4E70021297001222879294648
:10700000BDE8704003F090BD70BDF1B508F0C4FE5E
:10701000564F0088388001263879012402216D28D6
:10702000797104D103217971FFF7CFFEB8709DF813
:10703000000008B338796D2817D0FFF7C6FEB87086
:10704000032078713879652808BF78200CD06F2824
:1070500008BF772008D09C2808BF9B2004D0782840
:1070600018BF9B2801D06D20387108F08DFE09F003
:107070003AF808B90026002401F084F8054638796A
:107080006D2817D154B108F07FFE09F02CF8F0B943
:10709000F87902281CBF0128072818D07A79387996
:1070A000394603F041FD012269469A2003F03CFD78
:1070B0003046F2BD002CF6D008F066FE09F013F859
:1070C00028B9F87902281CBF01280728EBD1002D28
:1070D000E4D00121F9722748284945432A4607F19F
:1070E0001800FEF70EFADEE780B509F0E3F930B9D3
:1070F000BDE80840224A23492348FEF702BA09F0B6
:10710000DCF9014602222A2003F00EFD1849022074
:107110000870BDE8014002F028BA1448007D7047AD
:107120001248007A70471149C87370470F48C07BF6
:1071300070470E49087470470C48007C70470B4933
:10714000487470470948407C70470848807C704705
:10715000064988747047054AD17B29B1032818BFB6
:10716000012801D10120704700207047B47B002026
:10717000DC7C002040420F00F0AB0108196E0008D3
:10718000A0860100E97000084C7D002038B5DFF8CA
:10719000441ADFF8084B487B4FF4804530B9097A30
:1071A000481E8041C00F06F05FFA08B1656031BD2E
:1071B000256031BD80B5FFF7E9FFBDE80840DFF885
:1071C000182ADFF8181ADFF8D80AFEF79AB9DFF89C
:1071D000D41A0020087001F05BBB012802D00228FD
:1071E0000AD07047DFF8F809416941F40041416174
:1071F000026822F4004208E0DFF8E409416941F046
:1072000004014161026822F0040202607047DFF865
:10721000D009DFF8902A016841F4004101600020A4
:1072200090717047DFF8B809DFF8782A016841F0FB
:10723000040101600020D071704738B50446DFF8C2
:10724000680ADFF8681A0068012C0CBF00F40040DF
:1072500000F00400451EAD41601EC0B2ED0F0A5C97
:10726000AA420CD00D54FFF767FF40B98DF80040DB
:107270008DF8015002226946A02003F055FC31BD73
:10728000DFF82C2A0FF20901DFF8280AFEF739B9D6
:1072900070B500240125DFF8106AE8B2FFF7CDFFD2
:1072A000E8B2012830680CBF00F4004000F0040090
:1072B00000B901246D1CE8B20328EED34CB1DFF80D
:1072C000F029DFF8F419DFF8EC09BDE87040FEF7AB
:1072D00018B970BD80B509F02AF906F0E5F906F095
:1072E000F8F9DFF8C409DFF8C4290168C90B01F017
:1072F000010181F001011170111D0068800800F08A
:10730000010080F001005070DFF8B0098268BDE82C
:107310000840104710B5DFF8BC480020012120725A
:1073200021736073DFF89829DFF8981904F1A4003D
:10733000FEF7E7F8FFF72AFFDFF89C28DFF89C1834
:1073400004F1EC00FEF7DDF820E110B500F0AFFD30
:10735000D0B1FEF7BDFFB8B9FFF7E2FEA0B9FFF765
:10736000E5FE88B9FFF7D9FE04460D2C18BF0A2C9C
:107370000AD000F083FE00281EBFDFF828194879E4
:10738000002801D1092C01D1002010BD012010BD21
:1073900080B5FFF7DAFF60B1FFF7CEFE18B1BDE8A8
:1073A0000140FCF7D7BEBDE80240DFF81C09FCF73E
:1073B000EDBE01BD80B500F07AFD50B1FEF788FF4B
:1073C00038B9BDE80440DFF80419DFF8040903F018
:1073D0001BB901BD80B5FFF7AFFE08B1002002BDAB
:1073E000FFF7B3FF30B1DFF8E418DFF8E40803F08B
:1073F0000BF9012002BDF8B5DFF8D86707467078B1
:107400000C46154638B1FEF763FF48BBDFF8B808F5
:10741000FCF7BCFE24E0472F03D1207805F0D3FC15
:107420001EE07A2F02D1FFF781FEC8B9307901281A
:1074300018BF052804D009281CBF072808280AD12E
:10744000707940B9032003F009FADFF87C08FCF7F3
:107450009DFE012070712A463079214600F0CFF957
:10746000FFF76AFE18B92A462146384625E0F1BDE5
:10747000F8B5DFF860770446387901281CBF032887
:1074800008280D46164615D1387898B90022DFF83D
:107490004418DFF84408FCF72DFE022003F0DEF963
:1074A00001203870DFF83428DFF8341807F1740051
:1074B000FEF727F8324629462046BDE8F84003F09B
:1074C00033BB01B5DFF8DC170720087102226946DB
:1074D0007A20FFF790FF01BD1CB503461400084653
:1074E0008DF800300AD08DF800209DF80020092A80
:1074F00014D1DFF8B027012191731AE0612BF4DA7F
:10750000012B07D1DFF89C37052101228DF80010EF
:107510009A730EE006218DF8001005E0052AE8D0E8
:107520000A2A18BF062A04D1DFF878170122CA7385
:107530008A739DF80010DFF86C37197101226946D3
:10754000FFF759FF13BDDFF85C1701208873704700
:1075500010B5012006F0D5F8DFF87846B0B1207AF2
:10756000A0B9207905281CBF092808280ED0A07BC7
:1075700060B9012121712173FFF782FEDFF86427D2
:107580000FF2CD4104F15C00FDF7BBFF0020A073BA
:1075900010BD10B5022006F0B4F8DFF83846002818
:1075A0001EBF207906280A281AD0E07BC0B9207AAD
:1075B000DFF8FC26002807BF02212171012020717D
:1075C0000221217304F58270DFF8EC16FDF799FFB4
:1075D000DFF810270FF2794104F15C00FDF791FF0D
:1075E0000020E07310BDDFF8BC060179042901D149
:1075F0000120704700207047DFF8A8160871704717
:10760000DFF8A0060179042901DD01207047002080
:107610007047F8B500F03EFC064600F048FC044612
:1076200000F05CFCDFF8AC750546F87C20B1387CD6
:10763000401E8041C00F00E0012036B3D8B1FEF7F4
:1076400047FE18B9DFF88006FCF7A0FDDFF89806C2
:1076500008F0F1F8DFF894164FF48040086000223B
:107660000021012000F0CBF800220021022000F0D0
:10767000C6F8012078710121797005F05FFC0120C6
:1076800038747874B874F874F1BD387C18B100217E
:10769000797005F053FCF87C002832D124B1002227
:1076A0000021012000F0ABF825B1002200210220CA
:1076B00000F0A5F855EA04001BD0002C18BF002DDF
:1076C00004D0DFF8240608F0B6F804E0DFF8180666
:1076D00008F0AFF85CB1DFF814164FF48040086092
:1076E000FEF7F6FD18B9DFF8E005FCF74FFD0120C5
:1076F000787100210120797039747C74BD74F8743C
:1077000079E0787C844204BFB97C8D4205D13A7C13
:10771000561EB641F643F60F00E0012684420DD016
:1077200007F11400FDF724FF2CB1002200210120F5
:1077300000F065F802E0012000F050F9B87C8542C5
:1077400009D007F12C00FDF713FF7DB100220021C5
:10775000022000F054F80020002C18BF002D787093
:1077600023D0DFF8840508F066F822E000F0B6FBCD
:1077700008B1002018E00121F879797378B9012067
:1077800000F069FC401EDFF8281548430246DFF888
:10779000601507F1D400FDF7B4FE0120F871022056
:1077A00005F0E4FF002038717870DFF83C0508F040
:1077B00040F855EA040012D06CB1DFF830154FF4F0
:1077C000804008609EB1FEF783FD28B9DFF8F80419
:1077D000FCF7DCFC00E056B10120787107E07A7C10
:1077E000B97C387C0A43024318BFFDF7FEFB00203A
:1077F00038747C74BD74BDE8F14005F09FBB2DE981
:10780000F14FDFF8D06386B00D46934606F18C0049
:10781000FDF7AEFE00217173002000F00EFCDFF8D2
:1078200090740FF2C13907FB00F801A80021002273
:107830000023002480E81E009DF81810012918BFBD
:10784000052906F1440A04D009291CBF0729082983
:1078500044D1307A28B9DFF844044FF40051016074
:1078600004E0012005F082FFDFF888849DF818000D
:10787000072809D1DFF86803416941F400414161FB
:10788000026822F40042026006F1140A0FF2C529D0
:10789000DFF824143A4606F58270FDF732FE9DF8B3
:1078A0001800052818BF062803D0092818BF0A2881
:1078B00007D1FFF741FC20B9012206A9672003F098
:1078C00033F94CF25030804538BF8046FFF75EFCFC
:1078D000424649465046FDF714FE7CE002291CBF93
:1078E00006290A290DD1012000F0A7FB07FB00F8AB
:1078F000DFF8A8130FF29929082006F12C0A086076
:10790000C6E7042906D1012000F097FB07FB00F829
:1079100006F12C0A9DF818008DF800B06138042893
:1079200005EB0B0038BF012410F8010CF07008F0D3
:107930001BFE8DF8050083469DF818108DF8041085
:107940005FEACB7013D5DFF88003FCF71FFC012042
:107950007071A348416941F400414161026822F419
:1079600000420260032002F079FF06F020FE5FEA89
:107970008B7008D59A48416941F004014161026861
:1079800022F0040202601BF0030F06D03A46DFF833
:10799000281306F58270FDF7B4FDF07808F0D1FDEC
:1079A00035B19DF8002029460DF1060003F029FDB0
:1079B000102201A9672003F0B7F89DF81810F170A4
:1079C0000120002CB0703FF46AAF1BF0030F7FF46E
:1079D00066AFFFF7DBFB07B0BDE8F08F10B50128FD
:1079E00015D100F064FA58BB7A4CA079012161737B
:1079F00058B900F030FB421EAD48BF49424304F184
:107A0000BC00FDF77EFD0120A071012014E00228DA
:107A100017D0704CE0790121617360B9012000F04A
:107A20001AFB421EA248B249424304F1D400FDF7BA
:107A300068FD0120E071022005F098FE0020207111
:107A400010BD00F04BFA0028E3D010BD000000008C
:107A500010B5604C207BFFF7F0FB954A964904F582
:107A60008270FDF74EFD207B05F067FE28B1211DD9
:107A7000BDE8104001226720BDE404F18C00FDF751
:107A800077FD00F006F800206073BDE81040FFF7B6
:107A90007DBB10B5FFF741FB0D284E4C0DD0FFF715
:107AA0003CFB0A2809D000F0E9FA00281CBF6079E5
:107AB000002804D0FFF734FB08B1904807E0FFF737
:107AC0002CFB092806D1FFF731FB30B98C48FDF7B4
:107AD0007CFA02E00020FCF7C1FA6079A0B1FFF760
:107AE0002BFB28B1FFF722FB10B9FCF733FB09E0B1
:107AF000FFF71CFB10B9FCF7D7FA03E0FDF775FAA6
:107B0000FCF750FB00206071A07830B10021A1701B
:107B10000020BDE8104000F0BBBE10BD80B5FFF7EF
:107B2000B8FF604900204873BDE80140FFF72EBB55
:107B300038B50446734D2846FDF71AFD204600F07F
:107B40008AFA02465A48704942432846BDE83840FE
:107B5000FDF7D7BC10B500F0AAF9B0B91D4CA0795B
:107B60000121617360B900F076FA401E5049484324
:107B70000246614904F1BC00FDF7C3FC0120A0717D
:107B8000012005F0F3FD0020207100201EE0000020
:107B900010B500F0A3F9B8B90E4CE079012161737A
:107BA00068B9012000F057FA401E41494843024697
:107BB0004F4904F1D400FDF7A4FC0120E07102203C
:107BC00005F0D4FD00202071012000BFBDE8104069
:107BD000AEE700001805002020A10700B5710008DD
:107BE0000004014038B52F4C207AD8B900F05FF975
:107BF00008BB00F05CF9F0B90121A079617358B9B4
:107C000000F029FA421E2A483B49424304F1BC00D5
:107C1000FDF777FC0120A071012005F0A7FD0020F1
:107C2000207108E000F043F928B91C494FF40050D6
:107C30000860FFF7ABFA00F051F968BB00F04EF9AD
:107C4000B0B90121E079617368B9012000F003FA4D
:107C5000401E174948430246254904F1D400FDF768
:107C600050FC0120E071022005F080FD0020207111
:107C7000002000F0F0F90546012000F0ECF9854203
:107C800038BF05468C342046FDF772FC08481E4973
:107C900045432A46204659E731BD000010100140F7
:107CA00004060020180500200810014008050020E7
:107CB00040420F001C060020917200089806002028
:107CC000404B4C00D5720008E8AB010810050020BD
:107CD000947E002000093D00F0AB0108C0C62D00D5
:107CE000CF710008A086010000340140141001404B
:107CF00025720008C02709000F72000800AC0108B7
:107D0000E0AB0108A40500201D7B000810B5092880
:107D100002DA6FF04E0010BD08F066FCDFF88C1A36
:107D200008F070FC4FF07F54214608F0E9FCDFF8C2
:107D3000801A08F0ADFEDFF87C1A08F015FF08F095
:107D400085FF08F097FF41B2102901DB0F2010BD1D
:107D500011F10F0F02DA6FF00E0010BD40B210BD2E
:107D600080B54F3008F09CFFDFF84C1A08F090FE09
:107D70004FF07C5108F0F8FE08F07CFFC0B202BD65
:107D800080B508F031FCDFF8301A08F03BFC4FF00A
:107D90007C5108F0E9FEDFF8241A08F0E5FE08F04F
:107DA00069FF40B202BD030001D100207047884244
:107DB00006D20846401A90FBF2F0401CC0B2704751
:107DC000FF28F7D11020704700B585B008F07AFF82
:107DD0004FF420724FF46C2106F0F7F908F072FFAF
:107DE00010F8161FFF290CBF002101F003010170DC
:107DF000684608F0AAFF9DF80400FF2808BF80200D
:107E000006F096FBDFF8B809026905B05DF804EBEF
:107E10000021104700B585B0684608F055FF9DF871
:107E2000060005B000BD00B585B0684608F04CFFFF
:107E30009DF80200012818BF002005B000BD00B564
:107E400085B0684608F040FF9DF8100005B000BD01
:107E500080B508F037FF093002BDDFF8680900B5CA
:107E6000006885B081B221B9684608F02DFFBDF8E1
:107E700007004FF6FF7281B2914208BF002080B226
:107E800005B000BD80B508F01DFF407D012818BF7A
:107E9000002002BD80B508F015FF407D012805D007
:107EA000FFF74AF9401E8041C043C00F02BD80B5B4
:107EB00008F008FF407D01280BD0FFF73DF940B9DD
:107EC00008F000FF807DFF280CBF002000F00300B9
:107ED00001E0012002BD00F0010002BD80B508F004
:107EE000F1FE407D012809D0FFF726F930B908F0EE
:107EF000E9FE807DFF2803D1002002BD012002BDE4
:107F0000C0F3400002BD80B5FFF7C4FF40B908F0E0
:107F1000D9FE807DFF2805D000F00300032801D1A1
:107F2000012002BD002002BD38B5012818BF02287B
:107F300005460C4601D0012032BD022C01D302209F
:107F400032BD08F0BFFE11304179FF2904BF002285
:107F50004271012D0CBF012102214279002C12BF78
:107F6000114381F0030111404171417901F0030196
:107F70004171FFF7E8FADFF84808026900219047ED
:107F8000002032BD00B585B0684608F09DFE9DF822
:107F90000400012818BF002005B000BD00B585B061
:107FA000684608F091FE9DF80500012818BF0020E2
:107FB00005B000BD80B58AB0684608F0B9FEBDF8CE
:107FC00004000BB000BD80B58AB0684608F0B0FE72
:107FD0009DF808000BB000BD80B58AB0684608F077
:107FE000A7FE9DF8090021E080B58AB0684608F038
:107FF0009FFEBDF806000BB000BD80B58AB0684694
:1080000008F096FEBDF81E000BB000BD80B58AB02A
:10801000684608F08DFE9DF820000BB000BD80B5CD
:108020008AB0684608F084FE9DF82100FF2801D040
:10803000010000D103200BB000BD10B584B0044690
:10804000684608F069FE0DEB040148790B2828BF4B
:10805000042004B010BD10B584B00446684608F092
:108060005BFE0DEB0401C879002814BFFF28042033
:1080700002D00B2828BF0A2004B010BD80B584B000
:10808000684608F059FE9DF80400FF2808BF00204C
:1080900005B000BD80B584B0684608F04DFE9DF87F
:1080A0000500FF2808BF002005B000BD38B5054613
:1080B000052886B0A8BF4FF0FF301BDA684608F0ED
:1080C00027FE0024012D08BFBDF805000DD0022DAC
:1080D00008BFBDF8070008D0032D08BFBDF8090090
:1080E00003D0042D05D1BDF80B00B0F5966FB8BFD5
:1080F0000446204607B030BD0000000080B5401E99
:10810000032886B01CD8DFE800F002060D1468468C
:1081100008F0FEFD60E0684608F0FAFD9DF80D00ED
:1081200007B000BD684608F0F3FD9DF80E0007B0EB
:1081300000BD684608F0ECFD9DF80F0007B000BDDB
:10814000FF2007B000BD80B584B0684608F0E8FDA8
:108150009DF80500FF2814BF00283C2002D0B42859
:10816000C8BFB42005B000BD80B584B0684608F033
:10817000D7FD9DF80400B52801DA010000D1B42034
:1081800005B000BD80B584B0684608F0C9FD9DF813
:108190000700FF2808BF002005B000BD80B584B0EF
:1081A000684608F0BDFD9DF80600FF2808BF0020C6
:1081B00005B000BD80B584B0684608F0D2FD9DF8DA
:1081C0000400010014BFFF28842005B000BD80B565
:1081D00086B0684608F083FD9DF8040007B000BD36
:1081E00070B58CB004460D46164606A808F077FD1B
:1081F000684606A91522FBF743FE06220DF107018A
:10820000204603F0FEF89DF8060028709DF8051042
:1082100031700CB070BD80B586B0684608F05FFD67
:108220009DF80500FF2808BF032007B000BD00B57A
:1082300085B0684608F089FD9DF80800FF2808BF52
:10824000FE2005B000BD00B585B0684608F07DFD94
:108250009DF80900FF2808BFE62005B000BD00B565
:1082600085B0684608F071FD9DF80500FF2808BF3D
:10827000802005B000BD80B584B0684608F06FFD71
:10828000BDF804004FF6FF72904201D0010000D10A
:10829000052005B000BD80B584B0684608F05FFDDC
:1082A000BDF806004FF6FF72904201D0010000D1E8
:1082B000092005B000BD80B584B0684608F04FFDC8
:1082C000BDF800004FF6FF72904201D0010006D1C8
:1082D00005B05DF804EBDFF8F00408F0F0B805B085
:1082E00000BD80B584B0684608F039FDBDF80200D5
:1082F0004FF6FF72904201D0010006D105B05DF843
:1083000004EB4FF0804008F0DAB805B000BD38B596
:108310000078C208C0F10705C0088B5C012405EB9A
:10832000C005AC40A3438B5408F0CCFCBDE83840FA
:108330001DE080B508F0CAFC60B908F0C3FC4FF43A
:1083400080524FF46C2105F022FFDFF874040269BB
:1083500000219047002002BD80B508F0C8FC02E073
:1083600080B508F0C9FC08F0ADFCBDE808404FF44A
:1083700080524FF46C2105F00ABF80B508F0C5FCAF
:10838000F1E780B508F0BBFCEDE780B508F0BAFC7A
:10839000E9E710B50C4608F0DAFC204608F0DBFCF3
:1083A00008F090FCBDE81040E1E700B585B06846F4
:1083B00008F0CBFC9DF80A00FF2808BFF42005B0A8
:1083C00000BD00B585B0684608F0BFFC9DF806000A
:1083D000FF2808BFAD2005B000BD00B585B06846D8
:1083E00008F0B3FC9DF80700FF2808BFEB2005B09C
:1083F00000BD00B5FFE785B0684608F0B6FC9DF803
:108400000600FF2801D0102800DB002005B000BDC9
:1084100000B585B0684608F0A8FC9DF80800FF2864
:108420000CBF002040B205B000BD18B585B068464D
:1084300008F08BFC9DF80700FF2808BFEB2008F030
:10844000D3F8DFF8741308F0DDF84FF07C5108F032
:108450008BFBDFF8681308F087FB08F00BFC044681
:1084600008F030FC80F8AD414EE000B585B06846BC
:1084700008F07BFC9DF80900FF280CBF6FF0060098
:1084800040B205B000BD00B585B0684608F06DFC8F
:108490009DF80A00FF280CBF6FF00E0040B205B037
:1084A00000BD00B585B0684608F05FFC9DF80B0084
:1084B000FF280CBF6FF00E0040B205B000BD00B544
:1084C00085B0684608F051FC9DF8070099E718B59B
:1084D00085B0684608F039FC9DF80600FF2808BF03
:1084E000AD2008F081F8B44908F08CF84FF07C51C9
:1084F00008F03AFBB14908F037FB08F0BBFB044633
:1085000008F0E0FB80F8AE4160B206B010BD10B5D7
:108510000446FFF78AFF2070FFF7D9FF6070FFF76E
:1085200068FFA070FFF7CBFFE070FFF771FF2071CD
:10853000FFF79BFF6071FFF7A6FFA071FFF7B1FF88
:10854000E07110BD00B585B0684608F012FCDDF89A
:10855000060008F04BFC4FF6FF71884208BF9B48AD
:1085600004D0684608F005FCDDF8060005B000BD43
:1085700000B585B0684608F0FCFB9DF80500FF28B3
:1085800008BF002005B000BD00B585B0684608F002
:10859000F0FB9DF80400FF2808BF002005B000BDD7
:1085A00080B596B0684608F0E8FB9DF80400FF2807
:1085B00008BF002017B000BD10B596B0044668464D
:1085C00008F0DBFBC4EBC4010DEB4102537A012B35
:1085D00006BF0DEB410090F90A004FF0FF3016B0D6
:1085E00010BD80B596B0684608F0C7FBBDF84B00DB
:1085F00040F2E932904201DA010000D1AA2017B01E
:1086000000BD80B596B0684608F0B7FBBDF84D00D8
:1086100042F21172904201DA010001D14FF4FA6086
:1086200017B000BD10B596B00446684608F0A5FB2B
:10863000C4EBC4000DEB4000427A012A0CBF0120BC
:10864000002016B010BD10B596B00446684608F07C
:1086500094FBC4EBC4000DEB4000027B012A0CBF6D
:108660000120002016B010BD10B596B00446684633
:1086700008F083FBC4EBC4000DEB4000C07A0A286D
:10868000A8BF052016B010BD00B59DB0684608F023
:1086900049FB9DF8690020B11DB05DF804EB08F0BE
:1086A00045BB1DB000BD00B59DB0684608F03AFB63
:1086B0009DF80400012818BF00201DB000BD00B5C2
:1086C0009DB0684608F02EFBBDF802004FF6FF7122
:1086D000884218BF002803D040F2E931884203DB0A
:1086E0004FF4FA701DB000BD3228B8BF32201DB063
:1086F00000BD00B585B0684608F0F5FA9DF80400A5
:1087000005B000BD00B585B0684608F0ECFADDF8AC
:108710000500002814BF10F1010F2D4805B000BD61
:1087200080B584B0684608F0DCFA9DF804000128A2
:1087300018BF002005B000BD80B584B0684608F0C1
:10874000D0FA9DF80600012818BF002005B000BD32
:1087500010B584B00446684608F013FB0DEB040125
:108760000879030012BFFF280120A040C0B204B066
:1087700010BD00B585B0684608F0A6FA9DF8030064
:1087800005B000BD0F490860704700B585B0684668
:1087900008F0F9FADDF805000E490F4A0918914270
:1087A00028BF002005B000BD0000000000007F438E
:1087B0000000F041000070C1CDCC2C4000009EC2F2
:1087C00098060020907E0020000018419A99193FD9
:1087D00040E20100F0D8FFFF905F010000B585B0D6
:1087E000684608F0D0FA9DF80400012818BF002060
:1087F00005B000BD02460020032A18D8DFE802F0C9
:1088000002070B100879FF2810D108200FE04879E3
:10881000FF280BD102E08879FF2807D10A2006E063
:10882000C879FF2808BF6FF00E0000D07F3840B233
:10883000704710B5044608F045FA00F51C7105E0D4
:1088400010B5044608F03EFA00F518712046BDE860
:108850001040CFE780B584B0684608F099FA9DF8DB
:108860000400401E8041C043C00F05B000BD0100A0
:1088700018BFFF2801D10120704700207047000079
:10888000DFF8B807427800F11C010078FEF7B3BDAD
:1088900010B5DFF8AC47072104F11C0001F0D2FE4F
:1088A0000022227010BD2DE9FC4706460727002E46
:1088B0001446994600F089803078002818BFFF28B8
:1088C0001DD172788DF80020824202BFB2788DF8F7
:1088D0000020824213D1F2788DF80020824202BF3C
:1088E00032798DF80020824209D172798DF800200A
:1088F000824202BFB2798DF80020824265D08A465A
:10890000DFF8408770220021404602F08EFD50467D
:10891000FEF772FE08F1300585F800A0FFF73EFB78
:10892000A8702878032802D10A98687002E005F040
:1089300057FD07462F713A463146404602F061FD29
:10894000FFF720FBE870C8E90A49FFF763FA10B3A4
:10895000287804281DDA0721684601F073FE0722F3
:108960004146684602F056FD684600F02BFB80B990
:10897000E87880B108F029FB01460722684602F03A
:1089800049FD684600F01EFB401E8041C043C00FF9
:1089900002E0012000E0002088F818002878032871
:1089A00020D1DFF89C462A79414604F11C0008F0EA
:1089B00059FC88B9207840B9DFF88C26DFF88C168E
:1089C000201DFCF79EFD01202070002200210020C8
:1089D00003F06BFDBDE8F3870722414604F11C005C
:1089E00002F00FFD2878612810DB98F8180068B1B4
:1089F000FFF719FA50B90022002103F056FD0022BA
:108A00000021002000F081F8BDE8F3870FF20D018E
:108A1000404608F0FDF9BDE8F387000070B5FEF7A9
:108A2000E2FD50B9FEF7ECFD002801BFDFF8145657
:108A300005F131046078002803D0002200210020D5
:108A40005CE0E87905282FD108F04BFC30B12846CE
:108A5000BDE870400FF2994108F04BBCFFF7B7FB3F
:108A600000281EBF05F16501087800283ED0C878AF
:108A700006283BDA08F002FE012837D108F021FE73
:108A8000407D70B108F01DFE407D0B2804BFDFF86B
:108A9000C005FCF7B0F9BDE87040DFF8B8054168E3
:108AA00008470A22227021E0287EF8B1FFF78FFBE9
:108AB00000281CBF20780B2818D1FFF7B4F968B143
:108AC00001F0C5F890B9DFF88C657022294606F1EF
:108AD000080002F096FC0120307007E0DFF87425F2
:108AE0000FF245307121517008F05DFA002200212B
:108AF000002003F0DAFC207800220021BDE870405D
:108B000003E0DFF85015486070472DE9F74F86B055
:108B1000002007F0F1FC0E2101A801F093FD9DF863
:108B200018000E2201A900F0A8F9DFF81845DFF8B7
:108B30002885DFF82875054694F830006926042852
:108B4000CCBF5F210321401A8DF80100C1469DF87A
:108B5000010007F009FD8346E07905284FF0000A7F
:108B600040F08F8004F15F01C87AFFF780FE38B9CA
:108B70009826DFF8EC94EAB201A93046C847B4E081
:108B800004F15F00807A10EA0B012DD1387801A939
:108B900048556D1CEDB2DFF8C8946A26B87808B164
:108BA0009026C146C145E6D19DF8010001A948556E
:108BB0006D1CBAF1000FDED0DFF880440E22267063
:108BC000002104F11C0002F030FCEAB201A904F11A
:108BD0001C0002F016FC6570201DDFF88824DFF809
:108BE0008814FCF78EFC80E0FF2812BF8DF800107F
:108BF0000BF003008DF800009DF81CB09DF80010EC
:108C00009DF8010007F0B4FC9DF8000001A948554B
:108C10006D1CBBF1000FEDB206D09DF8200018BB13
:108C2000DFF83C9489261FE09DF8180000281EBF3D
:108C300004F15F018879002816D0FEF7D4FC98B9BA
:108C40009DF81800401E08D0401E0CD0801E08D091
:108C5000001F022898BF952606E0DFF804947C26C2
:108C600002E0942600E08026C14597D13B789DF82C
:108C70000020B4F85F0004F1580107F0A8F882461C
:108C80008CE7FFF7D0F878B1207E002883D000F081
:108C9000DEFF48B9DFF8D403FCF7ADF8012201A9E3
:108CA0009E2001F041FF20E0207E00283FF473AFBA
:108CB000FFF7B9F820B100F0CAFF00287FF46BAFCE
:108CC0009DF81800401E08D0401E0CD0801E08D011
:108CD000001F022898BF952660E7DFF884937C2662
:108CE0005CE794265AE7802658E709B0BDE8F08F84
:108CF00038B5D44D06280C4618BF85F8310095F8D4
:108D0000310000220021FFF700FF21462846BDE880
:108D1000344008F06CBB2DE9F04784B007460C46A0
:108D2000904699460E21684601F08CFC0E220021E7
:108D3000684602F07AFB0025C24EF079B24605285B
:108D400004BF06F1580AB6F85F500E2200216846AB
:108D500002F06BFB07225146684602F052FB0922E3
:108D6000842FADF807501BD0822F03D18DF80990C6
:108D70000A2215E0832F18BF872F07BF8DF80990AF
:108D80008DF80A408DF809408DF80A800B22852F56
:108D900006D104220CA90DF10B0002F032FB0F22C8
:108DA0006946384601F0C0FE04B0BDE8F08710B552
:108DB000040002D1FFF7C0FC00B101242246BDE847
:108DC000104001210020A0E69E48B0F85F007047E7
:108DD0009C48C179052901D10120704700207047C6
:108DE0009C480078704738B59A4D04462878C8B139
:108DF000702205F10801934802F003FB2046FFF7BB
:108E0000C1FC7120687005F108000FF21D0108F027
:108E1000D2F8002028700122BDE8384094499548D6
:108E2000FBF768B931BD000038B584B004460E21A7
:108E3000684601F007FC04B9824C864D6878932897
:108E400004BF0021E171E0798DF800000222217C4D
:108E50008DF801100DF1020004F1120102F0D1FAB7
:108E6000072204F1580101A802F0CBFA68780B221E
:108E7000694601F059FE05B030BD2DE9F8430446BE
:108E80000D4690460021284602F0CFFA00276D4E8D
:108E9000F079B146052804BF06F15809B6F85F70AD
:108EA00042460021284602F0C0FA072249462846D9
:108EB00002F0A7FAA5F807700920F179052915D164
:108EC000611E012906D9C91E0AD0091F022907D926
:108ED000BDE8F283FFF79FF968720A20BDE8F283CC
:108EE00006F15F00407AA8726C720B20BDE8F28335
:108EF0002DE9F84388B00E2104A8524E01F0A2FBE0
:108F000006F12107002438780125F0B90E2200214E
:108F100004A802F08AFAF079A046B146052804BFF9
:108F200006F15809B7F83E800E22002104A802F08D
:108F30007CFA0722494604A802F063FAADF81780CC
:108F4000092204A9862001F0EFFDB08B48BB0E2159
:108F5000684601F077FB0E220021684602F065FAB0
:108F6000F0790025A046B146052804BF06F158094E
:108F7000B7F83E800E220021684602F056FA07221A
:108F80004946684602F03DFAADF807800922694675
:108F9000842001F0C9FDFFF71AF910B1FFF7C0FBFB
:108FA0000446B28B2146284600F036F8002D08BF53
:108FB000002C04D1387C00220021FFF7A6FD09B067
:108FC000BDE8F083F8B50446FEF742FF0546FEF71C
:108FD00036FFC10703D42A7823789A421AD1012197
:108FE0006A1C631C20FA01F4E40703D416781C7889
:108FF000A6420FD1491C20FA01F4E50703D45578A5
:109000005F78BD4206D1491C9B1C921C0729E9DBF5
:109010000120F2BD0020F2BD70B504460D46164693
:1090200055EA04001CBF0A48FBF7E5FE3246294614
:109030002046BDE8704003F038BA0000147C0020E0
:10904000B87C002090790020A02526009188000897
:1090500054AB010890040020F7730008C079002089
:1090600071740008400D030081880008CCAA010833
:1090700080841E0018AC010880B50FF27900FAF761
:10908000BBFF0FF2C510FAF7BFFF0FF24D20FAF742
:10909000BFFF0FF2AD00FAF7C3FFBDE802400FF2C9
:1090A000F120FAF7B9BF80B501280FD1FDF7EAFD2D
:1090B000807B58B9FEF7E2FF40B9FEF737F818B1E8
:1090C000FDF7E0FD807B08B1002002BD012002BD5C
:1090D000DFF8380C818840886422A1E1DFF82C2C6D
:1090E000518010707047DFF8240C0278408800210E
:1090F00096E1000080B5DFF8142C5080918002F1D9
:109100000801DFF8AC0C01F07FFABDE80140FBF785
:109110009FBFE0B5FEF710F880B96846FFF7F7F992
:10912000684604F0D9F904F0B7F9022004F0D8FB3E
:109130004FF48071DFF87C0C02F04DF803B000BDF5
:1091400080B5FDF79FFD007A00287CD0FDF79AFDE1
:10915000C0790B2877D0FDF795FDC079FDF7DCFDD0
:1091600058B1002005F0D4F9FDF78CFD0021017203
:10917000FDF788FD002181723DE0FDF783FDC07998
:10918000FDF7D6FD00283ED0FDF77CFDC079FDF748
:10919000E7FD60B1FDF776FD807B40B905F0B8F9D9
:1091A00006F0FAFD01460222682001F0BDFCFDF741
:1091B000C3FF08B900F0D9F9FDF764FDC07A18B112
:1091C000DFF8F40BFCF7D4F9FDF75CFD807B50B1C0
:1091D000FDF758FD0021817306F0DEFD01460222F5
:1091E000682001F0A1FCFDF74DFD007B18B3FDF7F1
:1091F00049FD0021017306F0CFFD014602226820DF
:1092000001F092FC17E0FDF73DFDC079FDF7B5FDDB
:1092100088B106F0C1FD01460222682001F084FCFD
:10922000FDF730FD00210172FDF72CFD0021817258
:10923000002005F06DF9BDE80440DFF8801BDFF881
:10924000700B01F0E1B901BD10B5FEF7B3FE0446A5
:10925000FDF772FF00283ED1652000F059FA002882
:1092600039D0FDF70FFD1322002102F0DEF806F0E1
:109270008CFDFDF707FD6521017106F08DFD048071
:1092800006F08DFD00210180FDF7FCFC0446FEF791
:10929000F5FE08B1052008E006F07EFD4FF6FE71F0
:1092A000008888420CBF03200120E071FDF7EAFC32
:1092B000C0790A280ED1FDF739FF002814BF00201D
:1092C000062005F025F9FEF7E5FE18B906F067FD62
:1092D0000021018048E010BD10B5FEF78EFE044667
:1092E000FDF72AFF00283ED19C2000F011FA00284B
:1092F00039D0FDF7C7FC1322002102F096F806F0E2
:1093000044FDFDF7BFFC9C21017106F045FD048082
:1093100006F045FD00210180FDF7B4FC0446FEF790
:10932000ADFE08B1092008E006F036FD4FF6FE71EB
:10933000008888420CBF08200720E071FDF7A2FCDE
:10934000C0790A280ED1FDF7F1FE002814BF0020D5
:10935000062005F0DDF8FEF79DFE18B906F01FFDAA
:109360000021018000E010BDFDF78CFC012141725D
:10937000FDF7E2FE0446FDF785FC2146C0790FF6B5
:1093800091130FF20942BDE8104006F064BD0000E1
:1093900010B5FEF729FE0446FDF7CEFE00283ED1AB
:1093A0006F2000F0B5F9002839D0FDF76BFC1322CF
:1093B000002102F03AF806F0E8FCFDF763FC6F21AB
:1093C000017106F0E9FC048006F0E9FC002101804F
:1093D000FDF758FC0446FEF751FE08B1062008E0F0
:1093E00006F0DAFC4FF6FE71008888420CBF0420BC
:1093F0000220E071FDF746FCC0790A280ED1FDF786
:1094000095FE002814BF0020062005F081F8FEF725
:1094100041FE18B906F0C3FC00210180A4E710BD8D
:1094200070B504460E461546FDF786FE002840F04E
:109430009B80284600F06CF9002800F09580FDF72D
:1094400021FC1322002101F0F0FF06F09EFCFDF745
:1094500019FC057106F0A0FC048006F0A0FC068053
:10946000FDF710FC0646FEF709FE60B1652D08BF4A
:10947000052046D06F2D08BF062042D09C2D14BF7A
:109480000A2009203DE0652D09D106F085FC4FF644
:10949000FE710088884214BF0120032031E06F2D47
:1094A00009D106F079FC4FF6FE710088884214BF9E
:1094B0000220042025E09C2D09D106F06DFC4FF61A
:1094C000FE710088884214BF0720082019E0312D62
:1094D00008BF142015D01C2D18BF2F2D10D03F2DE4
:1094E00008BF12200DD03E2D08BF0C2009D0342D0E
:1094F00008BF162005D04B2D14BF1320172000E005
:109500001020312DF07105D04B2D06D1FDF7BAFB9F
:10951000312101710120FDF706FEFDF7B3FBC07993
:109520000A280ED1FDF702FE002814BF00200620F5
:1095300004F0EEFFFEF7AEFD18B906F030FC240C87
:109540000480FDF79FFB01214172FDF7F5FD044604
:10955000FDF798FB2146C0790FF2B5730FF22D226B
:10956000BDE8704006F077BC70BD80B5FDF78AFBA2
:1095700000210172FDF786FB00214172FDF782FB9D
:10958000002181720020FDF7CEFDBDE8014000F012
:1095900043BC3EB5FDF776FB0422002101F045FFF8
:1095A00006F0F2FB06F0B2FD06F0EEFB06F049FE17
:1095B000FDF7C2FD0446FDF7B9FD054606F0E4FBE4
:1095C0002246294606F052FEFDF75CFB044606F0F3
:1095D000DBFB0822C07C8E21FEF7E5FB6070FDF707
:1095E00051FB01460222212001F09EFAFDF74AFBC1
:1095F0000121817300F010FC03F056FF0FF66000AC
:10960000D0E90023CDE9002306F0BEFB007DFEF784
:109610007DFB8DF80000FEF752FF8DF80300FEF78A
:10962000F7FE8DF80400684603F056FFDFF8900758
:10963000FAF714FDFEF787FDDFF88827DFF8883793
:109640000021118018800020DFF88017DFF88027C4
:109650000870DFF88017DFF88007FBF752FFDFF8AC
:109660007C270FF27D61DFF87807FBF74AFF03B034
:1096700030BD38B500208DF80000FDF703FB007AFF
:1096800010B10C218DF8001001226946312001F043
:109690004BFA9DF800000C2839D0FDF7F3FA0B21A6
:1096A000C171FDF749FD0446FDF740FD0546FDF794
:1096B000E9FA2246C079294606F00DFCFDF7E2FAE8
:1096C000012101720B20FDF7FBFB092004F020FFB4
:1096D00003F0EAFEFEF737FDDFF8E826DFF8E836AC
:1096E0000021118018800020DFF8E016DFF8E02666
:1096F0000870DFF8E016DFF8E006FBF702FFDFF89E
:10970000DC260FF2DD51DFF8D806FBF7FAFE31BD9B
:1097100038B50446FEF7B2FC0546FDF7B3FA007A09
:10972000E8B1652C1CBF6F2C9C2C29D0212C18BFB4
:10973000312C0BD0342C18BF3E2C07D03F2C18BF37
:10974000482C03D01C2C18BF2F2C19D10C208DF8BD
:10975000000001226946204601F0E6F910E0FDF71D
:1097600091FA407A60B91C2C18BF2F2C0AD14DB148
:109770000C208DF8000001226946204601F0D4F942
:10978000002032BD012032BDC2E7000038B5FDF730
:1097900079FA00214172FDF775FAC079172809D1CD
:1097A0000120FDF7C6FCDFF83C0602690021904766
:1097B000FAF7D0FC06F0F5FA072808D1FDF762FAAF
:1097C000C07901281FD1FDF75DFA0321C171FDF7B2
:1097D00059FA0079312840F09A8006F0D5FA06F05F
:1097E00086FC002840F09380FDF7A6FC002840F09E
:1097F0008E80FDF79BFC002840F0898006F0CCFAB3
:109800000146022213E1FDF73DFAC079022803D197
:10981000FDF738FA0421D9E7FDF734FAC0790728B3
:1098200003D1FDF72FFA0821D0E7FDF72BFAC07915
:10983000132803D1FDF726FA0D21C7E7FDF722FA19
:10984000C079142803D1FDF71DFA1521BEE7FDF7F5
:1098500019FAC079122809D0FDF714FAC079102836
:1098600004D0FDF70FFAC0791628B0D1FDF70AFA37
:1098700000214172FDF706FA00218172FDF756FCC6
:1098800030B90122DFF84815DFF85C05FAF732FC41
:10989000FDF7F8F90C210170FDF7F4F90121417190
:1098A000FDF7F0F9C07910280FD1FDF7EBF91C2175
:1098B0000171FDF7E7F90446FDF7E4F90546FDF708
:1098C000E1F9627900792946B2E0FDF7DBF9C07968
:1098D000122803D1FDF7D6F93F21E9E7FDF7D2F9C8
:1098E000C079142803D1FDF7CDF93121E0E7FDF768
:1098F000C9F9C0790A28DCD0FDF7C4F9C0790C2871
:10990000D7D0FDF7BFF9C0791628D2D079E2FDF79C
:109910000DFC50B1FDF7B6F9C079172816D000201C
:1099200004F0F6FDFAF73EFC10E0FDF7ABF9C07964
:10993000102807D10022DFF8B414DFF8B404FAF7D6
:10994000D9FB03E0DFF8AC04FAF788FBFDF736FA41
:10995000F0B1FDF797F900791C2819D0FDF792F9BD
:1099600000792F2814D0FDF78DF900210170FDF743
:1099700089F901214171FDF785F90446FDF782F966
:109980000546FDF77FF962790079294601F0CCF8A8
:10999000FDF778F9C079FDF726FA002876D0FDF7B3
:1099A00071F96D210171002406F0EEF906F09BFBC0
:1099B00000283ED1FDF766F9C0790D2809D0FDF7E2
:1099C00061F9C079152804D006F0DEF906F08FFBA6
:1099D00078BBFDF7ABFB30B90122DFF8F413DFF8F9
:1099E0000804FAF787FB06F0D7F90446FDF74AF9B1
:1099F0000222214601F005FDFDF744F90446FDF77A
:109A0000E4F9A070FDF73EF903214171FDF73AF941
:109A10000446FDF737F90546FDF734F96279007918
:109A2000294601F081F806F0B7F9022201466820C4
:109A3000E4E106F0A9F906F05AFB01280AD1FDF786
:109A400021F9C079FDF7DFF920B1FDF71BF9642199
:109A500001240171FDF716F9C079FDF7D4F900284A
:109A600066D006F091F906F03EFB012809D106F018
:109A70008BF906F03CFB012803D1FDF703F96421C3
:109A800002E0FDF7FFF86D21017151E0FDF7FAF8F2
:109A90000024C079401E16284DD8DFE800F0353587
:109AA00029251D192D2115114C3A4C4C4C484C447C
:109AB0004C4C4C3F0C00FDF7E5F8012464212BE0F1
:109AC000FDF7E0F87B2127E0FDF7DCF89C2123E09F
:109AD000FDF7D8F86F211FE0FDF7D4F865211BE0F2
:109AE000FDF7D0F89B2117E0FDF7CCF8772113E0C4
:109AF000FDF7C8F878210FE0FDF7C4F801240473DE
:109B0000FDF7C0F89B2107E0FDF7BCF801240473C2
:109B10000EE0FDF7B7F86D21017109E0FDF7B2F82D
:109B20003421017103E0FDF7ADF83F2101710124FB
:109B3000204600F001F831BD7CB50446FDF7FCFA83
:109B40000546FDF7F3FA0646FDF79CF82A46C0796C
:109B5000314606F0C0F906F017F9014668460F31A4
:109B60000622FAF78DF9DDE9000107F0C7FD5CB1C7
:109B7000FDF788F80121817206F006F90FF20D1148
:109B8000408B00F029F873BDFDF7D0FA002814BF10
:109B90000020062004F0BCFCFDF749F9FDF772F83F
:109BA00001210172FDF76EF801210173FEF7DCFA65
:109BB0008449854B00220A8018800020834A854909
:109BC0001070834A8448FBF79CFC844A0FF2111101
:109BD0008348FBF796FC73BD38B5054684B00C4648
:109BE0000120FEF763FAADF800000220FEF75EFAEE
:109BF000ADF802000320FEF759FAADF80400042086
:109C0000FEF754FAADF80600ADF808500120FEF753
:109C100075FA8DF80B000220FEF770FA8DF80C0033
:109C20000320FEF76BFA8DF80D000420FEF766FAAC
:109C30008DF80E00200003D02146684604F033FF63
:109C400005B030BD80B5FDF71DF8007A02BD80B5C6
:109C5000FDF718F8407A58B9FDF714F8007A38B9CA
:109C6000FDF710F8807A401E8041C043C00F02BD4E
:109C7000012002BD80B5FDF705F8407B02BD10B59F
:109C80000446FCF7FFFF447310BD000038B5FCF735
:109C9000F9FF00218172FCF7F5FF0121017206F046
:109CA00073F8044606F070F8054607F059FEB4F85C
:109CB0001720B5F8151006F0AFFBFCF7E3FFC079ED
:109CC000102808D1FCF7DEFF012141730020BDE818
:109CD000324008F026B8BDE83240002007F056BEFA
:109CE00080B5FCF7CFFF007A78B1384908780128B1
:109CF00004D1BDE802401020FDF7E2B8BDE80840FD
:109D0000334A3D493648FBF7FCBB01BDAC06002099
:109D100038B5FCF7B7FF00214172FCF7B3FF002113
:109D20008172FDF703FA20B9012229492E48FAF77A
:109D3000E1F9FCF7A7FF0C210170FCF7A3FF01215B
:109D40004171FCF79FFFC07910280FD1FCF79AFFF3
:109D50001C210171FCF796FF0446FCF793FF0546B2
:109D6000FCF790FF62790079294647E0FCF78AFF0B
:109D7000C079122803D1FCF785FF3F21E9E7FCF702
:109D800081FFC079142803D1FCF77CFF3121E0E783
:109D9000FCF778FFC0790A28DCD0FCF773FFC079A4
:109DA0000C28D7D0FCF76EFFC0791628D2D028E057
:109DB000947E002000100140CC7B0020BC060020D7
:109DC00000AC0108DE7C0020E07C0020DC7C002070
:109DD00040420F00B9560008E47C0020E0930400E4
:109DE000347D002098060020F0AB010880841E001E
:109DF00030AC0108E0AB0108E19C000800F094FEE3
:109E000031BD05F0C9FF02220088ADF800006946A7
:109E1000742000F089FE31BD80B505F0B5FF06F075
:109E200066F9B0B9FCF72EFFC079122811D0FCF703
:109E300029FFC07901280CD0FCF724FFC079022843
:109E400007D0FCF71FFFC079072802D0FDF774F98F
:109E500028B104F05AFFBDE8014007F084BD01BD00
:109E600000B10F0000000000C11768B14840401A5F
:109E7000B0FA80F29040D21CC907C2F5846241EA70
:109E8000025202EBD0214005704700002DE9FC4D45
:109E90008AB00646DDE90A450F4624F0000035F099
:109EA000004108BF002800F051830020DFF8A81609
:109EB00032463B4608F018F800F04883DDE90AAB6B
:109EC000DFF89816CDF800B008F00EF806D168005B
:109ED0004015401C02D1290300F03883580040157A
:109EE000401C019700F0498237F0004308BF002A68
:109EF00000F043826A005215521C00F03E824FEA85
:109F00004B0353EADA734FEA4A0208BF002A1CD017
:109F100040F23340A0EB5352352A04DB0AF0000A2A
:109F20000BF0004B11E0202A05DD203A2BFA02F05D
:109F300000FA02FB00E002D14FF0000A05E0002A1F
:109F4000C4BF2AFA02F000FA02FAFA0F20D0002D5C
:109F500005D500224FF00043141B63EB0505CDE946
:109F600000455B46002B524605D500244FF00045C6
:109F7000A21A65EB0303DDE900459D4208BF944248
:109F800006D0AFF300804FF0FF306FF0004124E3C4
:109F90003B4623F00041B1F5801F09D2002000901C
:109FA0006A463046394607F0AFFF04460D460CE0DE
:109FB000DFF8AC45DFF8AC7504EB11503B40DFF83F
:109FC000A8150090344643EA0105E80F08BF0022B7
:109FD00043D04FEA4B0353EADA734FEA4A0208BF11
:109FE000002A25F00045504659461CD040F2344620
:109FF000A6EB5352352A04DB0AF0000A0BF0004BA3
:10A0000011E0202A05DD203A2BFA02F303FA02FBC5
:10A0100000E002D14FF0000A05E0002AC4BF2AFA8E
:10A0200002F303FA02FA002905D500224FF000439B
:10A03000101A63EB0101BBF1000F06D500224FF0AF
:10A040000043B2EB0A0A63EB0B0B594508BF5045BE
:10A0500002D10021049101E001220492009801281C
:10A0600033D120462946DFF80425DFF8043507F010
:10A0700083FF2AD20A4600265000400D4FF0000808
:10A08000DFF8D47400F1010311D0002B0FDD40F292
:10A09000FF70834206DBDFF8DC5401F0004100244E
:10A0A0000D4333E06FF31E5242EA03552EE024F0D5
:10A0B000000035F0004108BF002827D001222946C2
:10A0C00007F072FF04460D4620E00020DFF8A814D8
:10A0D00022462B4608F006F8DFF88C7400223B4637
:10A0E00008F0D2F808F08EF9A0F120084046FFF7FA
:10A0F000BBFE0022DFF8843407F0F4FF00223B4669
:10A1000008F0C2F806460F464FEA4818204629468E
:10A1100032463B4608F094F982468B4632463B462F
:10A120002046294608F0B0F802460B4650465946EC
:10A1300008F0F8F9CDE90601DDE9062307F0D2FFC2
:10A14000CDE90201DDE90223DFF83404DFF834143D
:10A1500007F0C8FFDFF83024DFF8303408F094F857
:10A16000DDE9022307F0BEFFDFF82424DFF8243402
:10A1700008F08AF8DDE9022307F0B4FFDFF81824BD
:10A18000DFF8183408F080F8DDE9022307F0AAFFB1
:10A19000DFF80C24DFF80C3408F076F8DDE9022350
:10A1A00007F0A0FFDFF80024DFF8003408F06CF8B7
:10A1B000DDE9022307F096FFDFF8F423DFF8F4333C
:10A1C00008F062F854465D4682468B460020DFF870
:10A1D000881332463B4608F033F90E467200520DA2
:10A1E00002F1010712D0002F10DD40F2FF729742FA
:10A1F00006DBDFF8807301F0004300261F4312E006
:10A200006FF31E5646EA075706460CE020F00002A0
:10A2100031F0004304BF002A002603D0012207F0DA
:10A22000C3FE06460F46DDE9020152465B4607F0D3
:10A2300059FF22462B4608F003F932463B4608F008
:10A2400023F8DDE9062307F04DFFC24A7A4402F500
:10A250004172424403922B46224608F015F882468A
:10A2600000988B46FFF700FE039CD4E9002308F01A
:10A270000BF806460F46DFF84003DFF8401352465E
:10A280005B4607F02FFF32463B4607F0FDFFDDE956
:10A290000A2307F027FF0022DFF8243307F06CFEC3
:10A2A00062D30122DFF81C3308F060FA59D9CA0FD3
:10A2B0001ABF0022C44BAC4B07F0E6FF08F0A2F82F
:10A2C0000022A54BC14CC24DCDE901238046DDE9FA
:10A2D0000A23CDF800805046594607F003FFDDF809
:10A2E0000CC082468B46DCE90223DCE9040107F05E
:10A2F000CBFFDDE90A2307F0F5FE22462B4607F0E7
:10A30000F1FE52465B4607F0BFFFDDE90A238246B5
:10A310008B463046394607F0E5FE06460F46404676
:10A32000FFF7A2FD02460B463046394608F088F892
:10A3300022462B4607F0D6FE52465B4607F0A4FFA6
:10A34000DDE9012308F02AFA20F0000431F000458D
:10A3500008BF002C08D04A005215521C06D10B032E
:10A3600004D10020834901E000200021049A002A42
:10A3700000F0EE8081F000412FE17800401510F1EF
:10A38000010C04D1380302D03046394625E169007A
:10A390004915491C05D1280318BFDDE90A0140F021
:10A3A000D7806A0001205215521C00F089802B468C
:10A3B00022464FEA430B5BEAD27B4FEA420A08BFD0
:10A3C000BAF1000F1DD040F2334EAEEB5B5EBEF132
:10A3D000350F04DB02F0000203F0004311E0BEF190
:10A3E000200F04DDAEF12002D340934000E001D104
:10A3F000002206E0BEF1000FC4BF22FA0EF202FAFC
:10A400000EF2CDE902232B000AD54FF0000A4FF0DF
:10A41000004BBAEB04026BEB0303CDE9082301E028
:10A42000CDE90843DDE90223CDE90623002B05D55C
:10A4300000244FF0004BA21A6BEB0303CDE9042379
:10A44000DDE908ABDDE904239B450CBF9245002004
:10A45000DDE906235C0054EAD2744FEA420A08BFE1
:10A46000BAF1000F18D040F2344EAEEB5454352CF4
:10A4700004DB02F0000203F000430DE0202C04DDB9
:10A48000A4F12002D340934000E001D1002203E078
:10A49000002CC4BFE240A24090B1DDE904ABCDE99D
:10A4A00002AB002B05D500204FF00044821A64EB6C
:10A4B0000303DDE902AB9B4506BF92450020012066
:10A4C000BCF1000F06D13A0304D1FE0F17D1EC0FF7
:10A4D00039D032E0D1B92A0318D127F00041B1F5C3
:10A4E000801F26F000001CD20022002908BF00288F
:10A4F00000921AD06A46394607F006FD15E0EC0FC7
:10A5000002D1002820D01BE038B965E0002814BF34
:10A51000FE0F0026EC0F12D17EB100204FF000415B
:10A520005BE00F4A02EB11500090EC0F009802D153
:10A53000002808DC01E0002805DD00204CE016B111
:10A540000020244949E000200A4946E00020024951
:10A5500043E000BFBCEC00000000F03F0000F0BF93
:10A5600002FCFFFFFFFF0F800000E03FCD3B7F6656
:10A570009EA0E63F0000F07F000050400000903FAA
:10A58000F7DE29BFD8F8C23FF4B3FECC1A99C33F17
:10A5900062CB68D96F46C73FC6C912DAC471CC3FD7
:10A5A0004AE98A942449D23FF75F97999999D93F0C
:10A5B000BC5555555555E53FFE822B654715F73F70
:10A5C0000000E0C00000E0400000E0BFEF39FAFE0C
:10A5D000422EE63F0000F0FF00210CB0BDE8F08DF8
:10A5E000400D491840EA81200CD2490DA1F5806147
:10A5F000491C40F0004005DBD1F11F0154BFC840A9
:10A60000C01770470020704780B572B60A680AB953
:10A6100008F07AFA62B601BDF8B506460D4600208C
:10A6200072B645B137462C46384608F077FA10B96D
:10A630003F1D641EF8D162B60028F1D000210160F0
:10A64000F2BD0000002201F0D3BA0000002102F0A8
:10A65000EAB938B5044607F094F90128DFF8C45385
:10A6600007D100F085F9A87B012818BF00202874C5
:10A6700031BD02F0F8F9287418B12046BDE8344025
:10A68000DCE131BD10B5044607F07BF980B900214B
:10A69000DFF894230870DFF8941300F065F806F0F3
:10A6A000FFFA214606F0F4F906F0E4FA00B210BD14
:10A6B000002010BD38B50C4640F2FF750AB940F2D3
:10A6C000FF35401B06F0ECFA214606F0E1F904469E
:10A6D000284605F089FF214606F046FA06F0CAFA38
:10A6E00080B232BD3EB5DFF838530446287EB8B993
:10A6F00001218DF8001020706A68002A1CBFA9682B
:10A70000002917D0684600F02FF89DF8001011B905
:10A7100000226A60A9609DF80010217003B030BD6E
:10A72000002001900021009100230022204600F02B
:10A73000E0F800B203B030BD0A46002300211970D2
:10A740000146002010E0002181600160017141712B
:10A7500070471CB500242470009313460A46014636
:10A76000002000F03AF816BD70B504460D461646B6
:10A77000012002F06DF92968B1B9701C697910F8EF
:10A78000110028B902F064F90020687104B120704A
:10A790006879721C014612F811301B022B60401CB4
:10A7A00016F81110A96068712868401E2860297980
:10A7B000481E2871C0B230B9A86838B12871B5F9FF
:10A7C0000C004042A881B5F90C0070BD02F040F9C0
:10A7D0002879401C2871002070BDF8B516460C463B
:10A7E000311D227951F832100546206888421F46F3
:10A7F00007D1012002F02CF9002121602079401CB2
:10A8000020712079B84208D10021217101202870DF
:10A81000A181002002F01CF91BE0012002F018F9D0
:10A82000207956F83050A07B80B92846002108F0E6
:10A8300083F907D0069B20687D4A294603F01CF95E
:10A84000A08103E00020A08102F002F92068401CF2
:10A850002060B4F90C0080B2F2BD000010B50446CF
:10A86000FDF7F8FF08B9012C40D1641E21D0641E09
:10A870000FD0641E15D0A41E03D0E41E0C2C1ED9CC
:10A8800027E0674872A1016000F170028260042332
:10A890001DE063486749016000F1500282600823AF
:10A8A00015E05F486449016000F1600282600623A0
:10A8B0000DE05B486EA1016000F1800205E05848A0
:10A8C00000F1A001016000F1900282600123436168
:10A8D00004E05348002141608160416100218068AB
:10A8E00001607F22017141718160828110BD1B2056
:10A8F00070477FB59DF9205004460020012D8DF84A
:10A90000040003DB2846FFF7A9FF23E00998D5B927
:10A910000021434D21702A68002A1ABFA968002926
:10A92000002018D0009001A86B69FFF756FF06467B
:10A930009DF8040020B1002100202960A86000E0FB
:10A940000120207006E00025257000902046FFF7CA
:10A9500044FF0646B0B204B070BD31494876704736
:10A960002F48407E70472F4A1060516070470000AA
:10A9700010B52C4C2089617B401C2081E07A401C62
:10A98000E072C0B2884213D30020E072217B481EDF
:10A99000A17B8041C00F0129207305D120B16168DE
:10A9A000206800F016FC03E06168206800F013FCEA
:10A9B000A07A052828D8DFE800F009120309121E42
:10A9C00021890222A273B1F5166F06E00122A2735B
:10A9D000082122896173B2F5166F15DB07E00121AA
:10A9E000A173052221896273B1F5166F0CDB002279
:10A9F0002281401C07E021890220B1F5FA5FA07393
:10AA000002DB00202081A072A07BBDE8104002F094
:10AA10001FB80448007C7047024900200874704742
:10AA2000881E0020381F002038AA01084C1F002073
:10AA300000007A45F8A7010838A80108012101F0B3
:10AA4000E3BF00000908080810080E0809080008FC
:10AA50007BD49243D0070000A4D08243D0070000EB
:10AA60007BD49243D007000000000000B80B000028
:10AA70000000DC43D0070000C0F3C75181B1FF29BB
:10AA800006D0C110400721F0E04101F1605170474C
:10AA900041020CBF40F4E0016FF00041002070471C
:10AAA00000F0004100020AD0B0FA80FC00FA0CF07D
:10AAB00001F16051A1EB0C5101EBD0214005704731
:10AAC00008B438B585B009AC002504940395002975
:10AAD0000EBF01950190491E0291009504AB01A99A
:10AAE000074878441A3008F035F8019901B10D7023
:10AAF000002858BF039806B030BC5DF808FB00BFC3
:10AB00002794FFFF80B5DFF82416002008700A2084
:10AB100003F0FEFC8D2001F0BCFFBDE802400020E8
:10AB2000FEF7F7BAFEF7DFBA03F0ADB980B500F073
:10AB3000FFFBDFF8FC25DFF8F815B0FBF2F201FBB4
:10AB400012000090042269463A20D1E280B500212B
:10AB50008DF800100078FEF7A6FAB0B1FCF7E0FA25
:10AB600028B1FCF79AF810B9FEF7EAFA01E0FEF70F
:10AB7000FCFCFCF792F810B9FAF740FA02E00A2060
:10AB800003F0C6FC0020FFF7BDFF0122694620202C
:10AB9000AEE2FEF7FEBC38B500250229144628BFF8
:10ABA00045780378472C03D1184602F01DF9034677
:10ABB0002A4621461846BDE83840FCF78DBC80B5D2
:10ABC00000208DF80000FBF7F0FADFF8600501784F
:10ABD000022908D0FCF7B0FA28B94FF48071DFF8E9
:10ABE000540500F0F8FA01226946232080E210B5EE
:10ABF000DFF84445204608F085FF2278BDE8104084
:10AC00000146292003F03FB980B500208DF80000EF
:10AC1000FBF7CFFA012269461D2003F046F9FBF746
:10AC2000CFFA642002F028FEFBF770FA01BD002085
:10AC3000FCF75ABA80B5FEF751FABDE808404CF26D
:10AC40005032DFF8F814DFF8F804FAF75ABC80B590
:10AC5000FDF76FFB8DF8000001226946302047E2C6
:10AC600080B508B1022901D2032003E041780078C1
:10AC7000FDF75AF98DF80000012269464F2037E2AE
:10AC80007CB5054614460E462046FCF791F810B1F7
:10AC9000FEF7EFFC73BDFDF7F1F9002818BF342C67
:10ACA00006D03E2C1CBF3F2C482C01D00C2036E196
:10ACB000224629463046FEF7B3FB73BD80B500201F
:10ACC0008DF80000FEF73CFA0122DFF86414DFF88B
:10ACD0007404F9F70FFA01226946362008E280B5BC
:10ACE00000218DF800108179C2794379090441EA85
:10ACF0000261027941EA032111438278C378120488
:10AD000042EA03624378007842EA0322104308F0E3
:10AD10000BFF8DF80000012269463720E8E180B57D
:10AD200000208DF80000FEF720FCFAF751F9012011
:10AD3000FCF753FA0220FCF750FADFF80C044FF44A
:10AD40000051016008220260FCF720FADFF8FC03E2
:10AD500004F071FDDFF8F81380200860DFF8F403D9
:10AD6000FAF749F8012269463820C1E110B50446D6
:10AD700005F01AF801460622392003F084F820462F
:10AD8000BDE8104005F01EB8E0B568460021C0E9F6
:10AD9000001100F0D4FA082269463B2021E080B57A
:10ADA00002218DF80010332804BF00218DF8001017
:10ADB000012269469CE10FF2EC3100B5D1E9002394
:10ADC00083B001A9CDE9012302680A6042684A60A4
:10ADD00001A802F081FB00218DF8001001226946D4
:10ADE000432003F050F803B000BD10B584B0044612
:10ADF00001F045FE0090002101A80022002380E818
:10AE00000E000422694600F0FCFA02A800F097FA4E
:10AE10000C2213E018B583B0044601F033FE009015
:10AE2000052101A8FFF70EFC0422694601A800F0E5
:10AE3000E8FA01F02AFE8DF80800052201A9204653
:10AE400003F021F804B010BD80B500218DF800108A
:10AE50004FF480510378C04A002B104602D000F016
:10AE6000B8F901E000F0B7F9012269463C203FE162
:10AE700001B50122694642203AE1B84808F086BE91
:10AE80007CB50446FCF758F9002847D1452CB44D51
:10AE9000B44E3CD1FDF757F9B34AB44B00211180B1
:10AEA00018803170A24AB249B248FAF72AFBB24A76
:10AEB0000FF295012846FAF724FB9C4902200870FE
:10AEC00002F0F2FAB9A0D0E90023CDE90023002076
:10AED000FDF7B6FC8DF800000120FDF7B1FC8DF800
:10AEE00005000220FDF7ACFC8DF806000320FDF7FD
:10AEF000A7FC8DF80700684602F0EEFA092003F07F
:10AF000007FB4FF480718B4800F063F906E00220E4
:10AF100030709A4A9A492846FAF7F3FA00208DF8D9
:10AF2000000001226946204602F0ADFF73BD0120FA
:10AF300002F06FBC80B50020FAF78DF9BDE8024041
:10AF40000020FAF7E7BE000086480078022809D002
:10AF5000012804BF0020FFF7D5BD8A4A8A498048EE
:10AF6000FAF7CFBA704780B501F0C3FA00218DF827
:10AF700000008DF8011002226946402002F083FF94
:10AF800001F0B1FA01BD80B5007820B101227F49FE
:10AF90007F48F9F7AFF8FEF7E8FA0020FFF7B2FDB7
:10AFA00000208DF80000012269463220A0E080B523
:10AFB00001F051FFBDE8084001468822492002F017
:10AFC00062BF08F01FBF00002DE9F84183B0804642
:10AFD0000F4600208DF8000015463C780122694696
:10AFE000404602F050FF6E1E6A4DB0B228608021CC
:10AFF000281DFFF727FBB2B2791C281DF8F740FF88
:10B000002CB9424601210020FFF73AFE0FE0012053
:10B01000FCF78FF80120FCF792F802F045FA0920BE
:10B0200003F076FA4FF48071424800F0D2F800BF86
:10B0300060A0D0E90023CDE901230020FDF7F9FB52
:10B040008DF804000120FDF7F4FB8DF809000220C3
:10B05000FDF7EFFB8DF80A000320FDF7EAFB8DF802
:10B060000B0001A802F038FA4B4802690021904712
:10B0700044B1F9F76FF8404A0FF27D0105F1840001
:10B08000FAF73FFA04B0BDE8F08138B50446414D07
:10B0900005F18400FAF76CFA0020FCF74AF800206A
:10B0A000FCF74DF800208DF80000FEF75EFA002056
:10B0B0002860FBF7F2FD10B9F9F7A0FF02E00A20C3
:10B0C00003F026FA0020FFF71DFD01226946204605
:10B0D00002F0D9FE304802690021904702F0DCF905
:10B0E00031BD80B501208DF800000122694697200E
:10B0F00002F0C9FE01BD000080B5FCF723F800B1E5
:10B10000F0E726490120FEF767FD01BD80B501216A
:10B110008DF800100122694602F0B5FE03F0F5FD3E
:10B12000034A1F490E48FAF7ECF901BD4F0600200B
:10B1300040420F0000100140337D002025AB000885
:10B14000647D0020F0AB0108101001400034014084
:10B1500080E100E010AA01080008014071AE00087B
:10B16000F0780020DC7C0020DE7C0020E07C0020E9
:10B17000B9560008E47C0020A0860100804F120030
:10B1800005AB0008400D030049AF0008404B4C00E0
:10B1900008AC01086C78002098060020E3B0000895
:10B1A000F9B00008000000000000000000B100003D
:10B1B0000000000000B1000000000000002A18BFDD
:10B1C00002F0B5B802F0B6B80B460322102102F027
:10B1D00053B802F0ACB802F0ADB802F0AEB802F06D
:10B1E000AEB8022303224821274802F045B880B5B3
:10B1F0000121012002F0D9F801220021022000F0F3
:10B200004FF8022000F08CF82149204B00200870F4
:10B2100080221A6001BD1F4980200860022000F0D2
:10B220007FB80FB410B50B460322482102F024F872
:10B2300005990498C9B2C0B202F0B7F8069C9DF80F
:10B240001C200021204600F02BF8204600F068F872
:10B250009DF91D00020007D50F4C00F00F0121449D
:10B26000002301F8043C02E00C4900238B54012424
:10B2700000F01F00054904FA00F0520941F82200CD
:10B2800010BC5DF814FB0000000C014000E100E080
:10B2900007E400E080E100E018ED00E000E400E0F9
:10B2A00070B4214B1D68C44325401D605E68264074
:10B2B0005E609D6825409D60DE682640DE6029B1A5
:10B2C000012902BF5D6805435D6002E01968014322
:10B2D000196022B1022A0ED009D370BC7047996858
:10B2E00008439860D8680440DC6070BC7047996877
:10B2F0000C409C6002E0996801439960DA68104351
:10B30000D86070BC704708494A6909680140024228
:10B3100018BF002901D001207047002070470000AD
:10B3200000BF024908607047000401401404014056
:10B33000134908684A688968504048407047104A75
:10B3400013689168CB181B0EC37191681368CB18F2
:10B350001B0C837191681368CB181B0A43719168A9
:10B360001368CB18037153681B0EC3705168090C26
:10B3700081705168090A417051680170704700007E
:10B38000107AF01F70B484B00A2A6C4604D10028E9
:10B3900002D50123404203E0002301E004F8015BF1
:10B3A00008B96C450AD1B0FBF2F602FB160005465F
:10B3B0000A2D3046ACBF57353035EFE76A46A01A44
:10B3C00043B12D2301F8013B401C03E014F8013D7B
:10B3D00001F8013BA242F9D300220A7004B070BC0C
:10B3E0007047034642B113F8010B11F801CB521E0E
:10B3F000604503D1002AF6D100207047A0EB0C0075
:10B400007047130005D011F8013B00F8013B521EB4
:10B41000F9D170471044401E130005D011F801CB3C
:10B4200000F801C9521EF9D17047130003D00A4633
:10B43000194600F0F7BB704701460020CA0748BF15
:10B4400080208A0748BF40F040004A0748BF40F0CC
:10B4500020000A0748BF40F01000CA0648BF40F06D
:10B4600008008A0648BF40F004004A0648BF40F082
:10B470000200090648BF40F001007047002200E0CA
:10B48000521C8A4205DA10F8013BFF2BF8D000204D
:10B4900070470120704770B40346FF2400200A0063
:10B4A00007D01D4615F8016B3440FF2C03D1521E06
:10B4B000F8D170BC7047002213F8014B2243D4B27C
:10B4C0001CB9491EF8D170BC704770BC0120704790
:10B4D000DFF8B8064068B7E1DFF8B0064068DDE2A3
:10B4E00038B50546DFF8A8262968DFF8A846914256
:10B4F00031D140F2157002F005F8012105F121006B
:10B5000085F82010017000220021417069682868C8
:10B5100008F041FE286800230022002108F095FE73
:10B52000286808F0BFFE2868012108F09BFE286803
:10B53000A0420FD14FF4C06008F052FF0222002158
:10B54000212008F052FFBDE83840012200212220CE
:10B5500008F04BBF31BD2868A042FBD140F2167005
:10B56000C9E710B50446206808F000FEA16851F84C
:10B57000142F206902430A60A16851F8142FE06873
:10B5800002430A602369A0680322102101F074FEBF
:10B59000E368A0680322102101F06EFE00BF00BF27
:10B5A00000BF00BF00BFA16851F8102F20690243FF
:10B5B0000A6000BF00BF00BF00BF00BFA16851F814
:10B5C000102FE06802430A602369A06803221C214F
:10B5D00001F052FEE368A06803221C2101F04CFE3A
:10B5E0002046BDE810407BE770B504460D46164680
:10B5F00040F2036001F086FFDFF89405DFF898154C
:10B6000025608542A160666007D18021E16040200D
:10B61000DFF8781520610C600CE0DFF878058542D2
:10B6200008D14FF40061E1604FF48060DFF85C15F1
:10B6300020614C602046BDE8704092E770B5054639
:10B64000DFF8584540F2016695F8200000281CBF3D
:10B6500095F82110002904D02868314608F03CFEF6
:10B6600030B1641EF0D12846FFF77BFF002070BD8B
:10B67000012070BD2DE9FC41054600200F4616460D
:10B680001C46009040F2016895F820000028FBD08D
:10B6900095F821100029F7D02868414608F01CFED3
:10B6A0000028F1D185F82000286808F001FE2868FC
:10B6B0004FF4A06108F010FE0028F8D028686FF061
:10B6C0000102394608F0E5FD40F2024029681431D4
:10B6D00009680091009A0242F8D00098810716D5B7
:10B6E000286840F2015108F004FE200014D040F216
:10B6F00007573178286808F0E7FD2868394608F0D0
:10B70000EBFD0028F9D0761C641E05D0F1E728680F
:10B7100040F20A5108F0EDFD286808F0CEFD2868D7
:10B7200000688105FBD4012085F82000BDE8F38185
:10B730002DE9F8435FEA030904460D46904635D0EB
:10B7400094F820000028FBD004F12106307800286E
:10B75000F6D0206840F2016108F0BEFD0028EFD16C
:10B76000089F2068012108F07DFD20684FF4847156
:10B7700008F0CAFD206840F2091108F0C5FD2068F4
:10B780004FF4857108F0C0FDDFF814140020087034
:10B7900084F820007070A4F81C90C4F81480B57070
:10B7A000A7622068BDE8F24308F082BDBDE8F183DE
:10B7B0002DE9F047089C05462000894692469846A8
:10B7C0003FD095F820000028FBD005F12106307805
:10B7D0000028F6D0286840F2016108F07DFD0028BD
:10B7E000EFD1099F2868012108F03CFD28684FF43B
:10B7F000847108F089FD286840F2091108F084FD81
:10B8000028684FF4857108F07FFD00203070012119
:10B81000DFF88C0371700022427086F8029086F87F
:10B8200003A0A983EC83C5F81880022CAF6203D172
:10B830002868002108F022FD2868BDE8F04708F0DC
:10B8400037BDBDE8F0870000F8B5044604F12106D5
:10B850007078002876D1DFF848532A78062A00F25B
:10B860001C81DFE812F00700160024001A011A01FB
:10B870003F0057002068CB4908F066FD002800F023
:10B880000C81B17820686FF0010208F002FD012000
:10B890003EE0C54E2068314608F056FD002800F015
:10B8A000FC802068314608F075FD022030E02068F9
:10B8B000BE4908F049FD002800F0EF806069411C96
:10B8C000616140F202560178206808F0FDFCA08B0F
:10B8D000411EA1832068314608F0FEFC0028F9D003
:10B8E000052015E02068B14908F02EFD002800F081
:10B8F000D4806069411C61610178206808F0E4FC33
:10B90000A08B401EA08380B2002840F0C680062095
:10B910002870F1BD206808F0D0FC012084F82000D8
:10B920004FF48471206808F0FFFC20684FF48571A3
:10B9300008F0FAFC206840F2091108F0F5FC00203C
:10B940002870A5E0012840F0A880954D687805286A
:10B9500000F2A380DFE800F0031220374B6220687A
:10B96000904908F0F1FC002800F09780B178206839
:10B970006FF0010208F08DFC01204DE08A4E206836
:10B98000314608F0E1FC002800F08780206831464D
:10B9900008F000FD02203FE02068844908F0D4FC54
:10B9A00000287AD0F178206808F08EFC40F2025628
:10B9B0002068314608F090FC0028F9D0206808F093
:10B9C00077FC032028E02068764908F0BDFC0028B9
:10B9D00063D0B1782068012208F05BFCE08B03287B
:10B9E00003DA2068002108F03DFC042014E06E4ECC
:10B9F0002068314608F0A8FC00284ED02068314667
:10BA000008F0C8FCE08B012818BF022803D1206889
:10BA1000002108F027FC05206870F1BD206864490A
:10BA200008F092FC00281CBFE08B002835D00328CA
:10BA30000AD1206840F2025108F04EFC0028F8D0EC
:10BA40002068002108F00EFCA769206808F040FC7F
:10BA50003870A069411CE08BA161401EE08380B278
:10BA6000D8B96870206808F028FC012030704FF4C5
:10BA70008471206808F058FC20684FF4857108F044
:10BA800053FC206840F2091108F04EFC0020707051
:10BA9000A06A10B1BDE8F2400047F1BD38B50446D8
:10BAA000444D2068294608F04FFC00B32068294621
:10BAB00008F070FC206808F000FC012084F82000E9
:10BAC00084F821004FF48471206808F02DFC206870
:10BAD0004FF4857108F028FC206840F2091108F045
:10BAE00023FCA06A00284FD0BDE832400047324D09
:10BAF0002068294608F028FC18B12068294608F07B
:10BB000049FC2E4D2068294608F01EFC18B120681B
:10BB1000294608F03FFC2A4D2068294608F014FC0D
:10BB200018B12068294608F035FC264D20682946C2
:10BB300008F00AFC18B12068294608F02BFC224DB9
:10BB40002068294608F000FC18B12068294608F052
:10BB500021FC1E4D2068294608F0F6FB18B120682C
:10BB6000294608F017FC20684FF4847108F0DCFBCC
:10BB700020684FF4857108F0D7FB2068BDE8344099
:10BB800040F2091108F0D0BB31BD0000887E0020D2
:10BB90000054004000580040000C014020A1070064
:10BBA000317D002009010005090101050901070592
:10BBB0000901060508010A0508010F0508010E051F
:10BBC00008010B05080109050801080508010C0515
:10BBD0004DF2FF718208014002F4006280001143BF
:10BBE00000F400500843704762F30F2262F31F42D3
:10BBF00000B500BF130096469446103928BFA0E850
:10BC00000C50FAD85FEA417C28BF0CC048BF40F80E
:10BC1000042BC90728BF20F8022B48BF00F8012BCE
:10BC200000BD000062F30F2262F31F42401810F0C3
:10BC3000030308D0C91A1FD3DB0748BF00F8012D42
:10BC400028BF20F8022D130030B4144615461039D1
:10BC500028BF20E93C00FAD8490728BF20E90C009A
:10BC600048BF40F8042D890028BF20F8022D48BFA6
:10BC700000F8012D30BC7047C91818BF00F8012D1D
:10BC8000CB0728BF00F8012D70470000F8B5054626
:10BC9000032D0F4602D34FF0FF30F2BD694E002056
:10BCA000705506F11004C5EBC501605506EBC500E3
:10BCB00002624362644800EB810422691368E06811
:10BCC00003431360607E01F057FC6168B0FBF7F03E
:10BCD00001F12802401E1060002341F8043B0B6074
:10BCE00001236068A16800F12C0200F114071160C3
:10BCF0003B60002140F8101F20683554606994F9BA
:10BD000018100B460001002B06D5504D01F00F0214
:10BD10002A4402F8040C01E04D4DE854012001F0E2
:10BD20001F014C4A00FA01F15B0942F823106068D8
:10BD3000016841F0010101600020F2BD042902DB2D
:10BD40004FF0FF307047404BC0EBC00C03EB8C0052
:10BD50004368806803F1340C02404CF82120022231
:10BD600053F80C0F02FA01F10143196000207047EB
:10BD70003549344BC0EBC00201EB820218445168D4
:10BD800051F80C2F42F001020A600121017400BF3A
:10BD900070472D49C0EBC00201EB8200436853F8A5
:10BDA000240F70472849C0EBC00201EB82004068B5
:10BDB000016849084900016070472DE9F84F2249A0
:10BDC000C0EBC00201EB8202D2F804B00BF12C01EF
:10BDD0000BF11002D1F8008014680BF10C052968F2
:10BDE0000C4018490B1801EBC006187C48B11368C9
:10BDF0005B085B001360706A326ABDE8F84F00218F
:10BE00001047106000270BF1340A4FF0020913E0CD
:10BE100009FA07F004420CD0C043DAF800100440DD
:10BE2000884506D32A68104028603946706A326A0D
:10BE300090477F1C0AF1040A002CE9D1BDE8F18F7C
:10BE400000000000487B002068A8010818ED00E011
:10BE500000E400E000E100E00022FFF7E7BE034657
:10BE600000E05B1C1A78002AFBD111F801CB83F8A3
:10BE700000C013F8012B002AF7D1704704E010F836
:10BE8000013B6BB1491C521E52B10B7890F800C0B7
:10BE90009C45F4D002D24FF0FF307047012070472C
:10BEA0000020704715494CF6CC400860704730B40C
:10BEB0000446124D124A45F2555028601346E86870
:10BEC0005B1E00F0010002D00028F8D100E090B91C
:10BED0006960E868521E00F002000AD00028F8D11C
:10BEE000C4F30B04AC604AF6AA202860012030BCE1
:10BEF00070470028F4D030BC00207047003000406C
:10BF0000FFFF0F00DFF87C080021017041704EF642
:10BF100060220FF24101DFF87008F9F7F2BA38B584
:10BF20000C46DFF868581946049B28626A6220466E
:10BF30001A4608F0B2FA0FF2D960FCF7E2FDBDE84C
:10BF400038400FF2A9620FF295710FF2C55008F058
:10BF500093BD00002DE9F841DFF8345805F14D0894
:10BF600044F6206098F80010A864162983B000F207
:10BF70008E82DFE811F017002A0092009B00A100DA
:10BF8000A800CA00E10059024F00D8004A028C0202
:10BF900064026C0279028C028002B100B600BB0020
:10BFA000C000C500DFF8EC07DFF8E037026842F0B8
:10BFB000040202604CF25030A8640021012088F88D
:10BFC000011088F80000197067E20F21012008F0C5
:10BFD00062FE9624012001F04FFC012008F070FE63
:10BFE000C00601D5641EF5D10FF2C87191E81C009E
:10BFF000684680E81C00FCF7DDF88DF8070068460D
:10C0000008F07AFEDFF89007A864012188F8011093
:10C01000092000E2DFF874470021E16108F001FF28
:10C02000092088F8010005F14C0008F0E4FE18B979
:10C03000022088F8000013E0DFF86067304603F064
:10C0400016F94CF25030A864304603F00BF9DFF8D3
:10C050004407016841F480210160002288F8002033
:10C06000608B78B908F03CFF60B900F07BFB0120E1
:10C0700088F80000DFF82467304603F0F8F830460F
:10C0800003F0F0F8608B401C608380B2B0F5967FBF
:10C09000C0F2038200206083FFE1DFF8E40608F0CD
:10C0A000DCFF284608F03EFF0220EAE12946002096
:10C0B00008F062FF0620AEE1DFF8C416284608F05B
:10C0C000D9FF0420DDE1DFF8B81601F12802284687
:10C0D00009F014F80520D4E1284609F0BDF8122033
:10C0E000CFE1284609F0D1F81320CAE1284609F02B
:10C0F000DFF81420C5E1284609F0DFF81520C0E17B
:10C10000284609F0EFF81620BBE1284608F067FF43
:10C1100041F28831A96408B907207CE1012800F0C8
:10C12000BC810A2077E108F0ACFC042840F0B5811E
:10C130000A2088F8010065E1DFF8447607F124065B
:10C140000020B0724021284608F06FFF98F80100E7
:10C15000022806D1B5F84000102857D008F033FD6A
:10C1600050E1042807D13A46294607F1280008F093
:10C17000A2FF05204FE1052858D10020B87207F131
:10C1800028023946284608F0E1FF00283CD1FCF798
:10C190001EF878B93078C1070CD43A7ED10709D49B
:10C1A000C0F3400030B90B2088F80000002000F0F8
:10C1B00071FA07E0F07A98B9DFF8D015087800BB7B
:10C1C0000C6A14B90120F07267E10B2000904FF067
:10C1D000FF32002303213846A0470127F7725CE1B4
:10C1E0003078C10748BF082000F11581397ECA07A1
:10C1F00048BF082000F10F81C0F3400008B10820BB
:10C2000009E10121F17248E1032801D1042002E192
:10C210003078C10707D43A7ED10704D4C0F3400078
:10C22000002800F0EF8008F0E3FCEBE008280CD1D8
:10C2300008F046FD0224000758BF0124204600F004
:10C2400067F9002840F02981DCE00D2818D130780A
:10C25000C0F3400050B3284608F0C3F9012808BFD6
:10C260000D2000F0D880032808BF0F2000F0D380F5
:10C27000022801D10E20CEE00428FBD0002084E06B
:10C280000E286CD1DFF80405417E491E8941C90F93
:10C290004176EFD0284609F0CFF800283078C0F377
:10C2A00040003CD000284DD00F20B4E03178C807C2
:10C2B00020D5284608F0F7F8012805D1B87D401CA4
:10C2C000B87508F046FB03E00228D3D008F06EFAF8
:10C2D000002840F0E28008F096FA387E40F0010035
:10C2E0003876FBF774FF002840F0D780002000F07C
:10C2F0000FF987E0284605F0EFF9DFF8904418B110
:10C3000000220021022002E0002200210120FCF78F
:10C31000FCFB0020F072207000F0C8F9BDE000289E
:10C3200070D108F043FA002840F0B78008F06BFAAB
:10C33000387E40F001003876FBF749FF002840F0D6
:10C34000AC80D3E73078C107EBD5284608F03BFA3C
:10C350000128E6D108F046FA08F0FBFAE3E70F28D7
:10C360000BD1DFF82804017E491E8941C90F0176EF
:10C3700018BF11204FD10F2186E0112808D128467F
:10C3800009F05AF8112188F8011008F04AFA39E04A
:10C39000122808BF13203ED0132804D1284609F0E4
:10C3A00057F8142037E01428DFF8E04312D128466C
:10C3B00009F0ACF850B9002200210820FCF7A5FBD9
:10C3C000162088F800000021217066E009F0DAF8F4
:10C3D000152020E0152812D1162088F80000E81C4E
:10C3E00005F07AF918B100220021042002E00022B1
:10C3F00000210920FCF789FB002020704DE000217E
:10C40000F172217000F052F947E0DFF88003C16952
:10C41000FA2903D1002088F800003EE04FF4FA62C8
:10C42000AA64491CC16138E0DFF8540300F1280216
:10C4300000F10B01284608F0D8FE082021E0DFF8C3
:10C440004003817C284608F05FFF0D2019E0DFF8EB
:10C45000300390F82410036AC1F34002817C28461F
:10C4600008F067FF0E200CE0C548817C284608F0E4
:10C47000A3FF0F2005E0C248817C284608F0CAFFD0
:10C48000112088F80100032188F8001005E0092038
:10C490004CF2503288F80000AA64AA6CC049BA482D
:10C4A000F9F72FF804B0BDE8F08110B5BD4C68B1C4
:10C4B0002280012008F018F980B908F0A4F9218839
:10C4C000062007F0E6FFBDE81040EFE0207C61F3B6
:10C4D00041002074C0F340000028F4D0AC49022091
:10C4E00081F84D0010BDAA48A84A90F84C1051712F
:10C4F00038E180B508F012FDA54981F84C0002BD75
:10C500009F49002081F82F000022A0480270704748
:10C51000F8B59C4C9A4E06F124050021A1702A78AA
:10C52000317ED30701D4CF0726D5CA071DD40128F1
:10C5300018D1002000900023717C0022832007F096
:10C54000A0FF08F033F900284ED108F05CF9307EE6
:10C5500040F001003076FBF73AFE002844D1FFF7A7
:10C56000D7FF28E00D2020703EE001F0FE0131767B
:10C57000B18A07F08EFF1EE0C2F3400181B196F947
:10C580001110012808D10020009000230022C9B218
:10C59000832007F076FF0EE08900C91CB17421E00A
:10C5A00001280AD10022FCF7B0FA0020774AE8728D
:10C5B000107000F07BF80020F2BD05F082F8007DDD
:10C5C00020B105F07EF8007DFF280BD1002200216C
:10C5D0000220FCF79AFA00206C4AE872107000F012
:10C5E00065F801E00D2020700120F2BD6549674A21
:10C5F0000F204870107E18B9112301200B7004E041
:10C600004FF00F0C002081F800C01076704700003A
:10C6100010B55E4C0120207005F053F8407D60702D
:10C6200001280FD0032808D00B2810D15E480178CC
:10C6300041F002010170022005E0002008F004FF33
:10C64000122000E00820524981F84D000AE0002243
:10C6500000210120FCF759FA53490020C8722070CC
:10C6600000F024F805F02DF8454C0078E07405F052
:10C6700028F890F91300607405F023F8407CA0744A
:10C6800005F01FF8411C04F10B00BDE81040062224
:10C69000F7F7F6BB1CB53D490C6A34B100904FF07A
:10C6A000FF32002303213648A04713BD10B534499B
:10C6B0003E4C91F82F0028B14FF4FA61162021600A
:10C6C000607110BD0021617108F0BBFB3148016849
:10C6D00041F4802101603648206010BD70B5284DBE
:10C6E000287E40F001002876FBF771FD08B101209B
:10C6F00070BD244C05F12406A0703178287ECA074D
:10C7000022D4C30720D4C1F3400028B195F9110009
:10C710008000C01CA87419E004F0D3FF007D38B17C
:10C7200004F0CFFF007DFF2802D00D21217017E01B
:10C73000002200210220FCF7E8F90020134AF072E1
:10C740001070FFF7B3FF0BE0C10702D40D2020707B
:10C7500006E000F0FE0028760020A98A07F099FE86
:10C76000002070BD10B5094C201D08F06EFB636AF7
:10C770002BB1211DBDE810401422FF20184710BD29
:10C7800094760020BD7A0020041D0020DC1C0020CF
:10C79000707A002010140140400D0300003C00405E
:10C7A00055BF0008A8760020B8760020B87A00208F
:10C7B000A08601008054E80360403D0003000000B3
:10C7C0001CB56846002101600422DFF8004304F133
:10C7D0002001FEF716FE94F8240004226946FEF7B5
:10C7E000A3F9DFF8EC12002008708D2284F82420D1
:10C7F00013BD80B501F0B8FEB5490120887001BDB8
:10C800007CB5B24CA01D08F09CFFE088000903F045
:10C81000EBFE4FF0665104F03BF9AE4904F038F9F5
:10C82000E0606078002860D0FBF7AEFE00283FD0C3
:10C83000FBF788FE0146E06800F00CFD38D220626C
:10C84000A34D6878C0B104F124068D200121307019
:10C850007170684600226A70026004F120010422AF
:10C86000FEF7CFFD307804226946FEF75DF900211E
:10C8700029708D2232701BE02878C8B9012104F19B
:10C88000240629707170FBF773FE60B10122924992
:10C890009248F7F72FFC01F05DFEE87818B98A217D
:10C8A00031700120E870281D8D4A8E49F8F729FE65
:10C8B000FBF76AFE40B1FBF745FEE16800F0CAFCF9
:10C8C00002D3FBF755FE80B9814DA87868B1864A3E
:10C8D000864905F11C00F8F714FE0020012104F13F
:10C8E0002402A87069705070E87073BD10B5FEF72F
:10C8F00090F8764C10B1FDF7BDF9F0B1A0880009B1
:10C9000003F072FE4FF0665104F0C2F8714904F072
:10C91000BFF8774904F0BCF8A16904F025F9617DFE
:10C92000A061491C6175C9B2322906D1714903F071
:10C9300069FEA060A061002060756088000903F0B6
:10C9400053FE4FF0665104F0A3F8624904F0A0F8DA
:10C95000694904F09DF84FF07C5104F005F9E16954
:10C9600004F002F9217DE061491C2175C9B2322928
:10C9700006D1604903F046FE2061E0610020207589
:10C9800010BD70B5010013D15C4C0121204603F0AD
:10C9900061F901282DD1204602F0C0FF58495948BD
:10C9A000FDF732FE2046BDE87040012103F060B97A
:10C9B00001281ED1544C55482668A568006880B2ED
:10C9C00008F0AEFEB10714D5AA0712D54D4D504E52
:10C9D00020B106F110012846FDF716FE3146284623
:10C9E000FDF712FE002001F00BFD606840F0020030
:10C9F000606070BD80B5FBF786FA20B9BDE80240E3
:10CA00003E4802F016BF01BD424B984202DBB0F532
:10CA1000006F01DB40F2FF703F4A52F8211000F234
:10CA2000FF7080B208473C4A52F82110084710B501
:10CA30003A4C4FF400612046FEF7C6FB002001F09F
:10CA400018F82046BDE810404FF40061FEF7C1BB66
:10CA50000128334A03D104211046FEF7BABB042152
:10CA60001046FEF7B8BB04212D48FEF7B8BB2D4891
:10CA700070471649487070471448806870471348DB
:10CA8000006970471148C0687047104890F8250049
:10CA900070470E4981F82400704780B501E080B5E9
:10CAA000002000F0E6FFBDE804404FF400611B48A1
:10CAB000FEF78FBB80B5002000F0DBFFBDE804402F
:10CAC0004FF400611548FEF786BB00006C7C002027
:10CAD0004C06002033335340C0CF6A0010AC01082D
:10CAE00080841E00C1C70008808D5B00F3C700086A
:10CAF0006ABC804000004842ABAA1A4100340140A1
:10CB00003C060020947E0020000002404C2801409A
:10CB10003406002001F8FFFF8006002000080140D5
:10CB2000000C01406E7C0020DFF898067047DFF8AB
:10CB30009806DFF898168268104710B500F02FF8B5
:10CB4000DFF88C46206D48B308F01CFE802104F508
:10CB50003E7008F0B0FEE26B1AB1E179DFF87406BE
:10CB60009047002000F067F8DFF86C260FF2F141E3
:10CB700004F1B000F8F7C5FCDFF860260FF2E551CC
:10CB800004F1C800F8F7BDFC04F1E000BDE8104076
:10CB9000DFF84C260FF2E551F8F7B3BC10BD10B525
:10CBA000FBF7FEFCA8BBDFF828464FF4007204F147
:10CBB000F80104F10C0008F0BDFEDFF82806DFF8EC
:10CBC000281620626162DFF82406DFF82416A062CE
:10CBD000E162DFF82006DFF8201620636163DFF8EA
:10CBE0001C06DFF81C16A063E163DFF81806DFF807
:10CBF000181620646164DFF81406DFF81416A064C8
:10CC0000E1640A200521E071A1710C20022160710C
:10CC10002171002000F05AFA012000F057FA02209A
:10CC200000F054FABDE8104003204FE2DFF8A025E1
:10CC30009065D165704770B5DFF89445A06C80476A
:10CC400040B9DFF89015B1F88400BDE87040C0B27B
:10CC500008F0B7BD207A002855D0616D626E01F1F1
:10CC600088008A4202BFB4F91C300278934202D194
:10CC70000021017604E0007E002818BF002911D1B0
:10CC8000216E00291CBFD1F8D800002801D1206DE9
:10CC900010B9D1F8D80000B12066206E606501217E
:10CCA00080F8A010606D606690F88810A18300F095
:10CCB0004DF9626D02F1A103D97849B918780028BD
:10CCC0001EBF1970216B002904D01046884701E06F
:10CCD0000020D870A16A69B1606D884750B1616A5F
:10CCE00009B1606D8847616DB1F88400C0B208F089
:10CCF00068FD30E0207A00283BD0012161720020DD
:10CD0000BDE87040AAE004F56276DFF8C85405F18A
:10CD100084033246002104F10C0008F066FEB5F8E9
:10CD200084003146C0B208F04CFD04F10C0008F05C
:10CD300091FE208A78B9012121720FF27D3000F036
:10CD40009CF9216D91F89E0000281CBFD1F8D810E5
:10CD50000029F7D16165FBF744FC4FF47A71484331
:10CD6000024604F16800BDE87040DFF8A814F8F747
:10CD7000C8BB70BD18B583B00421DFF89C0402F075
:10CD8000DBFFC8B108F031FDDFF84404446C9CB10E
:10CD900000F56071029100F55E720FF21D43019281
:10CDA000009300F581610FF20543DFF8282400F5B8
:10CDB0003E70A047022804D004B0BDE8104008F03F
:10CDC0001FBD04B010BDDFF80814096D91F89F2055
:10CDD000824204D0D1F8D8100029F7D1704711B1A0
:10CDE000012081F8A100704710B500F02CF9002453
:10CDF00000281EBFDFF8D813496B002901D08847EF
:10CE00000446204610BD10B508F027FD98B1DFF8A4
:10CE1000C043207A08B108F05FFD606D00F096F81D
:10CE2000FBF7EFFB024604F18000BDE810400FF273
:10CE30003D11F8F766BB10BD10B508F04DFDDFF8E9
:10CE4000844380212046FDF7FDFB2046BDE81040CD
:10CE5000802108F030BDDFF8C403704710B5DFF85B
:10CE60007043206DB0B30020FBF7DCFB21788142DA
:10CE700005D00020FBF7D6FB207001206072012056
:10CE8000FBF7D0FB6178814205D00120FBF7CAFB9C
:10CE90006070012060720220FBF7C4FBA178814220
:10CEA00005D00220FBF7BEFBA070012060720320BA
:10CEB000FBF7B8FBE178814205D00320FBF7B2FB1A
:10CEC000E070012060720FF2CD2000F0D6F8607A99
:10CED00010B910BD0121617208F05CFC04F168001A
:10CEE000F8F746FB04F18000F8F742FB04F19800E4
:10CEF000F8F73EFB04F1C800F8F73AFB04F1E00054
:10CF0000F8F736FB08F0E8FC08F0A7FCE16C00201D
:10CF100088470020207208F0F6FC606D00F016F8DB
:10CF2000AC4800F013F8002020656072882104F5F9
:10CF30008160FDF787FBBDE81040FEE5A449087A53
:10CF400018B101224A72002088E7704710B50446E4
:10CF50000022A4F884204021FDF774FB04F1400076
:10CF6000BDE810404021FDF76DBB000038B54FF41F
:10CF70008051AB48964C00F0DDF904F53E758021F8
:10CF80002846FDF75FFB8021284608F094FCE16A03
:10CF900091B1606D8847616D91F8A00060B9207A09
:10CFA00050B1FBF71EFB4FF47A7148430246994992
:10CFB00004F16800F8F7A5FABDE83240002008F057
:10CFC000A2BC70B5824DA86D84B028B3296D91F8CC
:10CFD000A20028B9D1F8D8100029F8D104B070BD4A
:10CFE0000C0019D004F19C06307801F0FDF931787D
:10CFF0000022CDE90222080003D0FF2202A8FEF79A
:10D00000F3FD00200090DDE9022304F18C00F178AB
:10D01000AC6DA0470020B07104B070BD6C48C36D0A
:10D0200083B1016D91F8A30020B9D1F8D81000297F
:10D03000F8D1704731B1002081F8A30001229E3160
:10D040008B201847704701466148006D90F89E207C
:10D050008A421CBFD0F8D8000028F7D170470000E2
:10D0600010B55B4CE16C0120884704F18000F8F7B3
:10D070007FFABDE810400020DDE510B50446002031
:10D08000FBF79AFA01005CBFC0B2A0470120FBF792
:10D0900093FA01005CBFC0B2A0470220FBF78CFAF4
:10D0A00001005CBFC0B2A0470320FBF785FA010076
:10D0B0005CBFC0B2A04710BD80B5FFF7C4FF444AB3
:10D0C0001179126ABDE8084010470000D0B5064645
:10D0D000FBF7A8FA78B353485DA2C6EBC60100EB94
:10D0E000411404F19E0004F1D0070670935D437073
:10D0F0003046FBF7A8FA38703046FBF7B5FA78707F
:10D1000001210020324BF870B9709955196D19B989
:10D11000B8601C6507E00146D1F8D8000028FAD1B4
:10D12000B860C1F8D8409A6B2AB12046BDE8D0401B
:10D1300003F10C011047D0BD80B5FFF784FF2449EF
:10D140000A6A1AB1BDE808408979104701BD80B567
:10D15000FFF779FF1E490A6A1AB1BDE8084049790C
:10D16000104701BD80B53048FFF787FFBDE8084094
:10D170001A4A2E492E48F8F7C4B9000080B52D4848
:10D18000FFF77BFFBDE808402B4A2C492C48F8F7F5
:10D19000B8B9000080B5FFF756FF0D490A6C1AB107
:10D1A000BDE808400931104701BD000041F2883256
:10D1B00018492448F8F7A5B94CF2503222492348BF
:10D1C000F8F79FB9F80200209806002024080020F4
:10D1D00000000020C8760020404B4C00002D31019B
:10D1E00080C3C901F97E01084D800108FB7E01085A
:10D1F0002D8101082182010871830108238401081F
:10D200000D850108418501087F85010879850108A0
:10D210007385010837CC0008004C0040080400204A
:10D2200000100140A86D002039D1000865D1000828
:10D23000C80000204FD1000840787D017DD1000852
:10D24000E0000020680000206DCF00088000002072
:10D25000616263644FF0807C1CEB400F94BF1CEB59
:10D26000410F05E040EA010C1CEB0C0F01D2884293
:10D27000704718BF814270472DE9F04304460846C5
:10D280001546194600F00F02C30648BF2A43002680
:10D29000B44604F1100504F114084FF00F0921FA07
:10D2A00006F3DB0716D5276809FA0CF327EA030310
:10D2B00002FA0CF73B43282805D10127B7400F405D
:10D2C000C8F8007005E0482803D10127B7400F4097
:10D2D0002F602360761C082E0CF1040CDFD308238A
:10D2E0004FF0000C241D21FA03F6F60718D5266826
:10D2F00009FA0CF726EA070702FA0CF6282846EA8C
:10D30000070E05D101279F400F40C8F8007005E0C7
:10D31000482803D101269E400E402E60C4F800E04C
:10D320005B1C102B0CF1040CDDD3BDE8F08340F83E
:10D33000101F704740F8141F7047083000E00C3091
:10D3400000680140481E8041C043C00F7047F0B4E0
:10D350002B4A00284CBF9369136800F44016B6F5B9
:10D36000401FC0F3034485B206D1146824F07064F2
:10D3700023F0706314600DE0C60204D5032707FA9A
:10D3800004F4A34304E0440D260105FA06F6B34372
:10D3900043F0706319B1440D21018D402B430028E7
:10D3A0004CBF93611360F0BC70478A0002F00C021E
:10D3B0000F239340DB4390400429124A06DA116898
:10D3C0000B4013601368184310607047082906DA91
:10D3D00051680B40536053681843506070470C29E4
:10D3E00006DA91680B409360936818439060704729
:10D3F000D1680B40D360D3681843D06070470000F9
:10D4000004000140080001401CB58DF800008DF8B3
:10D4100001100223384CA0686A468821FEF72AF9D9
:10D4200013BDE0B5F9F788FE28B96846FBF76FF839
:10D43000684600F051F803B000BD1CB52E4C2078B2
:10D44000810702D508F05EFB01E008F061FC606036
:10D45000606800281CBF0068002806D06846FBF7FB
:10D4600056F861680A686846904713BD3EB50446A1
:10D470002348214D826805F10C0190471F48019017
:10D4800001210091AC602B46132288212046FEF733
:10D490008FF903B0BDE830401748406818B14068C4
:10D4A000002818BF004770471348406818B18068CB
:10D4B000002818BF004770470F4A52681AB1D26857
:10D4C000002A18BF104770470B4A52681AB11269F8
:10D4D000002A18BF104770470749496819B14969C0
:10D4E000002918BF084770470349496819B189697D
:10D4F000002918BF08477047880600203BD4000861
:10D5000098060020FFE7DFF8281101EB90110123B6
:10D510000A6800F01F0003FA00F01043086070472B
:10D52000DFF80C1101EB901101230A6800F01F00D5
:10D5300003FA00F022EA000008607047E3E7EFE733
:10D540003C490A6822F4E062E7E73A4A3A4913683C
:10D550000B40032804D9411F05D0891E03D008E0E1
:10D5600043EA803305E0354901EA803141F08051DA
:10D570000B431360704700002DE9F00332A393E8DA
:10D58000F00088B004AA00BF33A382E8F000D3E91A
:10D59000008900BF32A302AAD3E90045C2E900898D
:10D5A000CDE90045234A13680021C3F38103022B10
:10D5B00015D11368DB0303D51468214BA40300D5F0
:10D5C000204B14681568C4F383442E0148BF44F00F
:10D5D00010040F2C34BFA41C641C634300E0184BE0
:10D5E000146804ADC4F3031402AE2D5D23FA05F4F0
:10D5F0001568C5F302250328765D1268C2F3C222BE
:10D6000024FA06F51DF8026024FA06F20AD8DFE8CB
:10D6100000F002040608194604E0214602E029460B
:10D6200000E0114608B0BDE8F0030846704700006E
:10D630000010024004100240FF3FFFEF00C0FEFF59
:10D6400000127A0000093D00000000000000000008
:10D650000102030406070809000000000102030498
:10D660000000000001020304014645480268D0089A
:10D67000520B02F0010209B982F0010202F001022C
:10D6800000F001001043704710B53E4C4FF480434A
:10D69000032210212046FFF7EFFD2046BDE8104091
:10D6A0004FF48041FFF743BE80B54FF4004303229F
:10D6B00048213448FFF7E0FD0F210220FFF775FEF7
:10D6C000022200214FF40040FDF7EAFD2E492F4BC6
:10D6D00011E080B50423032248212A48FFF7CCFD3E
:10D6E00002210220FFF761FE022200210420FDF743
:10D6F000D7FD2749274B002008704FF480721A602D
:10D7000001BD25490128486909D1020413D548699A
:10D7100040F4004048610A6822F4004208E04207F1
:10D7200009D5486940F0040048610A6822F0040203
:10D730000A600120704700207047184909680128D5
:10D740000CBF01F4004101F0040109B90120704748
:10D750000128114904D1086840F40040086003E042
:10D760000A6842F004020A60002070470C49012850
:10D7700007BF4FF40050086008220A60F9F706BDA1
:10D780000C1001400010014028E400E004E100E03A
:10D7900008E400E000E100E000040140081001405E
:10D7A000141001401CB54FF480711B481B4CFDF751
:10D7B00014FDD0B16178207878B114290DD31848C0
:10D7C000F6F74CFCFF208DF80000012269467F200F
:10D7D000FDF7AAF90020208013BD491C6170201DAF
:10D7E000104A1149F7F78DFE13BD607013BD00009C
:10D7F000E0B584B00EA168461822F6F751FB0FBCC5
:10D80000FDF70FFD03B000BD064A07490748F7F7CB
:10D8100078BE02490870704700080140FC7C002077
:10D8200028AC010840420F00A5D70008007D002069
:10D830000008014000010000000000000800000096
:10D840000001000000170000124801684FF47A72CE
:10D85000B1FBF2F0401EB0F1807F0CD20E4948605F
:10D86000F0220E48027000238B604FF0070CC1F8C5
:10D8700000C003707047FEE7094908600868002887
:10D88000FCD170470649086810B10A68521E0A6048
:10D8900070470000701F002010E000E023ED00E062
:10D8A000A47E002010B5224C01212046FDF78CFCFF
:10D8B00001212046FDF78FFC1E4C40212046FDF73C
:10D8C00083FC40212046FDF786FC08212046FDF719
:10D8D0007BFC2046BDE810400821FDF77ABC000023
:10D8E00038B5154908700124401E04280BD8DFE81C
:10D8F00000F0030905090700002404E0042402E005
:10D90000052400E002240B4D04F001020821284602
:10D91000FDF754FCC4F3400240212846FDF74EFCBD
:10D92000A208BDE8384001210148FDF747BC0000CE
:10D93000000C014000080140BC7E002010B5364CB0
:10D940004FF40073032218212046FFF795FC4FF493
:10D950008063032204212046FFF78EFC2F4C4FF4F6
:10D96000E131204602F088F90021204602F0B0F9AA
:10D970000021204602F0B1F90021204602F0B6F95C
:10D980008021204602F0D3F94021204602F0CAF956
:10D990000421204602F0BAF90821204602F0B1F92C
:10D9A000204602F0A8F91E491E4B002008702022D4
:10D9B0001A6010BD10B5194C0521204602F0BCF9C3
:10D9C00018B10521204602F0C4F90221204602F0D8
:10D9D000B3F918B10221204602F0BBF9012120461B
:10D9E00002F0AAF918B10121204602F0B2F9002193
:10D9F000204602F0A1F918B10021204602F0A9F951
:10DA00000321204602F098F928B12046BDE81040D5
:10DA1000032102F09EB910BD00080140003801400A
:10DA200025E400E004E100E080B508F083FA00207E
:10DA300008F09FFA0021002008F0ACFA002008F05E
:10DA40008CFA002008F081FA012008F092FA0021F7
:10DA5000012008F09FFA012008F07FFA012008F069
:10DA600074FA1C480021C160016001BD19490860B9
:10DA70007047194908607047F8B50C4616464FF0D4
:10DA800089470BB14FF08A4702F0AEFD214602F004
:10DA9000FFFFFCF7F1FF114A114B04F023FB044692
:10DAA0000D463046FCF7E8FF02460B462046294665
:10DAB00004F038FD08F08AFA08F0BCFA4FF07E5105
:10DAC00003F052F8394602F0E3FF03F0D3F880B2D6
:10DAD000F2BD000008740040147400405C3FBB4B72
:10DAE000FB211940DFF86816087A08B901220A728A
:10DAF000704710B50446DFF8580600F582514FF420
:10DB00000072243007F016FF200018BFA047BDE8C0
:10DB1000104000202DE9F84F84B001F045FD41F69A
:10DB20000F08A8EB00001FFA80FBDFF8286641F21F
:10DB30001000371838888345AEBFABEB000008EB08
:10DB40000B01081A80B2002800F053814FF0000A40
:10DB500040F34D8141F2010103918146DFF8F04528
:10DB60003888DFF8F4351FFA8AF10818424690FB2E
:10DB7000F2F208FB120080B2195C307840B9002242
:10DB8000AA297A80B880FA8040F02A81012030707A
:10DB9000321D78881154401C31787880012912D1C7
:10DBA000B988491CB980F988491CF98089B20229D1
:10DBB00040F0168180B23044C078552825D100212C
:10DBC000F98002203BE0022921D1F988BA88491C5A
:10DBD000F980521C89B20229BA8040F0018180B2DA
:10DBE000304440886080C108039A91420DDA00F009
:10DBF00007000021072818BF0328F98003D0062852
:10DC000003D103201BE0042138E0002017E00329A2
:10DC100017D1F988BA88491CF980521C89B20129A8
:10DC2000BA8040F0DD8080B200213044F980C378B2
:10DC300023716088C008801C8218BA80052030706B
:10DC4000CEE004291CD1F988BA88491CF980521CFD
:10DC500089B20429BA8040F0C380002180B2F980E3
:10DC600030586060608800F00701072904BF02EBAC
:10DC7000D002BA80B888801CB88005213170AFE02E
:10DC8000052902BFB98880B2884240F0A9800020EF
:10DC90003070A17801F0070103295ED0062902D077
:10DCA00007290FD09CE006F1090000F0C2F8002817
:10DCB00000F0968062882079D20806F1090108F008
:10DCC00009FA8DE006F10C0000F0B3F8002800F02E
:10DCD0008780606865880090ED08F8F76EFAC0B13B
:10DCE000052101A8FCF7AEFC0098206104226946DA
:10DCF00001A8FDF786FB08208DF80800207A00288F
:10DD00006ED0052301AAFE2104F1240007F01AFEBB
:10DD100061E00098206106F10C016161A5812A464D
:10DD2000009906F10C0000F032FA052101A8FCF779
:10DD300089FC042204F1100101A8FDF762FB002018
:10DD40008DF80800207A00284AD0052301AAFE2178
:10DD500004F1240007F0F6FD3DE006F10C0000F0B0
:10DD600068F800283CD0606865880090ED08F8F7F6
:10DD700024FAB8B1052101A8FCF764FC0098E06121
:10DD80000422694601A8FDF73CFB08208DF8080035
:10DD9000207A28B3052301AAFD2104F1240007F00D
:10DDA000D1FD18E00098DFF8B413884218D2E06182
:10DDB000258306F10C0121622A46009906F10C0028
:10DDC00000F003FA207A58B100230022FD2104F16B
:10DDD000240007F0B7FD18B9607A08B100F0BEF86A
:10DDE0000AF1010A1FFA8AF04845FFF6B9AEA7F812
:10DDF00000B0DB4941F2180042F210723044F7F7EC
:10DE000080FB05B0BDE8F08FFFF7D4BD01F0DCBBAF
:10DE100080B501F0B6FBCE4801214172243007F0F5
:10DE200019FEBDE8014099E0CB48704741F60F006C
:10DE3000704738B50446C6484188CD0841F2010311
:10DE40009D421EDA01F00701032904D0062916D0ED
:10DE5000072901D015E000250622811C43F28470B9
:10DE600008F008FA2A46214608F004FA6219615DB2
:10DE7000537841EA0321884203D1012032BD0322B5
:10DE8000EBE7002032BD10B5B14C1346227A5AB1EF
:10DE90000A46014604F1240007F054FD20B9607AD7
:10DEA00010B1BDE8104059E010BDFEB5A84D0746C1
:10DEB000287A00280E4614464ED000F036F943F278
:10DEC000847145F2AA5200206872ADF80010ADF8D6
:10DED0000420E10041F00601ADF806108DF8027053
:10DEE000042201A905F13400FDF78BFA01220DF19E
:10DEF000020105F13800FDF784FABDF800000322A5
:10DF000005F1360108F0B6F9ADF8000022463146B9
:10DF100005F13900FDF775FABDF80000224605F15C
:10DF2000390108F0A7F9ADF80000641D05F13400CF
:10DF3000A3B2022269461844FDF763FA01F000FB20
:10DF400001F011FBA41CA1B205F1340001F009FBA2
:10DF500001F005FB00F0E9F803B0F0BD78B57C4CAA
:10DF600083B004F1240007F09CFD002840F0DB8022
:10DF700004F5925602AB32460DF1030104F1240080
:10DF800007F033FD002840F0CE80607243F28472C7
:10DF90009DF803109DF80600BDF808508DF802109A
:10DFA00000F0070045F2AA51ADF8041040EAC500A0
:10DFB0009DF80210ADF80020FE29ADF806002AD128
:10DFC00040F00700ADF80600042201A904F1340076
:10DFD000FDF717FA042204F1100104F13800FDF7EF
:10DFE00010FABDF80000062204F1360108F042F9EB
:10DFF000ADF800002A46314604F13C00FDF701FA75
:10E00000BDF800002A4604F13C0108F033F9ADF8F0
:10E010000000083573E0FD2946D1032161F30200B9
:10E02000ADF8060001A9280008BF208BC00040F011
:10E030000300ADF80600042204F13400FDF7E1F915
:10E04000042204F11C0104F13800FDF7DAF9BDF8EF
:10E050000000062204F1360108F00CF9ADF80000CA
:10E06000280010D1228B216A04F13C00FDF7C9F988
:10E07000228BBDF8000004F13C0108F0FBF8258B71
:10E08000ADF800000EE02A46314604F13C00FDF7F1
:10E09000B8F9BDF800002A4604F13C0108F0EAF89E
:10E0A000ADF8000008352AE0062161F30200ADF862
:10E0B0000600042201A904F13400FDF7A2F90122AF
:10E0C0000DF1020104F13800FDF79BF9BDF80000E5
:10E0D000032204F1360108F0CDF8ADF800002A461D
:10E0E000314604F13900FDF78CF9BDF800002A46ED
:10E0F00004F1390108F0BEF8ADF800006D1D04F11F
:10E100003400ABB2022269461844FDF77AF901F0F7
:10E1100017FA01F028FAAD1CA9B204F1340001F09D
:10E1200020FA01F01CFA04B070BD38B50D4C084D52
:10E130000AE002220321204601F01EFB012803D140
:10E1400001F01FFA01206872687A0028F1D031BD11
:10E15000D4080020A838002098200020FFFF1F00CE
:10E1600015DB00080000024080B52A482A4B2B4AE4
:10E170002B490090002008F0A7F82A4808F0AEF8D4
:10E1800008F0D2F805F0FAFC03F04EFA3AE010B5C8
:10E190000C4625498C4208D3244B1B19B3F5A72FF5
:10E1A00003D22146BDE8104013E0214608F099F85B
:10E1B000A4F56C2441F20100844203D2BDE8104072
:10E1C00005F0DCBC10BD08F09EB808F090B808F06F
:10E1D00094B870B504460D461646284608F0AAF8CD
:10E1E00005F5006008F0A6F8B2B229462046BDE861
:10E1F000704008F0BBB808F08CB80D48704780B587
:10E2000008F06FF8BDE808404FF48052FF2108483D
:10E21000FDF70BB9CF9F0108A19E0108E19E0108FF
:10E22000599F0108179F01080160120000F8FDF7CF
:10E23000D85800200FF20500F5F7E2BE00BF11B577
:10E24000244C81B0162200212046FDF7EEF8012073
:10E25000F9F7D2F9042201A92046FDF7D2F8FAF71E
:10E2600094FA0199814205D101202076002000F026
:10E2700007F813BD0FF20901204608F0A9F813BDF5
:10E280007CB507216846FCF7DDF9124E04223146C1
:10E290006846FDF7B6F8308A0F4DADF804006B24E0
:10E2A0003079072804D0FAF799FA18B9307E40B1CE
:10E2B0000A4D6C24307E20B1012100208DF806101B
:10E2C00030760820F9F798F9072269462046A847D2
:10E2D00073BD0000187D0020F773000871740008FA
:10E2E0004349086170472DE9F84F414E7769182F6F
:10E2F00049D34FF0FF300146C7F1410208F0CAF898
:10E30000D6E9008904460D4608EA040009EA050139
:10E31000C6E90001D6E900ABBBF1000F08BFBAF1B6
:10E32000000F30D0282F18BF402F14D0012000211B
:10E330007A1E08F0BFF8D6E90023C043C943024063
:10E340000B405B084FEA3202C6E9002304400D404F
:10E350006D084FEA3404D6E90001D6E9008920F0BF
:10E36000FF3231F00003009212BF0720042025F095
:10E37000FF35C6E90289B061224634692B46042183
:10E3800006F10800A04700207061C6E90000C6E958
:10E390000200BDE8F18F1648D0E900235B0043EA94
:10E3A000D2735200C0E900234169491C416142F225
:10E3B000107211E018B40E48D0E900235B0043EA64
:10E3C000D273520042F00104C0E900434169491C84
:10E3D000416142F2107218BC06491C30F7F791B83F
:10E3E00003488069C0B270470149886170470000E6
:10E3F000807B0020E7E20008734AC2E90001704711
:10E400007CB501F0C1FC6846FCF76CF96F4D044621
:10E4100028780026092803D1FCF7A2FA002876D034
:10E42000F8F733FC20B9FBF70DFC08B1FBF79DF8BA
:10E43000287801281CBF032806280DD1FBF702FC11
:10E4400010B1F8F722FC38B92878092837D0072806
:10E450002AD068702E7032E02978012906D003296D
:10E4600011D0062919D007291ED028E0FCF73FFA61
:10E470000246002356495748FCF76BF969680022A9
:10E48000FCF718F90646A868FCF7FCF8FCF7E1F879
:10E49000FCF7BFFA03F04DFA11E0FCF728FA024648
:10E4A00000234B494B4803E0002302224A494B48D2
:10E4B000FCF74FF969680022FCF7FCF806469DF866
:10E4C000000028B169680022A0B2FCF7F3F8064604
:10E4D000287809281CBF3046FCF7B8F8FCF740FA4A
:10E4E000012814D1FBF7C6FB88B93D493D48FCF72C
:10E4F00023F902F0D5FBA96802F0CAFA02F0BAFBD0
:10E5000000B2FCF7A6F8FCF784FA03F012FA73BD28
:10E510002E490A78092A02D10A2806D07047072A0C
:10E5200003D1092802D0082801D14A700870704729
:10E5300080B502F059F82C4902F064F8234948608C
:10E5400001BD80B502F050F8274902F05BF81F4981
:10E55000886001BD1D480178092918BF072902D02C
:10E56000417007210170704718480178072903D1CD
:10E570000722082142700170704780B51849194878
:10E58000FCF7E1F80020FCF7E8F91048C06810B18A
:10E59000BDE80240004701BD80B50120FCF7DDF970
:10E5A000BDE80840114A12491248F6F7AABF124ABC
:10E5B0000FF209011148F6F7A4BF000003480069F3
:10E5C000002818BF00477047681F00205C1F00200C
:10E5D000CCA30108387E002084AB0108487E0020CF
:10E5E00044AA0008A81E002000007F4360E3160034
:10E5F0007BE50008C47D0020E0930400DC7D002062
:10E600002DE9F8431400814688461D4627D0089E10
:10E61000DFF8A07B6C20464345434146484607F05F
:10E620005AFF78687A68904204D23B681B185B1CDA
:10E630009A1A00E0821AAA42F4D34146484607F0EB
:10E640004CFF78687A68904204D23B681B185B1CC8
:10E650009A1A00E0821AB242F4D3641EDDD1BDE8FA
:10E66000F18300002DE9F04786B0684602F050FBC8
:10E670009DF811409DF812509DF813609DF8109080
:10E68000DFF834ABDFF8348B002727E0284602E0C0
:10E69000304600E02046FF2813D0032F11D8DFE8D2
:10E6A00007F002060A0C4FF40071504607E04FF4E1
:10E6B0008071504603E0012100E00221404607F04E
:10E6C0000AFF7F1C042F0BDA032FFAD8DFE807F0CC
:10E6D00006050403F5E7DBE7D8E7DBE74846DAE7BA
:10E6E00006B0BDE8F08738B5DFF8D44ADFF8D45A71
:10E6F000FF2084F8300084F8640084F8980084F8DF
:10E70000CC0004F1D401AA6828469047AA6804F115
:10E71000D80128469047002000F004F8BDE83240B8
:10E72000002063E02DE9F84D89B003A802F0F0FA6B
:10E730009DF81F10DFF8884A0FF21D12DFF8787A73
:10E74000DFF8788A8DF800100025264602924FF4F3
:10E75000007A4FF4807B9DF81C0010E0032D04D854
:10E76000DFE805F00205080BF5E7FF2007E09DF85C
:10E770001D0004E09DF81E0001E09DF8000096F8E1
:10E780003020904229D0FF2886F8300021D0032D78
:10E7900018D8DFE805F002060A0F2761C4F814A0B4
:10E7A00010E06764C4F848B00CE00121C4F8788038
:10E7B000E16707E004F1AC020192C2F80080022296
:10E7C000019B5A60002131707160B16060B902989C
:10E7D000F060F16809B1002088476D1C3436042DC3
:10E7E000BCDB0AB0BDE8F08DF160F6E780B586B01D
:10E7F000F9F744FC58BB684602F08AFA9DF810000D
:10E80000FF2804BF9DF81100FF2807D19DF81200D2
:10E81000FF2804BF9DF81300FF2801D0282011E035
:10E820009DF8040008281CBF9DF80D00082807D09B
:10E830009DF80E0008281CBF9DF80F00082806D17F
:10E8400040F6FF7007B05DF804EBFEF726B907B09D
:10E850005DF804EBFEF723B92DE9F84F86B03424B8
:10E86000DFF85C5904E02820FEF717F90121317028
:10E8700095F8D00060432E183178062900F2838085
:10E88000DFE801F005161D04626C7700EBE7282035
:10E89000FEF703F901203070DFF82C29DFF82C197E
:10E8A00006F1180007B0BDE8F04FF6F72ABE6DE09C
:10E8B000FFF7D8FE02203070DFF81429EEE7684633
:10E8C00002F026FA9DF811409DF812509DF813A011
:10E8D0009DF81090DFF8E0B8DFF8E088002727E027
:10E8E000204602E0504600E02846FF2813D0032FC0
:10E8F00011D8DFE807F00B0805020221404608E0C6
:10E900000121404605E04FF4807101E04FF40071B1
:10E91000584607F0E2FD7F1C042F0BDA032FFAD8CC
:10E92000DFE807F006050403F5E7DBE7DCE7D7E7F8
:10E930004846DAE70021317070680028B7D004211A
:10E9400031704CF25032A9E7FEF7A9F8002131707E
:10E9500070680028ABD0052131709DE72820FEF7B4
:10E960009CF80021317070680028A0D00621317019
:10E9700092E7FEF794F8002030707168002996D075
:10E98000DFF844288CE70020307000BF07B0BDE8F6
:10E99000F08F000038B5DFF83C48207C062800F2F4
:10E9A0008180DFE800F00415235162657400DFF810
:10E9B0002028DFF8241804F14000F6F7A2FDE189D1
:10E9C000606807F088FD012020740021A16031BD3E
:10E9D000DFF80828DFF8001804F14000F6F791FD91
:10E9E000E189606807F079FD02204EE0A289DFF836
:10E9F000E857521C332A0FD3C82000901923E1890D
:10EA00006068FFF7FDFD42F21072294604F14000F4
:10EA1000F6F777FD042038E0A06890420BD2192267
:10EA2000294604F14000F6F76CFDE189606807F0C3
:10EA300052FD032029E042F21072294604F1400001
:10EA4000F6F75FFD042020E0C822DFF88C1704F100
:10EA50004000F6F756FDE189606807F03EFDA068CA
:10EA6000401CA0600221217431BD2068D0B162E257
:10EA7000DFF85C27DFF8601704F14000F6F741FD8E
:10EA8000E189606807F027FD0620207431BD40F65B
:10EA9000FF70FEF702F8E189606807F01EFD0020B4
:10EAA0002074A06031BDF8B50E46DFF80C17DFF812
:10EAB000244705464FF4007228896160A081002137
:10EAC0002161A1602175E28126602988814221D2DD
:10EAD000A0F59660A08182B26988914215D2A0F516
:10EAE0009660A08183B2AA88DFF8D0169A4207D236
:10EAF0006160A0F59660A0810221E181A87B0AE017
:10EB00000120E0816160687B05E04FF48070E08166
:10EB1000287B00E0E87AA07400F074FBFF28E07422
:10EB200003D1E87A00F06EFBE074E07C022803D1A8
:10EB3000DFF88816E1622086002002F01EFFE07CEC
:10EB4000082806D1012002F018FFE1896068FBF770
:10EB50000AFFE089DFF86856012807D0022803D0B1
:10EB6000B0F5807F04D007E0032102E0022004E03A
:10EB7000012185F8D01002E0002085F8D000E07C6B
:10EB8000F8F7E6FAA07C08281ABF28280020012000
:10EB90002075E07C03280BD1A2890A27B2FBF7F786
:10EBA000BFB207EB8701B2EB410104BF0A32A28179
:10EBB000217D69B9A38919464FF0640CB1FBFCFCB7
:10EBC0001FFA8CF7642202FB171109B96433A38181
:10EBD00010B90FF2693073E0032815D1A089401EE7
:10EBE000A0810021A1636163C0B2FCF725FCDFF8BE
:10EBF000F0150843606302464FF0FF3042400FF2C9
:10EC0000A941A263E1635CE0022816D1E189606852
:10EC100007F063FC218EE06A07F05DFCA1890A22FF
:10EC20000846B0FBF2F080B2606200EB8003A1EB1B
:10EC30004301A1620FF2A93042E0092818BF07285A
:10EC40002BD1012084F82000F8F776FA50B101208A
:10EC5000A0810221E07C84F82010072804BF032152
:10EC600084F82010A08902460A21B0FBF1F080B29E
:10EC700000EB8003A2EB4302521CD1B2D0B207F0EA
:10EC80002FFCA0896168E083A1613146E089A083FF
:10EC900004F1180007F047FC13E008280CD1A08904
:10ECA00008B9B047F1BD401EA08140F6FF70FDF7E6
:10ECB000F4FEDFF8240503E0012161740FF2411036
:10ECC000E06395F8D000342250430121295405F126
:10ECD0000C0695F8D030E16B5343F05858B12C1D19
:10ECE0000020E15005F10C0195F8D0305A438A58C4
:10ECF000BDE8F240104739B104F14000BDE8F840EA
:10ED00004CF25032F6F7FDBBF1BD70B5DFF8B054F0
:10ED100095F8D00034246043002129542A1D95F829
:10ED2000D0006043115005F1080295F8D00060430F
:10ED3000115095F8D01004290CDA6143681890F846
:10ED4000300028B905F10800DFF88024425001E0C6
:10ED500000235350DFF87C64F07C20B9F18970689F
:10ED600007F0B9FB3BE0032802D1F189706807E0A6
:10ED7000022808D1F189706807F0AFFB318EF06A84
:10ED800007F0ABFB2BE008280FD105203074DFF82B
:10ED90004024DFF8441406F14000F6F7B2FBF18995
:10EDA000706807F098FB062018E0092818BF0728AC
:10EDB00003D1002007F0CCFB11E0042000213074C7
:10EDC000717406F14000DFF808240FF23501F6F700
:10EDD00098FBF189706807F07EFB05203074F07CA9
:10EDE00001280CD095F8D00005F1080144430959D9
:10EDF00029B100208847BDE87040FFF733BC70BDE3
:10EE000038B5DFF8D043207C062800F29380DFE895
:10EE100000F004122045617D8E00DFF8B423DFF896
:10EE2000C41304F14000F6F76CFBE189606807F059
:10EE300052FB012068E0DFF89023DFF8A81304F10B
:10EE40004000F6F75EFBE189606807F046FB0220B0
:10EE50005AE0207DDFF88C5398B14FF49671009101
:10EE60004FF4FA73A289E18960685200FFF7C8FB8A
:10EE7000DFF85C23294604F14000F6F742FB04204A
:10EE800042E04FF4FA72294604F14000F6F739FBEC
:10EE9000E189606807F01FFB032035E0E1896068C5
:10EEA00007F01BFBA068A289DFF83813401CB0EB09
:10EEB000420FA06006D1C64A04F14000F6F721FBDC
:10EEC000042021E04FF4967204F14000F6F719FB9C
:10EED000022019E0607CC34D58B101210020FDF7EC
:10EEE000A2FDB94A294604F14000F6F70AFB0620C4
:10EEF0000AE0B74A294604F14000F6F702FBE1892F
:10EF0000606807F0E8FA0520207431BDE189606887
:10EF100007F0E3FAAA4890F8D02000F10801342065
:10EF20004243895831B1BDE8344000200847206889
:10EF300000B100E031BDBDE83240004710B5A54C3E
:10EF4000207C04284AD8DFE800F003141732400080
:10EF500044F25062A44904F14000F6F7D2FAE18984
:10EF6000606807F0BAFAA089002814BF01200420C5
:10EF700029E04FF47A721CE0E189606807F0ADFA8D
:10EF8000A068A2899849401C9042A06007D144F231
:10EF9000506204F14000F6F7B4FA042013E04FF495
:10EFA000167204F14000F6F7ACFA03200BE04FF4C0
:10EFB00016728D4904F14000F6F7A3FAE189606802
:10EFC00007F089FA0220207410BD607C18B941F264
:10EFD000883285490EE1206800B162E010BD000072
:10EFE00010B57C4C207C04285AD8DFE800F0030AD6
:10EFF0002C334400E189606807F06DFA0121217427
:10F0000042E0E189606807F068FAA068401C0A28BD
:10F01000A0600CD2616A884209D041F288327349FB
:10F0200004F14000F6F76DFA0020207410BD0221B3
:10F0300021744FF6E8526D4904F14000F6F761FA89
:10F040000020A06010BDE189606807F044FA032049
:10F05000207419E0E189606807F03FFAA068401C5D
:10F060000A28A06004D2A16A884218BF022000D1F9
:10F070000420207408E0607C78B9E189606807F0BA
:10F080002CFA607C401C607404F14000BDE8104024
:10F0900041F288325549F6F734BA206800B100E0F1
:10F0A00010BDBDE81040004710B54A4C207C062832
:10F0B00000F27F80DFE800F004111D344860710029
:10F0C0004FF4C8724A4904F14000F6F71AFAE18990
:10F0D000606807F000FA01205DE0C822444904F1AD
:10F0E0004000F6F70EFAE189606807F0F6F90220B1
:10F0F00051E0E189606807F0EEF9606B3C49002857
:10F100004CBF4FF44872C82204F14000F6F7F9F9F9
:10F11000606B400060630321A068401CA06029E090
:10F12000C822334904F14000F6F7EBF9E189606841
:10F1300007F0D3F9A068202838BF02211AD3042091
:10F1400000212074A16010BDE189606807F0C3F957
:10F15000A06B274900284CBF4FF44872C82204F125
:10F160004000F6F7CEF9A06B4000A0630521A0682F
:10F17000401CA060217410BDC8221D4904F140004C
:10F18000F6F7BFF9E189606807F0A7F9A0682028C1
:10F1900034BF04200620207410BD607C30B9E189A2
:10F1A000606807F098F9C822114923E0206800B18F
:10F1B00077E710BD14E000E0000C014000100140B2
:10F1C000C406002098060020A086010059E8000827
:10F1D000E0930400A007002095E90008400D03001B
:10F1E0000080FFFF01EE00083DEF0008E1EF00089E
:10F1F000A9F0000804F14000F6F783F9607C401C98
:10F20000607410BD0A2811DBA0F10A01282901D27F
:10F2100001207047A0F132010A2901D20220704773
:10F220003C38072801D203207047FF2070470000B8
:10F2300010B404680B684A6804F441541C438B689A
:10F240001443CA681C430B6914434A6989691C4307
:10F2500014430C4340F81C4B026822F40062026025
:10F2600010BC7047016841F04001016070470168BF
:10F2700021F040010160704740F80C1F70470C30CE
:10F28000FFE7006880B27047083000680140481E00
:10F290008041C043C00F704770B504460122256805
:10F2A000A6686168284600F037F86269F1B228461E
:10F2B00000F0EBF8A169284600F05AF8E268F1B2D4
:10F2C000284600F081F8E2692169236AD2B2C9B206
:10F2D000284600F094F8F1B22846BDE870400122BB
:10F2E00000F0E6B810B5044600F04AF80120FEF739
:10F2F000C3FA2046BDE8104000F04BB800F002B859
:10F3000000F057B8DFF8E8110A6822F470220A60AA
:10F310000B68184308607047A2B1CA0504D5021DE6
:10F32000136843F4807313604A0504D5021D136803
:10F3300043F480631360890719D550F8082F42F011
:10F34000020213E0CA0504D5021D136823F480737A
:10F3500013604A0504D5021D136823F4806313600B
:10F36000890704D550F8082F22F002020260704786
:10F37000083001B123E0026822F4006202607047A5
:10F3800050F8081FCA0703D4016841F00101016069
:10F39000704750F8081F41F008010160026811072A
:10F3A000FCD4026842F00402026001684A07FCD4FF
:10F3B000704750F8081F41F4807101607047016880
:10F3C00041F4006101607047012902D002290BD08D
:10F3D000704750F82C1F21F470010160521E036821
:10F3E000120502F4700209E050F8381F21F44011B0
:10F3F0000160521E0368120502F4401255E070B419
:10F4000006290CDA00F1340401EB810125681F267E
:10F410008E40B54302FA01F12943216015E00C2921
:10F4200004DA00F13004891F256805E010290CDAA0
:10F4300000F12C040C39256801EB81011F268E4058
:10F44000B54302FA01F10D4325600A2A00DA00E013
:10F450000CE050F8101F02EB420207249440A14335
:10F4600003FA02F20A43026070BC7047122A0ADAF9
:10F470000A3A50F80C1F02EB420207249440A143C1
:10F4800093400B43036070BC7047012902D00229EE
:10F4900005D0704750F8081F21F4602103E050F8B0
:10F4A000081F21F4E041016003681A4302607047BD
:10F4B00072B1CA0705D500F10802136843F480133E
:10F4C0001360890713D550F8082F42F400420DE06D
:10F4D000CA0705D500F10802136823F480131360EE
:10F4E000890704D550F8082F22F4004202607047C3
:10F4F0000424014010B504462179206800F08AF800
:10F500002179206804F1080200F0ABF894F9240096
:10F51000010007D5394A00F00F001044002100F81F
:10F52000041C02E0364800224254012294F92410BF
:10F53000344B01F01F008240490943F8212010BDDF
:10F540004FF47A70304900E000BF0A68D30704D452
:10F550000246501E92B2002AF6D1032128E0032170
:10F560002AE02A4A43E010B5294C02220321204612
:10F5700000F045F92046BDE810400822032100F0C4
:10F580003EB910B5224C04220321204600F02EF98A
:10F5900002220321204600F029F92046BDE8104050
:10F5A0000822032100F022B90421194800F0D4B840
:10F5B000174800F0C1B80421154800F0ADB8082282
:10F5C0000421134800F01BB910B5114C042204218A
:10F5D000204600F00BF902220421204600F006F933
:10F5E0002046BDE810400822042100F0FFB89060DA
:10F5F000116070470421064800F07DB818ED00E066
:10F6000000E400E000E100E0440002404800024065
:10F610000000024030B4DFF80022904202D10529F8
:10F6200000DBFEE701EB810300EB830202F108033C
:10F6300000251C68640864001C601D6002F10C0455
:10F64000002302F1100523602B6042F8143F89006B
:10F6500050F8042F0F2303FA01F11143016030BC6D
:10F660007047DFF8B43110B4984202D1042900DDAC
:10F67000FEE701EB810300EB8300116800F1100449
:10F68000216000F1140193680B6000F10C01146912
:10F69000A4B20C6050F8084F5168D36824F47C542D
:10F6A0000C4351691C430C430460137E012B04D1AD
:10F6B000016841F04001016003E0036823F040036A
:10F6C0000360517E012904D1036843F08003036085
:10F6D00003E0016821F080010160917E29B9026890
:10F6E00022F01002026010BC7047016841F0100166
:10F6F000016010BC7047DFF82021904202D105293B
:10F7000000DBFEE701EB810200EB820050F8081FEE
:10F7100041F02001016070473F4A904202D1052923
:10F7200000DBFEE701EB810200EB820050F8081FCE
:10F7300041F0010101607047374A904202D105292A
:10F7400000DBFEE701EB810200EB820050F8081FAE
:10F7500049084900016070472F4A904202D10529AB
:10F7600000DBFEE701EB810200EB82000C30006859
:10F7700070470A430260704730B4022A04D0042A5A
:10F7800016D0082A22D02FE001EB8105026800EB99
:10F790008500083002248B0000689C40224000F065
:10F7A000020030BC002A1ABF002801200020704748
:10F7B00001EB8105026800EB8500083004248B0012
:10F7C00000689C40224000F00400EAE701EB81055C
:10F7D000026800EB8500083008248B0000689C401C
:10F7E000224000F00800DCE7FEE7000000BF50F810
:10F7F000043F890002FA01F1194301607047064B8A
:10F80000984202D1052900DBFEE701EB810300EB02
:10F81000830050F8081FACE700040240011D006897
:10F8200000F00CB800F110024168006889B200F0E5
:10F8300095B800F06DB800F071B8000030B40A88D7
:10F8400000F128031A60DFF8D423904218BFB0F10A
:10F85000804F27D0DFF8B03398421CBFDFF8AC43AD
:10F86000A0421FD0DFF8A83398421CBFDFF8B04396
:10F87000A04217D0DFF8AC3398421CBFDFF8A84392
:10F88000A0420FD0DFF8A43398421CBFDFF8A0439A
:10F89000A04207D0DFF89C3398421CBFDFF89843A2
:10F8A000A0420FD1036823F07003036004688B78D3
:10F8B00003F060031C43046004680B7903F0100339
:10F8C0001C43046000F12C048B68DFF8485323606C
:10F8D000A8421CBFDFF84033984213D0046824F4D8
:10F8E0004074046003688C8904F44074234390429C
:10F8F0001CBFDFF82C239042036003D1897B00F109
:10F900003002116050F8141F41F0010115E00000B1
:10F9100000BF016841F001010160704701684908BA
:10F92000490001607047016841F080010160704743
:10F93000016821F0800101607047016030BC7047B0
:10F940004430012904D1016841F40041016070474D
:10F95000026822F40042026070470000032900D9C7
:10F96000704730B4DFE811F0040048009000D70081
:10F9700000F12003196849084900196000F11801D5
:10F980000C68A408A4000C601D6811880D431D605C
:10F990001C6824F002041C601D689188DFF87C421A
:10F9A0000D431D60A0421CBFDFF87452A84240F016
:10F9B000DE80196821F0040119601C6851880C432D
:10F9C0001C601D6825F008051D601C68D1880C436B
:10F9D0001C6050F8043F23F48073036004681189AD
:10F9E0000C430460036823F40073036004685189C6
:10F9F0000C43046030BC704700F120010B6823F019
:10FA000010030B6000F118031C6824F440741C60A0
:10FA10000B68158843EA05130B600C6824F020047A
:10FA20000C600B68948843EA04130B60DFF8EC3138
:10FA300098421CBFDFF8E841A04240F098800B6874
:10FA400023F040030B600C68538844EA03140C60F5
:10FA50000C6824F080040C600B68D48843EA04131B
:10FA60000B6050F8041F21F4806101600368118964
:10FA700043EA81030360036823F4006303600168C1
:10FA8000528941EA820145E000F120010B6823F42C
:10FA900080730B6000F11C031C68A408A4001C60A8
:10FAA0000B68158843EA05230B600C6824F4007486
:10FAB0000C600B68948843EA04230B60DFF85C3128
:10FAC00098421CBFDFF85841A04250D10B6823F484
:10FAD00080630B600C68538844EA03240C600C6854
:10FAE00024F400640C600B68D48843EA04230B60A0
:10FAF00050F8041F21F4805101600368118943EA22
:10FB000001130360036823F4005303600168528902
:10FB100041EA021111E700F120010B6823F4805340
:10FB20000B6000F11C031C6824F440741C600B681B
:10FB3000158843EA05330B600C6824F400540C600C
:10FB40000B68948843EA04330B60DFF8D0108842D6
:10FB50001CBFDFF8CC30984209D150F8041F21F4C3
:10FB6000804101600368118943EA8113036030BC5E
:10FB700070470000032915D8DFE801F00204060BE6
:10FB8000183002E0183005E01C30016821F07001E7
:10FB900034E01C30016821F4E0410160036843EA6D
:10FBA000022303607047000003290BD8DFE801F04F
:10FBB00002040608343004E0383002E03C3000E053
:10FBC0004030026070470000032913D8DFE801F0DD
:10FBD00002040609183002E0183003E01C30016806
:10FBE0000AE01C30016821F400610160036843EA07
:10FBF000022303607047000021F0080101600368E0
:10FC00001A430260704700000004004000080040F2
:10FC1000000C00400010004000140040002C014087
:10FC200000340140004C01400050014000540140AC
:10FC300000180040001C00400020004000BF50F8A9
:10FC40000C2F11430160704750F80C2F22EA01017C
:10FC50000160704700F10C021030126800680A4021
:10FC6000084218BF002A01D00120704700207047C9
:10FC700050F8102FEAE7000038B5044600200F4A7C
:10FC800094421CBF0E4A94420D460AD00D4A94423B
:10FC90001CBF0D4A944204D00C4A944204D1032064
:10FCA00000E00220FDF768FC00EB5500B0FBF5F02A
:10FCB00080B244F8080F31BD00000000004400404D
:10FCC00000480040004C0040005000400038014017
:10FCD00050F80C2F22F4C06203E050F80C2F22F4ED
:10FCE00080520260036819430160704750F8102F7A
:10FCF00022F44052F5E750F80C1F41F40051016026
:10FD0000704750F80C2F22F0080203E050F80C2F37
:10FD100022F00402114301607047001D0068C0F327
:10FD20000800704750F8142F22F04002F2E750F814
:10FD3000142F22F08002EDE700EB911001F01F017B
:10FD40000068C84000F00100401E8041C043C00F61
:10FD5000704700EB9110012302680DE0C1F3891395
:10FD6000C1F389121B181058012201F01F0102FA79
:10FD700001F101431960704701F01F0103FA01F11D
:10FD800022EA01010160704707E01C220021DFF830
:10FD90001803FBF74ABB000000BFC3487047C348C5
:10FDA0007047C1480079704710B5F9F74BFFBE4C5A
:10FDB00028B90622002104F10F00FBF736FB04F1FD
:10FDC0000F0010BD01460622B948FBF71ABBF1B57A
:10FDD0000C46002818BF002C8AB017461E4619D0C2
:10FDE000ADF80C0003A800F091F99DF81800012867
:10FDF00010D19DF81A000025C0F3810001289DF85C
:10FE00001A0008BF0125C0F30110012808BF45F002
:10FE1000020515B900200BB0F0BD68460021002294
:10FE2000002380E80E0007222146FBF7EAFA0222AF
:10FE30000AA90DF10700FBF7E4FA8DF809708DF8B7
:10FE40000A608DF80B500C2269469620FAF76CFE7A
:10FE500001200BB0F0BDF8B5934C1646236207465F
:10FE60000D46E661F6F722FF38BB204600F04EF95A
:10FE70003846F6F7B8FF20B90A2F09D0204600F01F
:10FE80002DF9172F04D1012005216083217114E081
:10FE9000207B012806D138460A2806D1204600F0EA
:10FEA00022F950B9216AA9B110E1F6F724FF38B15F
:10FEB000132F04BF0D20F6F7ECFEE16951B109E103
:10FEC0000DB1B047F1BD2046BDE8F4400FF28911F5
:10FED00000F036B9F1BD70B517280C46154603D1B0
:10FEE00071490A7B012A02D1F6F7F1FE40B16E4C4E
:10FEF000204600F089F92046BDE8704000F08FB937
:10FF0000694E304600F09DF92A4621463046BDE84C
:10FF1000704000F0ABB93EB5F4F736F80090654C90
:10FF2000207A40B1FFF740FF014620460622F3F752
:10FF3000A7FF002020729DF800000B282CD15A4DFD
:10FF400005F10F0001F015FC01F037FC40B1284627
:10FF500000F0BCF9022229468F20FAF7E5FD0BE0FC
:10FF600001208DF80000A97C687CF8F712FA0122C4
:10FF700069469120FAF7D8FD0120207205F10F01A2
:10FF800068460622F3F77CFFDDE9000101F066FC1C
:10FF90000122494949480EE0052810D101F0F7FB3C
:10FFA00001F00BFC444C18B100222146444802E009
:10FFB000002221464348F4F79DF803B030BD28B92C
:10FFC000D4E9000101F04AFC03B030BD01F0F8FBB8
:10FFD00008B10120207203B030BD10B584B0F8F72D
:10FFE000F7FE38B3F9F72EFE20BBF8F747F808BB49
:10FFF0002D4C1C2200212046FBF717FAF8F7E4FEEF
:020000040801F1
:100000002080204600F082F8207B012812D168462B
:1000100000F0BEFE617E9DF80500022938BF08464B
:10002000012807D1204604B0BDE810400FF20901B5
:1000300000F086B804B010BD10B51B4C207905281F
:1000400008D1207CFEF77DFA608B1F49BDE8104087
:10005000F9F7C2BD10BD0000F8B5134C2079052892
:100060001AD1658B0126F0B2F8F748F80746F0B2CE
:10007000F8F71CF8A84212DA022F02D1F0B20428D5
:1000800006DAB5F5966503D4761CF0B20428EADDED
:10009000216A01B11AE0F1BD207B0128F8D1E169A4
:1000A0000029F8D016E00000947C0020967C002007
:1000B000A37C00209408002040420F0018AC0108E7
:1000C00048AC010840AC010899E50008BDE8F440DF
:1000D00000200847BDE8F44000200847817B41F03C
:1000E000030181737047807B00F001007047807BC3
:1000F000C0F340007047807BC10705D5400800F081
:10010000010080F0010070470020704730B430F8E3
:100110000C2BBE4C4FF49273B2FBF3F39BB24FF433
:1001200092711D0301FB1322C2EBC20305EB4305D1
:1001300005F545256560294630BC0E22FEF745B819
:10014000BCB5B24D286107220271002228694283A2
:1001500029604FF46823022200216B602A72ADF8F7
:100160000010408B08B901212973287B0DE011D0C4
:1001700018E0C2B22C69521E4FF496635A43090329
:10018000628301F567216960C0B2F7F78FFF040051
:10019000EDD50024287B0428DFBF401C2873C1B2A2
:1001A0000429E6DD287B04282DDC2A7A6968684664
:1001B000FEF70BF82869BDF800100288914202D1C1
:1001C000052303711FE0438B5B1C43834FF496624E
:1001D000297B4F1E02FB17339BB2A4B2A34204D269
:1001E0006968287A411869600CE0491CCBB2042B7D
:1001F000297308DCC9B2491E4A431B03428303F535
:1002000067236B60F9E0F2E010B50446F8F733F8C5
:10021000A4F81500F8F73FF8A4F8170010BD10B5C2
:100220000446F8F71CF82074F8F7CBF86074F8F778
:10023000D4F8A074F7F7FBFFE074F8F704F8207522
:1002400010BD38B504464FF6FF75B4F81500A84246
:1002500003D1F8F710F8A4F81500B4F81700A84275
:1002600003D1F8F718F8A4F8170031BD70B50446AB
:100270000D46207CFF28164602D1F7F7F0FF2074C8
:100280005DB11EB10020F8F7DBFA0BE0E07B607493
:10029000FF2808D1F8F789F804E0607CFF2802D134
:1002A000F8F78FF86074A07CFF2802D1F8F795F872
:1002B000A074E07CFF2802D1F7F7B9FFE074207D3D
:1002C000FF2802D1F7F7BFFF207570BD2DE9F84375
:1002D00007464FF49271B7F80080B8FBF1F5ADB264
:1002E0002C0303F00BFC04F5452481464FF48052A7
:1002F0002146FDF76AFF4FF4927000FB1588C8EBAA
:10030000C80109EB4100797C427900268A421CBF72
:1003100041710126B97C82798A4218BF817100D16E
:100320003EB121464846BDE8F8434FF48052FDF700
:100330002EBFBDE8F183BCB5344D29690020ADF86E
:100340000000488B002801BF6868B0F5682F0121C4
:100350002973287B0DE011D018E0C2B22C69521E1F
:100360004FF496635A430903628301F5672169607C
:10037000C0B2F7F79BFE0400EDD50024287B0428CB
:10038000DFBF401C2873C1B20429E6DD287B0428A6
:100390002DDC2A7A69686846FDF717FF2869BDF8E1
:1003A00000100288914202D1052303711FE0438BA4
:1003B0005B1C43834FF49662297B4F1E02FB17336D
:1003C0009BB2A4B2A34204D26968287A411869603A
:1003D0000CE0491CCBB2042B297308DCC9B2491EBE
:1003E0004A431B03428303F567236B6005E001204A
:1003F0002873296828698847B3BD054803F086FB40
:1004000001460448FAF700F9B3BD00008008002057
:1004100037030108947E002077B581B004469DF82B
:100420000800314D00F0E0F806469DF8090000F0A4
:10043000DBF8294600F02CFB314600F095FB2060EC
:100440009DF80C0000F0D0F806469DF80D0000F075
:10045000CBF8294600F01CFB314600F085FB6060BC
:10046000F7F729FFADF800009DF8000000F0BCF898
:1004700006469DF8010000F0B7F8294600F008FB99
:10048000314600F071FBA060F7F72BFFADF80000DC
:100490009DF8000000F0A8F806469DF8010000F065
:1004A000A3F8294600F0F4FA314600F05DFBE06065
:1004B00004B070BD0D48807870470C48704738B55F
:1004C000044600F0D7FB0A4D2870C0B200F08CF84B
:1004D0000146204606F040F9064900F0D9FA00F03E
:1004E000C9FB6870288832BD8180803BA07E0020D7
:1004F000B67E002000007F4310B50020234CF8F7A3
:1005000027F920710120F8F723F960710220F8F72C
:100510001FF9A0710320F8F71BF9E0710420F8F728
:1005200017F920720520F8F713F9607210BD80B535
:100530000020FFF7E1FF164816498268BDE8084031
:100540001047F8B5114908440025047901F1100657
:10055000012707FA05F004421CBF306880476D1C74
:10056000361D082DF5DBF1BD0849084400797047B8
:10057000064A10440171704707494FF40050086063
:1005800070470549082008607047000028080020CF
:1005900098060020500800201010014080B500206F
:1005A000F8F740F808B1002008E001BD80B501204F
:1005B000F8F738F808B1012000E001BDFCF714FCA1
:1005C000BDE80240FCF7FFBB80B50220F8F72AF82F
:1005D00008B10220F2E701BD80B50320F8F722F848
:1005E00008B10320EAE701BD00280AD0B0FA80F183
:1005F0008840D1F19D01C905020672F1004241EB2C
:100600001020704710B5FF2313EAD0541DBF13EA22
:10061000D1529C429A4239E0A41ADA0780EA0103D7
:10062000134042EA012142EA0020421A3CBF641E04
:1006300001EB4202090AB2FBF1FE01FB1E2212028B
:10064000B2FBF1F001FB10226EF30F201202B2FB9D
:10065000F1FE4EEA00207F3406DDFE2C24DA53EA58
:10066000500050EBC45010BDD4F1020401FB1E2217
:1006700040F08071192C1DDC21FA04F0C4F1200433
:10068000A140114371F10042584110BD9C421ABF74
:1006900003EAD1529A420FE080EA010E0EF00043C5
:1006A000400004D0490016D143F0FF4010BD49007E
:1006B00008BFD343180010BD9C4205D1D21AF7D011
:1006C00001F00041484010BD4A0212BF08464840B0
:1006D00000F0004010BD4AB90902B1FA81F2914020
:1006E00044B1A418C00140F000409EE7C90141F0A8
:1006F000004152420002B0FA80F4A040141B94E77B
:100700002DE9F8450D4606462C46600000F0A8810C
:1007100030464FF07E5102F00FFA00F0A181DFF871
:100720004C1302F009FA06D160000016401C02D1F9
:10073000610200F0958170000016401C00F00381FA
:10074000720000F0008160000016401C00F0FB8089
:10075000274678000DD0000EC0F196001828A8BFDB
:1007600007F0004705DA0028C4BF27FA00F202FAB2
:1007700000F7F00F0ED0002C48BFC4F10044380041
:1007800048BFC0F10040844204D0AFF300806FF056
:10079000004667E126F00040B0F5000F07D20020C8
:1007A00000906946304606F017F8064606E0C00D90
:1007B0007E3826F0FF46009046F07C56F00F1CD0A5
:1007C000780026F0004639460DD0000EC0F19700A3
:1007D0001828A8BF07F0004705DA0028C4BF27FA89
:1007E00000F202FA00F7002948BFC1F10041002FD2
:1007F00048BFC7F10047B94201D1002400E00124FD
:1008000030469B49FCF726FD1ED2334623F00041BB
:10081000C80D00F101070ED0002F0CDDFF2F05DB06
:100820004FF0FF4603F000431E430AE026F0FF4668
:1008300046EAC75605E021B10121304605F0ECFF3C
:1008400006460098401E00903146884800F08CF91A
:1008500007464FF07E50314600F086F90146384693
:10086000FFF7D0FE0646314600F012F98046814877
:10087000414600F00DF9804900F076F9414600F05C
:1008800007F97E4900F070F9414600F001F9394658
:1008900005F062FF314600F0FBF8394600F064F9DC
:1008A0000646009800F0FCF907467548314600F00E
:1008B000EFF8394600F058F9294600F0E9F84FF012
:1008C0004741FCF7C7FC37D36E4905F0EBFF30D941
:1008D000C10F14BF4FF03F414FF07C5100F044F97D
:1008E00000F0C8F982463046294600F0D1F80646A5
:1008F0003846294600F0CCF80546504600F0D0F9BD
:100900000146284605F028FF5F4900F0C1F831464E
:1009100000F02AF94FF07E585246414605F0D4FFC8
:100920000646720008D070000016401C05D1710206
:1009300003D14FF0FF4600E00026002C00F092802B
:1009400086F000468EE072001016401C02D11202A2
:1009500040F0888062001016401C04D1120218BFBB
:100960002E4640F07F80620001201216521C35D0C6
:1009700023465A000BD0120EC2F19602182AA8BFC5
:1009800003F0004303DA002AC4BFD340934022009F
:1009900048BFC2F100421F0048BFC7F10047BA423A
:1009A00018BF00209C465FEA4C020ED0120EC2F126
:1009B0009702182AA8BF03F0004306DA002AC4BF32
:1009C0002CFA02F303FA02FC634638B1002B48BF4D
:1009D000C3F100439F420CBF002001207200121699
:1009E000521C06D1730204D1F10F15D1E40F34D09B
:1009F0002DE062001216521C14D1630212D126F0AF
:100A00000040B0F5000F17D200210091B8B169463F
:100A1000304605F0E1FE12E0E40F01D1002819E0B4
:100A2000A8B106E0002814BFF10F0021E40F10D197
:100A300069B14FF0004615E0C00D7E380090E40F1C
:100A4000009802D1002808DC01E0002805DD00261E
:100A500008E0002918BF0D4E04D14FF0FF4601E019
:100A60004FF07E563046BDE8F28500BF000080BFE3
:100A7000F304353F1502993E11AECC3EC0AA2A3F81
:100A80003BAAB83F010000471872313F000080FFC9
:100A9000FF2212EAD05C1DBF12EAD1539445934263
:100AA0002BE09C44D30780EA01021A4043EA00206D
:100AB00043EA0121A1FB0030C04238BF40007CF175
:100AC0007F010BDBFE294ADA5B0842EAC15153EA97
:100AD000006373F1004C51EB10207047D1F1080C0A
:100AE000DCF120012FDB5B0810FA01F10B4320FA47
:100AF0000CF073F100415041704794451CBF02EA6D
:100B0000D153934280EA010202F000421DD040001E
:100B100019D0490017D05BB9634514D00902B1FA66
:100B200081F39940BCEB030CC00140F00040C1E7E9
:100B30000002B0FA80FC10FA0CF0B3EB0C0CC90107
:100B400041F00041B6E71000704740000AD049006C
:100B500008D010F1807F94BF11F1807F02E042F055
:100B6000FF407047D043704790EA010F45F1FA8586
:100B700081F00041431A4FF000423EBF5340C01A7B
:100B8000C91800BFD3095FEAD05C13EB400F34BF34
:100B9000B3EB410F40E07CEBD1530CD342EA01218F
:100BA00022D8D1EB402009D3400A28BF5FEA500188
:100BB00040EBCC507047401A15D04002B0FA80F29A
:100BC000521C9040400A4FEA3C23B3EB026384BFBF
:100BD00000EB730007E040F400001A16DB07C2F1D7
:100BE0000102D04018437047182BFCDC31FA03F2A5
:100BF00002FA03F3591A38BF42F00102D2EB402047
:100C00003CBF4000ACF1010C5FEACC5CC20572F164
:100C100000414CEB5020704713EB400F0FD2C942FC
:100C200009D0ACEBD153022B03DB4902172BDDDDDE
:100C300070479143401AC042D5D10020704713EB52
:100C4000410FD0D36FF0000070470000C0F3C752CF
:100C50007E3A09DD182A0CDA6FF07F41D14020EA94
:100C6000510040188843704700F0004008BF40F032
:100C70007E507047C0F3C7517E390EDDC217D1F1E7
:100C8000200106DD000240F00040C8401044504002
:100C90007047D04380F0004070470020704700004C
:100CA000C2175040801AB0FA80F10AD08840D1F1C2
:100CB0009D01D20742EAC151020672F1004241EBA6
:100CC000102070473348704732490DE031494B7D61
:100CD000984202D0487500207047052070472E4981
:100CE00017E02E4919E02E491122F3F7C9B8294916
:100CF000002081F8460070472649887170472549D1
:100D000048717047234908717047224988707047BD
:100D100024491522F3F7B4B823490F22F3F7B0B8EA
:100D20002249FAE722497222F3F7AAB8214870470C
:100D300021492622F3F7A4B82049FFE70E22F3F752
:100D40009FB81F4870471F4870471F4912E011495C
:100D500081F8720170470F4981F8730170471B4990
:100D600013E01B490D22F3F78BB81A491422F3F74D
:100D700087B819491222F3F783B818495522F3F7B7
:100D80007FB81749DAE71749AEE71022F3F778B8CA
:100D90001549D3E728710020467100205B710020BF
:100DA0006A7100207B710020907100209F710020EB
:100DB000AE710020B3710020207200204672002026
:100DC000627200205A73002094720020A6720020E4
:100DD000B6720020D1720020E5720020F772002068
:100DE0004C73002077730020C372002000180CD2CF
:100DF000010E7F3909D4D1F11F015DBFC00140F060
:100E00000040C8406FF000007047002070470000AD
:100E1000F8B5DFF84444E060074686B097F8330041
:100E200000280D4638D00722002107F14D00FAF7BF
:100E3000FCFA39780026002902BF787800280126BC
:100E40007878002802BFB8780028761CB878002887
:100E500002BFF8780028761CF878002802BF38799D
:100E60000028761C3879002802BF78790028761C83
:100E70007879002802BFB8790028761CB879002854
:100E800002BFF8790028761CC6F10706F2B239468F
:100E900007F14D00FAF7BEFA18214FF444302172E1
:100EA00060600146E068022258302560FDF78DF948
:100EB000E668684606F158011822F2F7E1FF0222BF
:100EC00031466846FAF78DFA0725C0B2D8B1E36813
:100ED00093F8331029B1022203F14D016846FAF765
:100EE00080FAC0B278B104F10802211D102002F08E
:100EF00011FEE068418F491C41876168B1F5452FBB
:100F000038D3C5714AE0227A6168E068921E891C74
:100F10005A30FDF75AF9E668684606F1580118227A
:100F2000F2F7AEFF06F12802107A032805D0D2E9C5
:100F30000001009B157B034000932A46314668461A
:100F4000FAF74FFAC0B2E0B1E36893F8331029B171
:100F50002A4603F14D016846FAF743FAC0B280B160
:100F600004F10802211D102002F0D4FDE068418F39
:100F7000491C418704F11001B848F9F745FB07B057
:100F8000F0BDE1680520C87100F0B0FBE1684B8F4F
:100F9000B349102201EB0311FDF717F9E06821684E
:100FA000884707B0F0BDAC4908604FF444321823BD
:100FB0004A600B7207E0A84AD0604FF4443050609A
:100FC0001823137211600020B3E0A348C16801F137
:100FD0004D007047F0B444780378C678877804EA07
:100FE000030506EA07021540427990F804C023433E
:100FF0003E4302EA0C00334342EA0C02054013432D
:10100000FF2D1EBF002B0878FF2802D1F0BC012065
:101010007047F0BC0020704770B58F4E0D46F168E8
:1010200004462A46FAF7DDF9C0B250B1F36893F8E6
:10103000331029B12A4603F14D012046FAF7D1F9C0
:10104000C0B270BD70B5844DEB68696886B002228D
:1010500003F15800FDF7B9F8EE68684606F158014B
:101060001822F2F70DFF022231466846FAF7B9F965
:101070000724C0B2D8B1EB6893F8331029B102222B
:1010800003F14D016846FAF7ACF9C0B278B105F149
:101090000802291D102002F03DFDE868418F491C1F
:1010A00041876968B1F5452F2AD3C4713CE02A7A9B
:1010B0006968E868921E891C5A30FDF786F8EE6868
:1010C000684606F158011822F2F7DAFE06F1280206
:1010D000107A032805D0D2E90001009B147B03405D
:1010E000009321466846FFF797FF80B105F108029B
:1010F000291D102002F00EFDE868418F491C418730
:1011000005F110015548F9F77FFA06B070BDE9689E
:101110000520C87100F0EAFAE9684B8F50491022A7
:1011200001EB0311FDF751F8E8682968884706B01C
:1011300070BD10B5484CE0680021C1715830227A6A
:101140006168FDF742F8E068217A5830FAF796F9BD
:1011500010B104F120010BE004F10802211D102060
:1011600002F0D8FC6168B1F5452F06D204F11801F0
:10117000BDE810403948F9F747BAE068C1F30B02FF
:10118000A1F54431090B017442820321C171226827
:10119000BDE8104010477CB52F4CE36818220021B1
:1011A00003F15800FAF741F9F6F757FEE16801F14B
:1011B0005F0210800120907191F838105172F7F79A
:1011C000D8FAE16881F86900FF2804BF012081F89E
:1011D0006900072201F15800FAF713F9FDF70DF83D
:1011E0006668360B05464FF480523103FCF7EDFF7D
:1011F000E068636800F15801A3EB06331822E81891
:10120000FAF7FFF84FF4805231032846FCF7F7FF56
:101210006068E168183060601822A0F54430B0FBC7
:10122000F2F2000B4A820874FFF78BFD011DE068A3
:101230001030F7F76CF8E068418A090A8DF8001061
:10124000FFF781FD01466846F7F761F8E068002185
:10125000C1712268904773BD141C0020947E002049
:10126000007012000300002013F0030F09D0521E7B
:1012700022BF13F8010B11F801CBB0EB0C00F3D037
:10128000704711F0030F14D1121F22BF53F8040B43
:1012900051F804CB6045F7D0121D0AD200BA9CFA6F
:1012A0008CFCB0EB0C0038BF6FF0000088BF012051
:1012B0007047521E22BF13F8010B11F801CBB0EB9F
:1012C0000C00F6D0521C08BF1046704780B503F0E2
:1012D000D5F8BDE8084040F292424FF46E21FCF789
:1012E00074BF80B503F0CAF80078012818BF002049
:1012F00002BDF8B5CA4C0E4686B06060002180F889
:1013000021104FF46F2502F0FBFB0921456020609E
:101310000172684627683E60F9F794F93A7A79686D
:101320006846FCF752FF616807226846FAF759F8E9
:10133000002844D0206800F10802011D012002F0BD
:10134000E9FB26687068B0F5931F38BF04F1080107
:1013500027D361684FF6FF7088837560092103A861
:10136000F9F770F9327A294603A8FCF72EFF2068B6
:10137000017A03A8FAF782F828B10FF2452002F0AB
:10138000C5FB01460DE0206800F10802011D0120A7
:1013900002F0C0FB21684868B0F5931F06D204F143
:1013A0001001A048F9F730F907B0F0BD0968002036
:1013B00088476168002081F8210007B0F0BD6068AF
:1013C000BDF80710818322685168C1F30B03A1F5B2
:1013D0006F21090BC38380F820100120616881F818
:1013E0002100002022681168884707B0F0BD2DE970
:1013F000F04105460E46A98B8E4235D095F82070F7
:1014000002F07CFB8046022105F11C003F03FAF745
:1014100035F807F56F27002400B90124AE834FF497
:10142000805239464046FCF7D0FEE88B6CB1404410
:10143000022205F11C01C01DF9F7E3FF4FF48052B1
:1014400039464046FCF7A3FE06E0C019C11D022242
:1014500005F11C00FCF7B7FE39464046BDE8F041F7
:101460004FF48052FCF7B1BEBDE8F08138B586B0CC
:1014700009216846F9F7E6F8694C2068027A416864
:101480006846FCF7A2FE616807226846F9F7A9FFE3
:10149000002847D0206800F10802011D012002F059
:1014A00039FB25686868B0F5931F38BF04F108015F
:1014B0002AD361684FF6FF70888309214FF46F20AB
:1014C000686003A8F9F7BEF82A7A4FF46F2103A8E1
:1014D000FCF77BFE2068017A03A8F9F7CFFF28B15B
:1014E0000FF2DD0002F012FB01460DE0206800F172
:1014F0000802011D012002F00DFB21684868B0F5CB
:10150000931F06D204F110014648F9F77DF807B0A1
:1015100030BD0968002088476168002081F82100FB
:1015200007B030BD6068BDF807108183226851683C
:10153000C1F30B03A1F56F21090BC38380F82010C1
:101540000120616881F82100002022681168884725
:1015500007B030BD18B583B009216846F9F772F8B5
:101560002F4C2068027A41686846FCF72EFE2068FE
:10157000017A6846F9F782FF28B10FF2450002F0C0
:10158000C5FA01460DE0206800F10802011D0120A6
:1015900002F0C0FA21684868B0F5931F06D204F142
:1015A00010012048F9F730F804B010BD0968002098
:1015B00088476168002081F8210004B010BD000058
:1015C00018B583B00922FF216846154CF9F72DFFA5
:1015D000616807226846F9F714FF2068616840686F
:1015E000C0F30B02A0F56F20000BCA8381F8200026
:1015F000FFF7A7FB00F1230160682030F6F787FEB4
:101600002068416809226846FCF7DDFD6168012019
:1016100081F82100002022681168884704B010BDBD
:101620009C1C0020947E002010B5314C16224FF4F3
:1016300093112046FCF7C9FD16212046F9F72BFF30
:10164000D8B916212046F8F7FDFF0120002160756A
:10165000217504F113022146601CF6F7C1FD04F167
:101660001301601CFFF7B6FC38B92046BDE81040F6
:1016700016224FF49311FCF7A6BD10BD70B50446B9
:10168000162221461B4D514301F593112846FCF7C4
:101690009CFD16212846F9F7FEFE0646344303D189
:1016A00016212846F8F7CEFFE87C697C01EB800123
:1016B00028786974FF280CBF00200120287030466C
:1016C00070BD0C4870470B48C17C007800EB4100AE
:1016D00000F5804080B2704780B506490A7D183118
:1016E000FFF7C0FD401E8041C00F02BD0248704799
:1016F0007C7D0020FC0700201408002073B59DF8B5
:1017000003409DF802605B4DF5F716FD38B9304691
:10171000F6F736FB28702046F6F732FB06E000208D
:10172000F7F787F828700020F7F783F868703046DD
:10173000F6F726FB28712046F6F722FB6871F6F7CC
:1017400040FEF6F71DFBA870F6F747FEF6F718FB0C
:10175000E870F4F772F830B1474900200870AA78B1
:10176000E8782A7068709DF80100BDE87640FCF7C3
:10177000E8BE38B53F4D044695F90000F6F7F0FA9B
:10178000A07095F90100F6F7EBFAE07031BD3A4828
:10179000384A0178491E8941C90F0170007830B17B
:1017A00092F9041092F905001170507003E092F95B
:1017B000021092F90300FBF77FBE2F4800787047B4
:1017C00070B5032884B0014602D10022002108E050
:1017D000062803D101220021284803E0012805D171
:1017E0000022244800F04CF8064629E0042832D1B3
:1017F000204D95F90100F6F7B3FA0A2202A9F9F78C
:10180000C1FD0026040013D0202207216846FAF704
:10181000EBF900BF3BA00268009202A92246644295
:101820000DEB0400801DF2F72BFB6846F2F716FC67
:1018300095F9010010F14E0F02DB401E6870012681
:101840004EB10C4890F9001090F90100FBF734FEFE
:10185000012004B070BD002004B070BD80B5FFF75A
:101860004DFF044890F9021090F90300BDE80440D0
:10187000FBF722BE6C6D0020BE7E00206D6D002047
:101880002DE9F0410546002684B0A8570F46904642
:10189000F6F766FA0A2202A9F9F774FD040018D0D7
:1018A000202207216846FAF79FF9B8F1000F0CBF14
:1018B0000FF248000FF24C0002A902680092224683
:1018C00064420DEB0400801DF2F7DAFA6846F2F785
:1018D000C5FB380004D1A8570F280ADA401C06E0DF
:1018E000012F06D1A85710F14E0F02DB401E2870C1
:1018F0000126304604B0BDE8F0810000C380C392E9
:1019000000000000C38FC38000000000DFF88825BE
:10191000DFF888350021118018800020DFF880155D
:10192000DFF880250870DFF88015DFF88005F3F711
:10193000E8BD38B50446F9F713F801280FD0DFF8F1
:101940007055E87A34B150B940F21460FBF7A5F84D
:10195000012003E018B1FBF7ADF80020E87231BDBB
:10196000DFF850057047DFF84815087A10B90622ED
:101970000A720BE006220A727047DFF834154872CB
:101980007047DFF82C05407A704700007CB5DFF81F
:101990002045DFF82455207A0E281ED8DFE810F005
:1019A0000F0025006F00EF00CF005401AD01DF00F4
:1019B000C3001D001D004D011D001D005E00F6F757
:1019C000EDFBE07140F6FF70FBF767F80120207235
:1019D000F5F7B2FB08B14FF47A752A46DFF8DC144C
:1019E00004F12400F3F78DFD73BDFBF745F8DFF834
:1019F000D014FEF707FEDFF8CC14FFF7B5F8F9F7BF
:101A00003BF821F0004104F0E1FA2062F5F78EFB8B
:101A100090B194F9001094F90100FBF74DFDF5F732
:101A20008BFB38B10520FBF75BFF94F90100FBF756
:101A30005BFD06E0032000E00120FBF751FFFBF710
:101A40002BFDFBF737F8F5F777FB10B10E2020726E
:101A5000C3E702212172DFF87054BEE70F20207225
:101A6000F5F773FB072807D001208DF8000001224D
:101A700069469720F9F758F842F21075ADE7607A99
:101A8000A8B9FAF7F9FFE169FBF7E4FB26D3FAF707
:101A9000F3FF0146A069FBF7DDFB38BF03261ED329
:101AA000FAF7EAFF2169FBF7D5FB15D20CE0FAF74C
:101AB000E3FF6169FBF7CEFB08D2FAF7DDFF0146D1
:101AC0002069FBF7C7FB01D2002608E0FAF7D4FF34
:101AD0002169FBF7BFFB01D2022600E00126304658
:101AE000F5F739FB18B10C20F5F7EAF9C4E73046F1
:101AF000F5F78BFA98B146B104202072F5F716FB82
:101B000000280CBF0620002002E0082020720420DC
:101B1000FCF7FEFCF6F728FBFFF7F8FE5DE70F2069
:101B2000F5F7CEF9A8E7E07920B907202072DFF8B1
:101B30009C5352E7401EE071DFF868534DE7DFF831
:101B400060030178012942F210757FF446AF00204E
:101B5000FCF7DEFC1020F5F7B3F9062077E7032148
:101B600021720920F5F7ACF9F5F7E0FA00280CBF6F
:101B700001200320FCF7CCFC42F210752DE7DFF8C2
:101B800020030178012942F2107507D10020FCF7EB
:101B9000BFFC1020F5F794F9062058E7FAF76CFF20
:101BA00001462069FBF756FB34BF01260026F8F7F3
:101BB00030FF00287FF411AF607A012807D1FAF7CF
:101BC0005BFF2169FBF746FBBFF407AF02E0002E85
:101BD0003FF403AFF6F7C8FAFFF798FE0220FCF7D0
:101BE00097FCF5F7A3FAB0B194F9001094F901004D
:101BF000FBF762FCF5F7A0FA38B10520FBF770FEA1
:101C000094F90100FBF770FC0EE00320FBF768FE7F
:101C1000FBF742FC08E00120FBF762FE94F900109C
:101C200094F90100FBF748FCFAF744FF0B202072FF
:101C30000A20F5F745F9A64DCFE605202072F6F704
:101C400082FAFFF763FE17E795480178012907D16B
:101C50000020FCF75DFC1020F5F732F90620F6E6CF
:101C6000207B38B9F5F762FA10B99A48F2F7F6F91D
:101C700001202073607AB8B9FAF7FEFE2169FBF7FC
:101C8000E9FA03D20C20F5F71BF9A4E6FAF7F4FE03
:101C900001466069FBF7DEFA04D20D20F5F710F972
:101CA0008D4D9AE68D4D98E6FAF7E6FE23690246D9
:101CB00018461146FBF7CEFA11D261691046FBF7C0
:101CC000C9FA0CD2A07A401CA072C0B264287FF47A
:101CD00082AE0C20F5F7F4F80020A0727BE6A07A23
:101CE000012807DD10461946FBF7B4FA02D200219D
:101CF000A172D2E74FF496756FE6F5F717FA28B19F
:101D00000020F3F76FF80020F5F70DFA0020F5F743
:101D1000D7F80220FBF7E4FD00F095F800202073CF
:101D200073BD38B5624C207A30B102282FD0032819
:101D300075D00D2859D084E0694800210180817058
:101D4000F5F7F4F990B194F9001094F90100FBF75C
:101D5000B3FBF5F7F1F938B10520FBF7C1FD94F9B4
:101D60000100FBF7C1FB06E0032000E00120FBF7C8
:101D7000B7FDFBF791FBFAF79DFE0220207204F1FC
:101D80002400BDE83840524A5649F3F7BABBF4F78D
:101D90007CFF102827D1FAF76FFE0146A069FBF7F8
:101DA00059FA09D2FAF768FE4D4DFEF788FB2880F4
:101DB0000120A87006200EE0FAF75EFEE169FBF74D
:101DC00049FA10D2FAF758FE454DFEF778FB288005
:101DD0000120A870052003212172F5F771F81E205B
:101DE000FFF794FDCBE70D20C8E7FAF745FE216920
:101DF000FBF730FA34BF07200820F5F761F803201D
:101E0000254A264B2072002111801E20244A18806A
:101E10001170244A24492548F3F773FBAFE72048A3
:101E20000178012904D11020F5F74AF80620A5E72A
:101E3000FAF722FE2A4DFEF742FB28800120A87007
:101E40009DE7BDE8314010B586B00020FCF760FB8F
:101E5000F8F7E2FD164C0020E072F8F77EFD6846C8
:101E6000FEF756FF9DF81000FF2804BF9DF81100F3
:101E7000FF280AD19DF81200FF2804BF9DF8130027
:101E8000FF2802D1FAF70BFE02E02820FAF705FE40
:101E90000020207206B010BDDE7C0020E07C002017
:101EA000DC7C002040420F00B9560008E47C002092
:101EB0006C6D00207C6D0020400D03008D19010821
:101EC000CDCCCC3D9A9959C2A0860100801A06005B
:101ED000E093040000AC0108C0C62D00F0490200E8
:101EE000A07E0020231D010890420CD141EA030C82
:101EF00050EA4C0C07D0994205D14FF4001C1CEB62
:101F0000410F38BF8942704710B5144600F002F8FF
:101F1000226010BDC1F30A5343B14A0012F5001FFD
:101F200028D2A3F2FE32A1EB0251704750EA410CD5
:101F300020D001F0004C31EA0C01B1FA81F204BF6B
:101F4000B0FA80F3D2180B3AB2F120032CBF00FA9A
:101F500003F1914041EA0C013EBFC2F1200C20FA8E
:101F60000CF319439040524240F2FD33D21A01EB78
:101F700003517047002270474FF4001C1CEB410FC7
:101F800094BF1CEB430F09E041EA030C50EA4C0CF0
:101F900052EA0C0C03D2994208BF9042704714BF1A
:101FA0008B42824270470000124254D440F2FF7CC0
:101FB0001CEA11530FD0634531D09B1863453CBFD9
:101FC00001EB0251704701F0004141EA0C51002041
:101FD000AFF30080704750EA410320D001F0004C7D
:101FE00091EA0C011CD0B1FA81F30B3B9A420DD956
:101FF000D21A994051EA0C01C3F1200C20FA0CFCD2
:1020000061449840531C40F2FF7CD7E7914041EA7D
:102010000C01C2F1200C20FA0CF3194390407047D8
:10202000B0FA80F31533202BE0D3202AEED3203AE8
:10203000203B9A4209D9D21A00FA03F141EA0C0175
:102040000020531C40F2FF7CB8E700FA02F141EA9D
:102050000C0100207047524240F2FF7C1CEA1153F1
:102060000DD06345DBD0B2EB030C3CBFA1EB0251BA
:1020700070470CF1010221EA035141F4801150EA4A
:10208000410CCCD001F0004C352A27DC30B481EA79
:102090000C01B2F1200309DAC2F12003044601FA6F
:1020A00003F5D0402843D1409C400CE0C3F120020E
:1020B000450020FA03F418BF44F0010421FA03F0AC
:1020C00091400C43002174F1004550F1000051EBA8
:1020D0000C01244230BC7FF47BAF70476146002086
:1020E00076E70000B0B581EA030C0CF0004C40F23A
:1020F000FF7515EA11541DBF15EA1357AC42AF42E4
:1021000039E0E41923EA455343F48013C90241F04E
:10211000004141EA505EC7021100A7FB02020028FD
:102120004FF00000EEFB01204FF00001E3FB072120
:1021300018BF42F00102401800214941E3FB0E01A3
:10214000A4F580640F0302D252004041494154F18A
:1021500001046CDD470872F1004250F1000051EBC0
:102160000451A1F580115CBF41EA0C01B0BD4CEAFD
:1021700005510020B0BD05EA1357AC4214BFAF4271
:1021800041E050EA410E1CBF52EA430E02E06146B4
:102190000020B0BD24423C441BD15FEA070EF6D0BC
:1021A000090302BF01460020AEF1140EB1FA81F717
:1021B000AEEB070401FA07FE0C37C7F1200100FA65
:1021C00007F7C8404EEA000E23EA455343F4801354
:1021D000A2E733F00043B3FA83F704BFB2FA82FEFA
:1021E00077440B3FE41BB7F1200E2FBF02FA0EF32A
:1021F000BB40C7F1200E22FA0EFE38BF43EA0E03A1
:10220000BA40641C82E750EA410E14BF52EA430E02
:102210006FF000014FF4001717EB430F8ABF194608
:1022200017EB410FB5E74CEA05510020B0BDD4F1E2
:102230000104B4F120070FDAC4F12007520828BFC7
:1022400042F0010210FA07F501FA07F7E1BF2A434D
:10225000E0403843E1400FE0352C98DCC7F1200422
:1022600052EA400220FA07F218BF42F0010231FAA6
:1022700007F0A1400A43002172F1004250F1000032
:1022800051EB0C01B0BD000070B44FF0004591EA75
:10229000030F40F1DD806B40841A71EB030604D21A
:1022A0006E40001BB141121973414FF4001C1CEB2E
:1022B000410F34BF7CEB430683E00C0DA4EB1356B7
:1022C000362E00F37C80012E45EAC32341DC43EA2D
:1022D000525312BFD20292025B08240545EAC12183
:1022E00041EA5051D2EBC020994125D407D1B0FA30
:1022F00080F610FA06F162D00020203608E0B1FA2C
:1023000081F6B140C6F1200220FA02F21143B0403A
:102310004FEAF474B4EB465434F001064FEA740407
:102320000AD8D6F50016760D04F00044F04061FAA4
:1023300006F25040F1404840C00A40EA415021F0C6
:10234000004128BF5FEA500550F1000044EBD12165
:1023500035E0DB0A45EAC121C90AB6F120050EDDE8
:1023600042EA0242120CC5F1200603FA06F6EB40DF
:1023700042EA06056D42984161F100010DE062FA02
:1023800006F5F240554063FA06FC82EA0C02F3407F
:102390005A406D42904161EB030111F4801F05D159
:1023A000641E620502D06D004041494121F4801154
:1023B000430875F1004350F1000041EB045170BC3B
:1023C00070471CEB410F15D223F0004352EA43063D
:1023D0000BD04FEA4C0CBCEB410F04D80C0D661E21
:1023E000342EB7DDEBE7801A994150EA410608BF69
:1023F0000021E4E708BF1CEB430F28BF6FF000018A
:10240000DDE70000C1F30A5340F2FE329B1A14DDEF
:10241000D3F120034FEAE17208DDC90241EA5051CD
:1024200041F00040D84080185040704703F2E1303E
:1024300010B1D24382F00040704700207047000086
:1024400070B44FF0004591EA030F7FF525AF6B4064
:10245000841A71EB030603D2001BB14112197341B8
:102460004FF4001C1CEB410F34BF7CEB430442E0F3
:102470000C0DA4EB1356352E4FDC45EAC323DB0AC3
:1024800045EAC121C912B6F120050DDD63FA05F652
:10249000EB4086EA0305124218BF45F00105C0185B
:1024A00051F100010CD213E062FA06F5F2405540FA
:1024B000F3415A40B340F3405A408018594107D382
:1024C00049085FEA30005FEA350528BF45F001059D
:1024D00001F58011420875F1004250F1000041EB16
:1024E00004514E0016F5001F70BC38BF7047002025
:1024F000090D090570471CEB410F10D252EA430643
:102500000BD0BCEB410F05D80C0DAB43661E342E2F
:10251000B6DD02E0AB438018594170BC704770BC17
:1025200070470000F0B540F2FF7581EA030C0CF033
:10253000004C15EA11541DBF15EA1357AC42AF42C7
:10254000E5E0BC41C1F31301C3F31303801A9941C1
:1025500043F4801304D2641E40004941801859415D
:10256000C90241EA5051B1FBF3F603FB1611A2FB7D
:102570000675D7EBC020A94102D2761E80185941BA
:10258000C90241EA5051B1FBF3FE03FB1E11A2FB4D
:102590000E75D7EBC020A94103D2AEF1010E801811
:1025A0005941890241EA9051760546EA8E2EB1FBE7
:1025B000F3F603FB1611A2FB0675D7EB8020A941A9
:1025C00002D2761E80185941C90241EA50514EEAA2
:1025D000060EB1FBF3F603FB1611A2FB0675D7EB53
:1025E000C020A94102D2761E80185941C90241EA91
:1025F0005051B1FBF3F703FB1711A2FB0735D3EBE7
:10260000C020A94167F100070CBF004247F0010755
:1026100066F3D5274FEA1E31B80814F5806412DD41
:10262000BD0775F1004250EB0E5051EB045111F50E
:10263000801F5CBF41EA0C01F0BD4CF07F6141F0AE
:10264000E0410020F0BDBD076D0840EA0E5041F4A6
:102650008011D4F10104B4F120060ADAC4F1200695
:102660000200E04001FA06F3E1401843B24015438E
:102670000EE0342C13DCC6F1200445EA40056D0859
:1026800020FA06F2154321FA06F0A1400D4300217D
:1026900075F1004250F1000051EB0C01F0BD00203B
:1026A0005FEA0C01F0BDCFB992185B41B3FA83F732
:1026B00004BFB2FA82F6BF190B3FB7F120062FBF55
:1026C00002FA06F3BB40C7F1200622FA06F638BF2D
:1026D0003343BA401CB1E419641E33E77F4231F042
:1026E0000041B1FA81F404BFB0FA80F6A4190B3CA2
:1026F000B4F120062FBF00FA06F1A140C4F1200674
:1027000020FA06F638BF3143A0403C1B1AE7AC4222
:102710001ABF05EA1357AF4212E050EA41061CBF48
:1027200052EA4306BFE750EA4107304661461CBF04
:1027300041EA0551F0BD52EA430C08BFC143F0BD68
:1027400000204FF4001616EB410F98BF16EB430F15
:1027500008BF16EB410F24BFC14305E016EB430F42
:102760000CBF61464CEA0551F0BD00004FF4001C5F
:102770001CEB410F94BF1CEB430F09E041EA030C33
:1027800050EA4C0C52EA0C0C03D28B4208BF824236
:10279000704714BF99429042704700002DE9F04DF8
:1027A000044648004015401C84B00D4616461F469E
:1027B00022D0CDE90245DDE9022322F0000033F00A
:1027C000004B08BF002817D078004015401C13D0DC
:1027D00026F0000037F0004B08BF00280CD0DDE9E0
:1027E000020100297BD54FF0000A4FF0004BBAEBF5
:1027F00000006BEB010172E048004015401C02D163
:102800000A0340F05581BC464FEA4C02521512F1C2
:10281000010E02D15FEA0C323FD132463B4622F034
:10282000000A33F0004B08BFBAF1000F03D1A0BB80
:10283000090332D108E0BEF1000F08BF5FEA0C388F
:1028400009D150BB090328D1AFF300804FF0FF300E
:102850006FF000412EE124F0000735F0004B08BF77
:10286000002F1DD1614648000C9C400D241808BB68
:102870000C9A3046FFF798FB06460F4626F00004F8
:1028800037F0004508BF002C05D078004015401CEB
:1028900003D1390301D1AFF300803046394609E155
:1028A000C8B9090317D12046294604B0BDE8F04D48
:1028B000FFF718BC002CDBDD40F2FF70844205DB23
:1028C0007E4F0CF0004000260743D7E76FF31E5100
:1028D00041EA0457D2E700200CF00041EAE0CDE9DC
:1028E000000100207649002944BF4FF0004B6BEBFC
:1028F0000101DDE900AB8B45B8BF07F00041C0F234
:10290000D9807049002944BF4FF0004B6BEB0101A7
:10291000DDE900AB594509DC01DB504506D2AFF3D8
:102920000080664907F000421143C3E066486749EA
:10293000FFF7D8FB664B01F0004213430022FFF77C
:10294000A3FCFFF75FFD8046F7F78EFA82468B46C1
:102950004FF078405F4952465B46FFF7C3FB0246A3
:102960000B4620462946FFF76BFD04460D465A48A4
:102970005A4952465B46FFF7B5FB02460B462046D6
:102980002946FFF75DFD0D4625F000410022544B1E
:10299000FFF7F2FA044602D234463D4652E02246A0
:1029A0002B462946FFF79EFB82468B464D484E49F3
:1029B00052465B46FFF796FB4C4A4D4BFFF764FCD3
:1029C00052465B46FFF78EFBCDE90201524649486D
:1029D00049495B46FFF786FB484A494BFFF754FCE1
:1029E00052465B46FFF77EFB0022394BDFF814B1FD
:1029F000FFF74AFC22462B46FFF774FB04460D46C0
:102A0000DDE9020122462B46FFF73EFC00225B4631
:102A1000FFF73AFCCDE900012246DDE902012B4631
:102A2000FFF70EFD00225B46FFF72EFC02460B4629
:102A3000DDE90001FFF776FD32463B46FFF752FB2A
:102A400004460D460C98294600EB08020B46580038
:102A5000400D02EB000610D0002E0EDD40F2FF709C
:102A6000864205DB154D01F0004100240D4310E0C6
:102A70006FF31E5343EA06550BE024F0000035F0D7
:102A8000004108BF002804D02946FFF78DFA04460C
:102A90000D4624F0000235F0004308BF002A05D09F
:102AA00068004015401C03D1290301D1AFF3008019
:102AB0002046294604B0BDE8F08D00000000F07FFC
:102AC00000C89CC000C89C40FE822B654715F73F9C
:102AD0000000E03F422EE63FF2E4D5BCE7E84B3E83
:102AE0000000903C112E5781A03F503F5843128C5C
:102AF0008F71BC3F4BE8A541B752013F0BBDF3DAE4
:102B0000E8708C3F0000F03F026822B112680A6052
:102B10000368196000E009600160704702461168AF
:102B200041B10868814202D10021116070470268FA
:102B30000A6070470020704740EA010C1CEB0C0F44
:102B400007D0884205D14FEA400C1CF1807F98BF26
:102B5000804270472DE9F14FB0B0924604910DF1DB
:102B600042013A9A2B9199464A7000200AE01AF8DD
:102B7000011B0498309A90470028049000F0A68624
:102B80000D98401C0D909AF8000050B12528EED108
:102B9000002100220791089209910A920B910C9250
:102BA00004E00D9800F094BE41F001011AF8010F05
:102BB0002028F9D023280CD02B2804D02D2805D08C
:102BC000302809D00BE041F00201EFE741F00401A9
:102BD000ECE741F00801E9E741F01001E6E72A28B7
:102BE0000FD1D9F8002052F8040BC9F800200028B2
:102BF0000F9003D540420F9041F004010AF1010A01
:102C000014E00F92DFF824380AE00F98984205DAB2
:102C100000EB800402EB4402303A0F920AF1010A01
:102C20009AF80020A2F130000A28EED39AF80000AA
:102C30002E2803D04FF0FF320E9229E01AF8010F30
:102C40002A2809D1D9F8000050F8042BC9F800004F
:102C50000E920AF1010A1BE02D280CBF0AF1010AAD
:102C6000002000220E92DFF8C4470BE040B90E9A14
:102C7000A24205DA02EB820503EB4503303B0E93DB
:102C80000AF1010A9AF80030A3F130020A2AEDD3C2
:102C9000ADF84010DFF89807784400F294709AF885
:102CA000001003F033FF08B11AF8010B8DF8420051
:102CB0009DF84200682805D19AF8000068280CD1D8
:102CC000622106E06C2804BF9AF800006C2804D149
:102CD00071218DF842100AF1010A12A806901AF823
:102CE00001BBBBF125012CD01C3900F0CF81091F9D
:102CF000022940F2CB81133900F01385093900F025
:102D0000C581891E00F0A885491E00F05585491E21
:102D1000022940F2BB81091F00F04E85491F00F0D7
:102D20002881491E00F0FD84491E00F0D080C91E94
:102D30000DD0891E00F0F584C91E00F0F28400F069
:102D400096BD25238DF84830012100F09BBDD9F8B0
:102D5000000050F8044BC9F80000002C059440F026
:102D6000A3802B994878002800F099804FF0FF3419
:102D70000FF6643003F0D6FE201A40F0A78500F06D
:102D800082BD6D1E40F099853096079D12AF75B1DA
:102D9000309E17F8012B02A9304600F063FE002890
:102DA00001D46D1EF5D10028309640F08F850A9D24
:102DB0003020002D8DF804000CDD309E012301AA87
:102DC00002A9304600F05EFE002840F07F856D1EAF
:102DD000F4D13096059F089D75B1309E17F8012BF0
:102DE00002A9304600F03EFE002801D46D1EF5D148
:102DF0000028309640F06A850B9D3020002D8DF81C
:102E000004000CDD309E012301AA02A9304600F027
:102E100039FE002840F05A856D1EF4D13096059891
:102E20000899099D471875B1309E17F8012B02A922
:102E3000304600F017FE002801D46D1EF5D10028A1
:102E4000309640F043850C9D3020002D8DF8040015
:102E50000CDD309E012301AA02A9304600F012FECB
:102E6000002840F033856D1EF4D130969DF8400067
:102E700041077FF588AE2020002C8DF804007FF7F5
:102E800082AE309D012301AA02A9284600F0FAFD76
:102E9000002840F01B85641EF4D1309573E60FF6D0
:102EA0004440059000F0EFBC0E9D002D04D5204657
:102EB000F3F7CCFE044607E02A46204603F052FE14
:102EC000002814BF041B2C46089400F0DCBCD9F881
:102ED000001051F8040BC9F8001020F00004002184
:102EE00021F0FF3512ABCDE902450593DDE9022360
:102EF00006993C2413B90AB90E9898B102F00F054F
:102F00003035641EEEB23A2EA8BF2735120942EAC8
:102F100003721B090D5508BF002A03D005980D192F
:102F2000A842EBD308190590C4F13C020E98089210
:102F300082420ADABDF84010821A4FF6EF70014063
:102F40000A92ADF8401000F09EBC002840F19B842E
:102F50009DF8400000F01400102840F094840F9B6E
:102F600007990A985B1A1B1A9A1A002A40F38B8455
:102F7000D5E32B99487820B14FF0FF340FF6343069
:102F8000F8E69DF84200622861D0682817D06A28C8
:102F90003FD06C2806D0712847D074282CD07A28CE
:102FA0001DD064E0D9F8001051F8040BC9F80010E6
:102FB000002868D14FF0FF340FF61030DAE6D9F868
:102FC000001051F8040BC9F8001020B94FF0FF347D
:102FD0000FF6F820CEE60D99018000F054BCD9F828
:102FE000001051F8040BC9F8001000284BD14FF025
:102FF000FF340FF6D820BDE6D9F8001051F8040BC5
:10300000C9F8001000283ED14FF0FF340FF6BC2065
:10301000B0E6D9F8001051F8040BC9F8001080B9D7
:103020004FF0FF340FF6A420A4E6D9F8001051F8B1
:10303000040BC9F8001020B94FF0FF340FF68C20B4
:1030400098E60D9AD317C0E9002300F01CBCD9F80C
:10305000001051F8040BC9F8001020B94FF0FF34EC
:103060000FF6682086E60D99017000F00CBCD9F8C7
:10307000001051F8040BC9F8001020B94FF0FF34CC
:103080000FF6482076E60D990160FCE3D9F80020A0
:10309000D21D22F00702C9F80020D2E9000108324F
:1030A000C9F80020CDE90201C80F02D007982D21F0
:1030B0000AE0BDF84000810702D507982B2103E004
:1030C000C00705D50798202112AA1154401C07906B
:1030D00012A807994BF020024318DDE90201CDE95F
:1030E0002C01612A059321AC0BD00E98002802D543
:1030F00006200E9005E001BF4BF02000672801215B
:103100000E91DDE9020148004015401C0A460DD130
:1031100009030BD0ABF1610503201A2D089002D2F0
:103120000FF6C4110DE00FF6C4110AE070B91203D6
:103130000CD1ABF1610503201A2D08901AD30FF6BC
:10314000B41103221846F0F79BFE9CE3DDE902016F
:10315000CDE92E01DDE92E2323F00047B7F5801FCE
:1031600022F000060DD20022002F08BF002E009290
:1031700003D116E00FF67811E3E76A46FEF7C4FEC6
:103180000FE0DFF8C008DFF8C01800EB1750009020
:10319000DDE92E234FF0FF301940DFF8B078104002
:1031A0003943CDE902014BF0200061280DD105988B
:1031B00030210170821CBBF1610F05920CBF782198
:1031C000582141700798801C0790DDE9020120F02A
:1031D000000231F0004308BF002A02D1002600257A
:1031E00068E14BF02008B8F1610F40F0B4800E9810
:1031F000002847BF21210191401C0190019FDDE97A
:103200002C017F1C00220023DDE90245FEF7B4FEFD
:1032100000998DF8842038BF85F00045091F002FE4
:1032200000910DF1850653DD20462946002200233A
:10323000FFF79CFA4CD24800400D00F11C0312D05D
:10324000002B10DD40F2FF70834206DBDFF8001830
:1032500005F000421143002011E06FF31E5141EAD6
:10326000035120460BE024F0000035F0004108BF78
:1032700000280FBF29461C222946FEF795FE04466A
:103280000D46FFF7BFF8FF1F002F804609DDF6F758
:10329000EBFD02460B4620462946FFF7D1F80446CF
:1032A0000D46F01D0721B8F1000F0CDD491E5EBF71
:1032B00008F00F0200F8012D4FEA2818F3D502E0BC
:1032C000002200F8012D491EFAD5C61D002FABDCE7
:1032D0000DF18500361A01988642D8BF3046002885
:1032E0000DF1850430D4B04206DA0DF185010A5C97
:1032F000082AA8BF0F2100DA0021024621AB13449F
:1033000000E0401E13F80159521E8D42F9D00F29DA
:1033100004D10DF185018B5C5B1C8B54002A04D514
:103320000099091D21AC401C0091411E0CD462186B
:10333000ABF13A0613783033DDB23A2DA8BFF3185B
:10334000491E02F80139F5D50E99002940F1B080E7
:10335000421E0E92ACE00099DFF8F82647F2975033
:10336000414391FBF2F2DDE92C45009225F0004546
:10337000D2F1070204DD2046294600F040FB0BE0B5
:1033800052420020DFF8D01600F039FB02460B460F
:1033900020462946FFF7C6F80446B8F1660F0E9896
:1033A00006BF009F0A3706273F18142FC8BF1427EF
:1033B00030200D468DF884000DF18506002F39DD93
:1033C00020462946F7F70CF901460A4606F108039C
:1033D00004200A26B2FBF6F606EB860EA2EB4E029E
:1033E000303203F8012C0A22B6FBF2F202EB820E15
:1033F000A6EB4E063036401E03F8026DE9D1083FB9
:10340000002F03F10806D9DD084603F0D7FB02467A
:103410000B4620462946FFF713F80022DFF83C361A
:10342000FEF760FE04460D46CAE700BFCBCCCC0CCD
:10343000387800000DF18500361A0DF1850404E09E
:103440000098401E761E0090641C20783028F7D02B
:10345000B8F1660F02D10099491C04E0B8F1650F7C
:103460000CBF012100210E9808188642B8BF701EBB
:1034700000281DD4B04204DA215C3429C8BF3921A8
:1034800000DC30210246631E9D1800E0401E15F846
:103490000169521E8E42F9D0392902D1A15C491C22
:1034A000A154002A04D50099491C1C46401C0091D7
:1034B0000646009D0E9F30B2002802DC01260FF266
:1034C00038644BF02000662808BF6D1C15D06728B3
:1034D0000FFA85F841D118F1040F44DBB84542DA00
:1034E0009DF840006D1C010703D430B2B842B8BF4C
:1034F000074628B23F1A48BF00270FFA85F8B8F1EF
:10350000000F00F3AF800898411C08913022059904
:103510000A54002F03DC9DF84000010705D50898E8
:10352000411C08912E2205990A5417EB080FB8BFC9
:103530007D4228B2C51932B2414295420B91B8BFC3
:103540002E46059B089836B2099632462146184405
:10355000F0F796FCAD1B0C95CCE0BBF1610F15D1DB
:103560004FF0700B17E030B2B84204DA9DF840100B
:103570000A0758BF07467F1E48BF0027BBF1670FE9
:1035800014BF4FF0450B4FF0650B04E0BBF1410F4A
:1035900008BF4FF0500B0898411C0891002F059967
:1035A00014F8012B0A5403DC9DF84000010719D5DB
:1035B0000898411C08912E2205990A54002F11DD0C
:1035C000761E30B287420598089BB8BF3E4632B29D
:1035D00021461844F0F754FC089836B23018BF1B47
:1035E00008900B97059808990844B8F1000F80F8E7
:1035F00000B003D42B224270821C04E02D214546EA
:103600004170821C6D4200212CAB28460AE0044622
:103610000A2094FBF0F000EB8005A4EB450403F8CE
:10362000014B491C00B20028F1DC012906DC4BF0FB
:103630002000652804BF302002F8010B00292CABC4
:1036400008D1302002F8010B06E0491E585C3030EA
:1036500002F8010B0029F8DC059908980844121AB1
:10366000099247E030B229B288421BDA0598089BDC
:1036700032B221461844F0F703FC089936B27118AB
:10368000A8EB0606002F08910B9603DC9DF840007E
:10369000020705D5059A2E2050540999491C099115
:1036A0000C9727E00598089B2AB221461844F0F7AA
:1036B000E7FB0898761B4044002F089003DC9DF838
:1036C00040100A0704D5411C08912E2205990A547E
:1036D00030B287420598089BB8BF3E4632B204EB31
:1036E00008011844F0F7CCFB089836B23018BE1B1E
:1036F00008900B969DF8400000F01400102840F050
:10370000C280079A08990B988A18099982180C9810
:103710008A1882180F98824280F2B580821A0A9223
:10372000B1E09DF84200622808D068280ED06A28CF
:1037300014D06C281FD0712810D01CE0D9F80010CC
:1037400051F8040BC9F80010C0B21AE0D9F8001003
:1037500051F8040BC9F8001080B212E0D9F800202B
:10376000D21D22F00702C9F80020D2E90001083278
:10377000C9F8002006E0D9F8001051F8040BC9F888
:1037800000100021CDE902019DF8400001075AD543
:10379000DDE90223002B08BF002A54D04BF02000A3
:1037A000782850D1079812A930220A54401C431C93
:1037B000079301F800B046E09DF84200622808D067
:1037C00068280ED06A2814D06C281FD0712810D019
:1037D0001CE0D9F8001051F8040BC9F8001040B2F1
:1037E0001AE0D9F8001051F8040BC9F8001000B223
:1037F00012E0D9F80020D21D22F00702C9F80020FB
:10380000D2E900010832C9F8002006E0D9F800101A
:1038100051F8040BC9F80010C117CDE902010029C5
:1038200002D507982D210AE0BDF84000810702D596
:1038300007982B2103E0C00705D50798202112AA7D
:103840001154401C079012A807990144059102A841
:10385000594600F04FF816E001200790D9F8000013
:1038600050F8041BC9F800008DF848100BE0252122
:103870000122BBF1000F8DF84810079203D08DF89C
:1038800049B0022107910F9A07980A990C9C121AC5
:103890000898521A0B99121A0998521A121A9DF87E
:1038A0004000141B41073FF570AA2020002C8DF822
:1038B00004007FF76AAA309E2546012301AA02A9C7
:1038C000304600F0DFF800283FF45BAA4FF0FF30ED
:1038D00031B0BDE8F08F00007072696E74665F737E
:1038E0003A2062616420257320617267756D656E90
:1038F000740000002DE9FC4307466F293E6908BFAC
:10390000082405D041F02000782814BF0A24102490
:103910003C25D7E90023642918BF692990469946B8
:1039200005D1002B03D5D8F1000869EB4909B9F19D
:10393000000F08BFB8F1000F0CD1386B50B9082C3C
:1039400039D197F83800010735D530203B2586F866
:103950003B0030E08DF80010404649462246E31710
:1039600003F03AF93032D0B26D1E3A28019504DBEB
:103970009DF80000A0F151018A1872554046494651
:103980002246E31703F028F980465FEA010908BFE1
:10399000B8F1000F03D0F86871198842DCD3082C05
:1039A00009D197F83800010705D5705D302802D09D
:1039B0006D1E30207055C5F13C02BA617119F96075
:1039C000386B824208DA821A3A624FF6EF70398F0A
:1039D00001403987BDE8F38300280ED597F83800F9
:1039E00000F01400102808D17B6B7969386A5B1AE3
:1039F0001B1A9A1A002AC8BF3A62BDE8F3832DE960
:103A0000D04306460F4614464FF00008DFF85090AA
:103A100012E0E00707D542464B4630463946FEF7EE
:103A200061FB06460F464046494642464B46FEF776
:103A300059FB641080468946002CEAD1304639464D
:103A4000BDE8D08302FCFFFFFFFF0F800000E03FD6
:103A50000000F07FA08601000000F03F84D797416E
:103A60000000244010B503460C461146A068984754
:103A7000A06020B1E06A401CE062002010BD4FF061
:103A8000FF3010BDF8B505460E4617461C4600200F
:103A90005CB117F8011BB068A847B06030B1F06A9C
:103AA000401CF0620020641EF3D1F2BD4FF0FF30E5
:103AB000F2BD00007072696E74665F733A20256E05
:103AC00020646973616C6C6F776564007072696EF5
:103AD00074663A2062616420256E20617267756D9C
:103AE000656E7400000000006E616E004E414E0075
:103AF000696E6600494E4600300000001A48704763
:103B00001A48704704210170194870470146194846
:103B1000416070470B681278D318C0185FEA005CE8
:103B200008BF03460B60704738B504460D4655EA9A
:103B3000040005D11048F1F75EF9FAF75CFB0CE0E0
:103B4000A54201D2022032BDAC4206D22046FAF78D
:103B50003EFB04F58054AC42F8D3F4F735F9FDF799
:103B6000B5FB002032BD0000D8480020587E002060
:103B7000F8070020707E002064AB010880B5F4F7E0
:103B800023F9BDE80140FDF7A1BB000010B5974C3B
:103B90009749A1600022A276C4F81B0002F0C4FB82
:103BA0004FF0006003F04CF9A07670B94FF0082098
:103BB00003F046F9A07640B98E4803F041F9A076AB
:103BC00018B98D4803F03CF9A076A07E20B904F125
:103BD0002401BDE81040E7E00520D4F81B10A076D2
:103BE000BDE81040084770B5804C8449A068884201
:103BF0000CD303220020A27684F8200003F004F9FD
